:100000000C94910E0C94C20E0C94C20E0C94C20E61
:100010000C94C20E0C94C20E0C94C20E0C94C20E20
:100020000C94C20E0C94C20E0C94C20E0C94C20E10
:100030000C94C20E0C94C20E0C94C20E0C94C20E00
:100040000C94C20E0C94C20E0C94C20E0C94C20EF0
:100050000C94C20E0C94C20E0C94C20E0C947092AE
:100060000C94C20E0C94EE6F0C94C46F0C94C20EE0
:100070000C94C20E0C94C20E0C94C20E0C94C20EC0
:100080000C94C20E0C94C20E0C94C20E0C94C20EB0
:100090000C94C20E0C94C20E0C94C20E0C94E4206C
:1000A0000C94C20E0C94C20E0C94C20E0C94C20E90
:1000B0000C94C20E0C94C20E0C94C20E0C94C20E80
:1000C0000C94C20E0C94C20E0C94C20E0C94C20E70
:1000D0000C94C20E0C94C20E0C94C20E0C94C20E60
:1000E0000C94C20E07634236B79BD8A71A396856DC
:1000F00018AEBAAB558C1D3CB7CC5763BD6DEDFD4A
:10010000753EF6177231BF000000803F0800000006
:10011000BE922449123EABAAAA2ABECDCCCC4C3EFC
:1001200000000080BEABAAAAAA3E00000000BF00EB
:100130000000803F0000000000084178D3BB4387E7
:10014000D1133D190E3CC3BD4282AD2B3E68EC82FB
:1001500076BED98FE1A93E4C80EFFFBE01C4FF7F80
:100160003F00000000000C940D720C94F4630C949A
:10017000B2130C94F72A0C9450730C94035C0C94F7
:10018000AF2B0C94234E0C947C1B0C94122B0C94D0
:10019000135C0C948E670C9427110C94082A0C9411
:1001A0005DA40C9443660C9485130C945D110C941F
:1001B000AC2C0C940F110C9447710C94864C0C943D
:1001C000EA850C94B9750C94294E0C9408290C946A
:1001D000D4710C9463110C94C2710C940D860C9420
:1001E00057890C94412A0C9435140C9443890C942F
:1001F0008F750C94ED640C94572C0C9482160C940F
:10020000174A0C945D390C94EC2B0C9495670C9464
:10021000D5660C94C4670C94C7740C948EA90C9486
:10022000B8A90C94BA100C94344A0C94F90E0C949E
:1002300035890C942B7C0C94772C0C94BA2C0C9450
:10024000C62C0C944D890C9485120C94FBA80C942C
:10025000D1650C94DC0E0C94D34C0C941B650C945F
:10026000DC160C9421540C9473120C94DA670C94E1
:100270005A590C943E650C942F360C94004D0C94F6
:100280007C690C940D0F0C9488680C94EE850C948A
:100290009A2C0C9424890C942C2B0C944C650C9463
:1002A000938E0C94DE6E0C9451A30C9436110C9426
:1002B0001B390C94254A0C9437120C9416890C9413
:1002C0002B890C940B4A0C94BA2B0C942F2B0C9466
:1002D0007B110C947D4D0C943B890C9431890C94CA
:1002E0006A360C94D0850C94710F0C94C71A0C9438
:1002F000B6170C9489660C942F110C9484650C9499
:10030000FA170C9485140C94E30E0C9478710C94E9
:10031000FB2B0C94FA8E0C94BC660C9472170C9404
:10032000431B0C943C660C94EE640C9461710C9429
:1003300018110C949F4C0C941A4A0C94689C0C94C1
:10034000412C0C94950F0C94452B0C94FA670C944B
:1003500022660C9469120C94FC280C94ED5C0C94AD
:100360004F9A0C94D6540C94D02B0C94D7850C94A3
:10037000964D0C941C890C94CD390C9487A80C9440
:10038000D5130C9456110C942A5A0C94E81B0C9417
:10039000504C0C9481120C9451890C94C12C0C94E7
:1003A000194D0C94CD490C945A690C940D2F0C9452
:1003B00049890C949C0F0C94F92B0C94634A0C946F
:1003C000720F0C94DB640C94B4690C9452670C9417
:1003D0002B2C0C940B2D0C9443670C9495160C94B9
:1003E0005E680C94D9130C943B290C94C40E0C94A5
:1003F000038F0C94CB4D0C9436490C9446660C94A8
:10040000191D0C94A29E0C947B470C9427860C9487
:100410002F0F0C9412680C941A4C0C94802C0C9492
:100420002A650C94D62C0C940FA90C945B890C941F
:1004300049120C94EA690C94F3130C94264E0C9414
:1004400070130C94AAA90C9401A90C942D0F0C9470
:1004500030120C94AD390C94C80E0C947EA10C94FF
:10046000284A0C94E1490C94820F0C94FD120C94D0
:100470003F890C9427670C94C90F0C948E360C940A
:10048000230F0C944C360C94A89E0C94F1390C94C8
:10049000C6390C9473490C94F0280C94CC0E0C942F
:1004A00070750C944C660C9456890C9431A90C947C
:1004B000E61A0C940D2D0C94040F0C94CC280C947B
:1004C000F4490C94242A0C948A120C94442D0C9414
:1004D00028890C941B2C0C945B4D0C9487120C9463
:1004E000642D0C948A390C9480AB0C947C670C942A
:1004F00020890C94B3360C9458710C946C110C94A4
:10050000A1290C94C8100C94730F0C94D72C0C9444
:10051000A8160C94B8290C94A35C0C94FD8E0C9432
:100520004A4E0C94A51C0C940C0F6364696E6F709A
:10053000737578585B002F00496E3A20003D0049E2
:100540004E3A003D004C454741435920494E3A0040
:10055000000020002300260029002C002F0032007C
:10056000000100000301060109012D3E00200023C7
:10057000002D3E00200050656E6465643A20230023
:100580007261770076616C0074656D7000736174E0
:10059000006875650066616E005247420048535618
:1005A000006D6F646500536574436D643A00537465
:1005B0006F726564204558543A00737566666978B1
:1005C000436F64653A004452590046414E5F4F4EB6
:1005D0004C5900584F4E0048414C54002074696DEE
:1005E000653A004374726C205265733A002054538C
:1005F0003A0020543A003D0050696E3A004F4E3A9E
:10060000416C7265616479204163746976650A00A2
:1006100048414C543A416C726561647920496E617D
:1006200063746976650A00584F4E3A416C72656191
:100630006479204163746976650A00584F46462004
:10064000736B69707065642E205072657620636DDF
:10065000643A005475726E6564206F666620667237
:100660006F6D3A00526573746F7265642066726FC5
:100670006D3A0049676E6F7265642C206368616E25
:100680006E656C20636D643D0020457865633A00BB
:100690004163746976653A0048414C543A416C7242
:1006A0006561647920496E6163746976650A0058F2
:1006B0004F4E3A416C72656164792041637469768A
:1006C000650A00584F464620736B69707065642E4A
:1006D000205072657620636D643A005475726E65C1
:1006E00064206F66662066726F6D3A00526573749F
:1006F0006F7265642066726F6D3A00206D73203AE8
:100700000041726D656420666F7220002044697339
:1007100061726D6564004F75744F664D656D6F72E3
:1007200079210A0020436D643A00205375623D0030
:10073000204974656D3D0052414D3D00282D292012
:1007400000282B2920002076616C756520697320B4
:100750000020756E6B6E6F776E0A005D3D005B006A
:1007600020696E76616C6964002000206F6B003A2E
:1007700000206661696C6564003A005265747279A4
:10078000696E67206D6F6462757320434D440A0083
:10079000207365632072656D61696E696E670053D1
:1007A00074617475732064656666657265640A00B9
:1007B00020002D3E00436F6E76657274696E67206F
:1007C000002D3E0057726F6E672041737369676E2C
:1007D0006D656E742000524742783A2000485356A7
:1007E0002064697361626C65640020764C6576658F
:1007F0006C3A0020436F6E76563A0020436F6E7657
:10080000533A0020486F743A00436F6C643A0020FA
:10081000436F6E76657274656420563A00436F6E5E
:1008200076657274656420533A002D3E0057726FEE
:100830006E672041737369676E6D656E7420002D5D
:100840003E0057726F6E672041737369676E6D6506
:100850006E74200053617665643A00000000000069
:10086000000000004F4E000000000000004F464610
:1008700000000000000052455354000000000054E6
:100880004F47474C4500000048414C5400000000D1
:1008900000584F4E000000000000584F4646000030
:1008A000000000494E4352454153450044454352E0
:1008B0004541534500484541540000000000434F66
:1008C0004F4C00000000004155544F000000000054
:1008D00046414E5F4F4E4C590044525900000000B3
:1008E000000053544F5000000000004849474800A2
:1008F000000000004D454449554D0000004C4F5745
:100900000000000000005452554500000000004661
:10091000414C534500000000454E41424C454400C7
:100920000044495341424C454400524742000000B4
:100930000000004853560000000000002053756678
:10094000663A002041543A00436F6E66696720633F
:1009500068616E676564206C6F63616C6C792C20D4
:10096000706F7274616C2064697361626C6564009D
:100970002F636F6E6669672E6A736F6E00726562B1
:100980006F6F742000436D643A20002F636F6D6DAC
:10099000616E642F002F72616D2F002F6974656D79
:1009A0002F002F6974656D2F004C6F636174696F40
:1009B0006E3A20687474703A2F2F6C617A79686F80
:1009C0006D652E72752F707761003F6D61633D001C
:1009D0002669703D0026706F72743D00266E616D51
:1009E000653D002F002000536B697070696E672EA3
:1009F0002E004F75744F664D656D6F727921005DE5
:100A000020003A5B000A003A004D41433A00554449
:100A100050205379736C6F6720696E697469616CDB
:100A2000697A65642E0A005379736C6F6720706170
:100A300072616D733A003E003C00543A0043757297
:100A400072656E74204C414E20636F6E6669672834
:100A500069702C646E732C67772C7375626E657485
:100A6000293A000A55736520746865736520636FC1
:100A70006D6D616E64733A202768656C7027202D58
:100A8000207468697320746578740A276D61632027
:100A900064653A61643A62653A65663A66653A3019
:100AA00030272073657420616E642073746F7265E3
:100AB000204D41432D6164647265737320696E201B
:100AC000454550524F4D0A276970205B69705B2C79
:100AD000646E735B2C67775B2C7375626E65745DF7
:100AE0005D5D5D27202D20736574207374617469CA
:100AF000632049500A277361766527202D20736192
:100B000076652063757272656E7420636F6E6669B8
:100B10006720696E204E5652414D3B204F4E7C4F10
:100B20004646202D20656E61626C652F6469736195
:100B3000626C65206175746F736176650A276765FD
:100B40007427205B636F6E66696720616464725D01
:100B500027202D2067657420636F6E6669672066A5
:100B6000726F6D207072652D636F6E666967757246
:100B700065642055524C20616E642073746F7265F9
:100B800020616464722C204F4E7C4F4646202D20FD
:100B9000656E61626C652F64697361626C65206467
:100BA0006F776E6C6F6164206F6E20737461727406
:100BB00075700A276C6F616427202D206C6F61644B
:100BC00020636F6E6669672066726F6D204E5652A5
:100BD000414D0A2770776427202D20646566696E71
:100BE0006520616E642073746F7265204D5154549A
:100BF0002070617373776F72640A276F7461707706
:100C00006427202D20646566696E6520616E64200E
:100C100073746F72652048545450204150492070BD
:100C2000617373776F72640A276C6F67205B7365FB
:100C30007269616C5F6C6F676C6576656C5D205B7B
:100C40007564705F6C6F676C6576656C5D27202DD1
:100C500020646566696E65206C6F67206C657665DB
:100C60006C2028302E2E37290A276B696C6C2720C0
:100C70002D2074657374207761746368646F670AEC
:100C800027636C65617227202D20636C656172207B
:100C9000454550524F4D0A277265626F6F74272089
:100CA0002D207265626F6F7420636F6E74726F6C4B
:100CB0006C657200536F6674207265626F6F746941
:100CC0006E672E2E2E0052414D3D000A312D776960
:100CD000726520000A6D71747420000A696E707567
:100CE000747320000A6974656D7320000A436F6E87
:100CF000666967757265643A0020416464723A00FF
:100D000064657623000944533234383220657272A8
:100D10006F720009526573657420646F6E65000917
:100D2000436865636B696E6720666F7220312D576B
:100D300069726520646576696365732E2E2E0044A2
:100D400053323438322D3130302070726573656E15
:100D500074004572726F7220312D7720696E69744C
:100D600020233220467265653A0077737461742ED1
:100D700020467265653A005465726D2E2046726594
:100D8000653A004572726F7220312D7720696E6965
:100D90007420233100467265653A0044533234387A
:100DA000325F3130305F4932435F544F5F31575FBC
:100DB00042524944474520696E6974003B003D003A
:100DC00050696E3A003B003D4C4F570054686572C5
:100DD0006D6F3A004F6E65207769726520526561CC
:100DE00064790A004170706C79696E6720636F6E78
:100DF000666967004C6F6164656420455441473AF9
:100E0000004E6F2073746F72656420636F6E666945
:100E100067004C6F616465642066726F6D204545A4
:100E200050524F4D006C6F6164206661696C65645F
:100E3000004C6F6164696E6720436F6E666967205E
:100E400066726F6D20454550524F4D00436F6E6680
:100E50006967206175746F736176653A000A53792A
:100E6000736C6F67206465627567206C6576656C6E
:100E70003A0053657269616C206465627567206C25
:100E80006576656C3A0053617665640A0053657453
:100E90002064796E616D69632049500A00454550B0
:100EA000524F4D20636C65617265640A004D515468
:100EB000542050617373776F72642075706461742D
:100EC00065640A004F54412050617373776F7264F8
:100ED00020757064617465640A00636F756C6420CA
:100EE0006E6F742070617273653A20005570646192
:100EF0007465640A004E6F20495020616472657306
:100F0000730052656C656173696E6720736F636B04
:100F1000657420616E64207265747279002053617B
:100F2000766564004C6F6164696E67204854545064
:100F300020636F6E666967206F6E207374617274D0
:100F400075703A004F4646004F4E002B002D00456D
:100F50005461673A200047657420455441473A2060
:100F600000485454502F312E312025690025733A02
:100F70002025730D0A0020485454502F312E310D76
:100F80000A486F73743A2025730D0A4163636570D4
:100F9000743A202A2F2A0D0A436F6E6E65637469B6
:100FA0006F6E3A20636C6F73650D0A002573002025
:100FB000000D0A00474554006661696C6564207441
:100FC0006F20636F6E6E6563740A004552524F5214
:100FD0003A205365727665722072657475726E651B
:100FE000642000436F6E666967206E6F74206368CB
:100FF000616E6765640A00446F6E652E0A00436F78
:101000006E6669672070617273696E6720666169D8
:101010006C65640A00676F7420436F6E6669670AC7
:1010200000667265652000436F6E666967205552E1
:10103000493A20687474703A2F2F00204465666125
:10104000756C7420636F6E66696720736572766570
:101050007220757365643A20006C617A79686F6DEF
:10106000652E7275000A282D294D444E53000A281A
:101070002D2955415254425249444745000A282BD4
:10108000295359534C4F47000A282D2950494400F1
:101090000A282D294D43503233303137000A282D8C
:1010A000294152544E4554000A282B294F544100DF
:1010B0000A282D29535049204C4544000A282D293F
:1010C0004D4F544F5220435452000A282D2941437A
:1010D000204841494552000A282D294343533831BD
:1010E0003120262048444331303830000A282B294B
:1010F000524553544152545F4C414E5F4F4E5F4DE9
:101100005154545F4552524F5253000A282D2948DA
:1011100041524452455345542C207573696E6720E3
:10112000736F6674000A282D29434F554E5445525B
:10113000000A282D29444854000A282B294F5749D2
:101140005245000A282D294D4F44425553000A2884
:101150002D29444D58000A282B2957697A6E657449
:1011600035313030000A282B294453323438322D9F
:10117000313030000A282B294672656552616D2096
:101180007072696E74696E670064653A61643A6290
:10119000653A65663A66653A6566000A4669726D43
:1011A00077617265204D41432041646472657373B9
:1011B00020006C617A79686F6D652E7275000A4344
:1011C0006F6E666967207365727665723A000A28E9
:1011D0002B295741544348444F4700323031313076
:1011E000334C0020432B2B2076657273696F6E3A67
:1011F00000313834616265665F323032312D313210
:101200002D3235000A4C617A79686F6D652E7275E2
:10121000204C6967687448756220636F6E74726FE2
:101220006C6C65722000204F464600204F4E002017
:1012300042595041535300757074696D6500667270
:10124000656568656170002054696D65723A0020BB
:101250004C6F636B733A002000204C6F636B733AE2
:10126000000A52414D3D0020457870697265640A5C
:1012700000202D746172676574207A6F6E652D0091
:1012800020416C61726D20457870697265640A0056
:1012900020636D643A00204375723A0020536574F0
:1012A0003A00536176656420746F20454550524F73
:1012B0004D00536176696E6720636F6E66696720C3
:1012C000746F20454550524F4D2E2E0020697320DB
:1012D0000044656C6574696E6720636F6E662E20CE
:1012E00052414D207761733A0053746F707065649A
:1012F0000053746F7070696E67206368616E6E650D
:101300006C73202E2E2E004E6F7420756E6C6F63E2
:101310006B656420696E20313073202D20636F6E01
:1013200074696E7565202E2E2E00556E6C6F636B82
:10133000696E6720636F6E666967202E2E2E00200F
:10134000416464723A00646576230020616C6976BA
:101350006500204E6F64653A00312D776972652013
:10136000636F756E743A2000312D77697265207352
:10137000686F72746564005B305D3A2000202D2038
:101380002D202D20EFBBBF003E003E31202D200040
:1013900020002E00696E00735F6F7574006D7968B0
:1013A0006F6D6500202D3E2000456D69743A200068
:1013B000202D3E20004974656D436D643A20002065
:1013C0002D3E20004974656D3A2000005EBCE2614C
:1013D0003FDD83C29C7E20A3FD1F419DC3217FFC76
:1013E000A2401E5F01E3BD3E6082DC237D9FC142BF
:1013F0001CFEA0E1BF5D0380DE3C62BEE0025CDF5C
:1014000081633D7C22C09E1D43A1FF4618FAA4279C
:10141000799BC584DA3866E5BB5907DB856739BA3D
:10142000E406581947A5FB7826C49A653BD987047A
:101430005AB8E6A7F91B45C6987A24F8A6441A9923
:10144000C7257B3A6486D85B05E7B98CD2306EED50
:10145000B3510F4E10F2AC2F7193CD114FADF3700D
:101460002ECC92D38D6F31B2EC0E50AFF1134DCE26
:1014700090722C6D33D18F0C52B0EE326C8ED053F3
:101480000DEFB1F0AE4C1291CF2D73CA947628AB0C
:10149000F517490856B4EA6937D58B5709EBB536C5
:1014A000688AD495CB2977F4AA4816E9B7550B88F2
:1014B000D6346A2B7597C94A14F6A8742AC89615AB
:1014C0004BA9F7B6E80A54D7896B35436F6E6E6542
:1014D000637465642E00436F6E6E2E2061626F72BE
:1014E000746564003E3E2000496E76616C6964203C
:1014F000636F6D6D616E64003E3E3E004E6F204D29
:10150000414320636F6E666967757265643A207344
:101510006574206669726D776172652773204D412D
:10152000430A004E6F2076616C6964204545505235
:101530004F4D20646174612E20496E697469616C3D
:10154000697A696E672E00476F7420495020616484
:1015500064726573733A00276970205B69705B2C55
:10156000646E735B2C67775B2C7375626E65745D5C
:101570005D5D5D27202D207365742073746174692F
:10158000632049500A004661696C656420746F20CD
:10159000636F6E6669677572652045746865726E03
:1015A0006574207573696E6720444843502E205936
:1015B0006F752063616E20736574206970206D61A2
:1015C0006E75616C6C7921000A75736573204448EF
:1015D00043500A00204D41534B3A002047573A00F0
:1015E00020444E533A004C6F616465642066726F0C
:1015F0006D20666C6173682049503A0053746172C3
:1016000074696E67206C616E0041424344454647F1
:1016100048494A4B4C4D4E4F5051525354555657D2
:1016200058595A6162636465666768696A6B6C6D74
:101630006E6F707172737475767778797A30313233
:10164000333435363738392B2F3D004261736963A7
:10165000200061726475696E6F3A004F54412069D1
:101660006E697469616C697A65640A004445464133
:10167000554C542070617373776F726420666F727B
:10168000204F5441204150492E20557365206F74DE
:101690006170776420636F6D6D616E6420746F207C
:1016A0007365740070617373776F72640075707422
:1016B000696D652C66726565686561700024737478
:1016C00061747300313834616265665F3230323183
:1016D0002D31322D3235004C6967687448756220AF
:1016E00000246E616D6500726561647900546F6FEE
:1016F000206D616E79204D51545420636F6E6E657C
:101700006374696F6E206572726F72732E205265FA
:101710007374617274204C414E00207472792061A0
:101720006761696E20696E2035207365636F6E6432
:1017300073006661696C65642C2072633D004177BB
:10174000616974696E6720666F7220726574616981
:101750006E656420746F7069637300636F6E6E658D
:10176000637465642061732000202E2E2E00207586
:101770007365723A003A000A417474656D70746959
:101780006E67204D51545420636F6E6E65637469AB
:101790006F6E20746F200024737461746500646937
:1017A00073636F6E6E6563746564005573696E670D
:1017B000204D5154542070617373776F72642066AA
:1017C000726F6D20636F6E6669670044657669634A
:1017D00065204E616D653A004174206C65617374DB
:1017E00020646576696365206E616D6520616E6455
:1017F0002062726F6B6572204950206D7573742082
:10180000626520636F6E6669677572656400526514
:1018100062696E6420737563636573732E2049502B
:1018200020616464726573733A004572726F723A34
:1018300020726562696E64206661696C0052656E33
:101840006577656420737563636573732E204950F3
:1018500020616464726573733A004572726F723A04
:101860002072656E65776564206661696C000A4E5A
:101870006F206C696E6B00526573746F72696E676E
:1018800020636F6E6669672066726F6D20454550F4
:10189000524F4D00416363657074696E6720636FDA
:1018A0006D6D616E64732E2E2E0A004E6F204D51A9
:1018B000545420636F6E66696775726564004C6F7F
:1018C0006164696E6720636F6E6669672066726F18
:1018D0006D20706F7274616C2064697361626C65F5
:1018E000642E2075736520676574204F4E20746FD9
:1018F00020656E61626C6500436F6E666967206982
:10190000732076616C696400436F6E74696E7565EF
:1019100020776974682070726576696F75736C7969
:10192000206C6F6164656420636F6E666967000098
:10193000002200250028002B002E00310034000278
:10194000010000050108010B0100000A0B02090C4F
:101950000D0E080703040100000000000000000055
:101960000000000000000000000000000000000077
:101970000000000000121110000000000000000034
:101980000000000000000000000000000000000057
:10199000002100240027002A002D00300033000120
:1019A000010000040107010A0101021020200808BB
:1019B00010204010204080020102010804020101B1
:1019C000020408102040808040201008040201809A
:1019D00004020180402010080402010804020101F1
:1019E00002040810204080010204081020408005F5
:1019F000050505070508080808020202020A0A0888
:101A000008040404040101010101010101030303AD
:101A10000303030303040707070C0C0C0C0C0C0C4A
:101A20000C0202020206060606060606060B0B0B51
:101A30000B0B0B0B0B2F64617461002F736B6574C0
:101A40006368004163636573732D436F6E74726FD7
:101A50006C2D416C6C6F772D486561646572733ACB
:101A600020436F6E74656E742D747970652C436FAE
:101A70006E6E656374696F6E2C417574686F726900
:101A80007A6174696F6E2C507261676D6100416399
:101A9000636573732D436F6E74726F6C2D416C6C44
:101AA0006F772D4D6574686F64733A20504F5354AF
:101AB0002C4745542C4F5054494F4E5300416363BB
:101AC0006573732D436F6E74726F6C2D416C6C6F08
:101AD000772D43726564656E7469616C733A207426
:101AE000727565004F5054494F4E530044454C4564
:101AF0005445005055540047455400504F5354002E
:101B0000617574686F72697A6174696F6E3A2000EA
:101B1000417574686F72697A6174696F6E3A2000FA
:101B2000436F6E74656E742D4C656E6774683A20F1
:101B3000006F637465742F73747265616D00696DF5
:101B40006167652F6A70656700696D6167652F67FA
:101B5000696600746578742F68746D6C00617070CC
:101B60006C69636174696F6E2F6A736F6E00746560
:101B700078742F706C61696E00436F6E74656E745B
:101B80002D547970653A2000436F6E6E65637469F9
:101B90006F6E3A20636C6F736500416363657373A6
:101BA0002D436F6E74726F6C2D416C6C6F772D4F7F
:101BB000726967696E3A20687474703A2F2F6C618D
:101BC0007A79686F6D652E727500556E6B6E6F77E2
:101BD0006E004F4B004D6F766564207065726D61CD
:101BE0006E656E746C7900496E7465726E616C20FE
:101BF000536572766572204572726F72005061791A
:101C00006C6F616420546F6F204C61726765004E89
:101C10006F7420666F756E64005757572D41757449
:101C200068656E7469636174653A204261736963C3
:101C3000207265616C6D3D22416363657373207230
:101C40006573747269637465642200556E6175749E
:101C5000686F72697A6564005061796C6F616420A5
:101C600073697A652077726F6E67004261642072D3
:101C700065717565737400485454502F312E3120AE
:101C8000002000202D3E2041543A004368616E2020
:101C9000747970653A004E6F2073746F72656420BA
:101CA00076616C756573202D2064656661756C7452
:101CB0003A20002D3E005075623A2000636D6400AA
:101CC000434F4F4C0048454154004155544F002D5F
:101CD0003E005075623A20007365740064656C00C4
:101CE0002D3E005075623A20002D3E005075623A3C
:101CF0002000556E6B6E6F776E20636D64200A0056
:101D00004F4646004F4E005361766564204554416E
:101D1000473A0053657420455441473A200080AB50
:101D20004F9A11241FBECFEFD1E2DEBFCDBF00E03E
:101D30000CBF15E0A0E0B2E0E4E7FFE701E00BBF75
:101D400002C007900D92A437B107D9F72AE0A4E7A3
:101D5000B5E001C01D92A334B207E1F71EE0C0E96F
:101D6000DEE000E006C021970109802FFE010E94FD
:101D700070BACF38D10780E00807A9F70E94619AAE
:101D80000C94A8BF0C940000FC01818D928D0895E5
:101D9000FC018489958908952AE733E0FC013183A9
:101DA0002083FB014089518962897389FC01428348
:101DB0005383648375830895DC01ED91FC91048C59
:101DC000F58DE02D1994CF93DF931F92CDB7DEB739
:101DD0006983DC01ED91FC910280F381E02D41E00B
:101DE00050E0BE016F5F7F4F19950F90DF91CF914B
:101DF0000895FC019485FB018485981303C081E05C
:101E0000943009F480E0089521E0FC018485843059
:101E100009F420E0822F08950895CF93DF931F9255
:101E2000CDB7DEB76983DC01ED91FC910280F381CF
:101E3000E02D41E050E0BE016F5F7F4F19950F909C
:101E4000DF91CF910895DC01ED91FC91068CF78D27
:101E5000E02D199591E089270895862F089581E056
:101E600086270895DC0180E0615038F0ED91E82785
:101E7000F0E0E553FC4E8491F7CF0895FC01818199
:101E800091E09093B6078093D8071092B70710920D
:101E9000D907089520911B06260F3327331F2132BF
:101EA0003105ECF42091B007FC0190E080E0243093
:101EB00069F082E00895A0911B062191AC01475082
:101EC0005A4FA40FB52FB11D2C930196861798F386
:101ED00080911B06680F60931B0680E0089581E0E7
:101EE000089508950895E091410680914006E8170D
:101EF00030F4F0E0EE5BF94F808190E008958FEFD1
:101F00009FEF089590914106809140062FEF3FEF9B
:101F1000981748F4E92FF0E0EE5BF94F208130E0AC
:101F20009F5F90934106C90108958091400690916A
:101F30004106891B990B0895CF92DF92EF92FF9291
:101F40000F931F93CF93DF937C01CB018A012091E4
:101F5000B607222389F0EB016B01C40ED51ECC1508
:101F6000DD0569F06991D701ED91FC910190F08157
:101F7000E02DC7011995F3CF642F0E944A0FC801C5
:101F8000DF91CF911F910F91FF90EF90DF90CF9055
:101F90000895CF93DF931F92CDB7DEB76983209169
:101FA000B6072223F9F02091D907203258F021E01A
:101FB00030E0FC013383228390E080E00F90DF91DA
:101FC000CF9108958091B707E82FF0E0E854F84FDB
:101FD000998190838F5F8093B7078093D90781E0C1
:101FE00090E0ECCF61E0CE0101960E944A0FF7CF5E
:101FF0008F929F92AF92BF92CF92DF92EF92FF9219
:102000000F931F93CF93DF9300D000D000D01F9287
:102010001F92CDB7DEB77C018E010F5F1F4F6801A5
:102020008AE0882E912CA12CB12CC601801B910B2B
:10203000411551056105710581F0CB01BA01A5017A
:1020400094010E94E5B9942F852F605DF60161939C
:102050006F01A901692F782FE8CFF801E80FF91F68
:10206000D7010150110922912D93E017F107D9F7FB
:10207000E80EF91EF70110822B960FB6F894DEBF1A
:102080000FBECDBFDF91CF911F910F91FF90EF90C9
:10209000DF90CF90BF90AF909F908F900895FC01FC
:1020A000DC018D918111FDCF30E020E050E040E077
:1020B0008AE09191992301F1443051055CF59E32FB
:1020C00071F42F3F310509F02CF5DB01A40FB51F8A
:1020D00012962C934F5F5F4F30E020E0EACF829F53
:1020E000D001839FB00D1124292F990F330B20535A
:1020F00031092A0F3B1FDDCF2F3F310509F054F482
:10210000443051053CF4640F751FFB01228381E0CC
:1021100090E0089590E080E00895CF93DF931F92C0
:102120001F92CDB7DEB78091370A9091380A009799
:1021300011F483E49AE0BE016F5F7F4F681B790B57
:10214000072E000C880B990B0F900F90DF91CF9109
:1021500008959FE9980F963010F4875508959FEBE6
:10216000980F963010F48753089580538A3008F002
:1021700080E00895DC0115968D919C91009739F0CF
:10218000DC01ED91FC910680F781E02D1994089512
:10219000FC01848195810895CF93DF9300D000D016
:1021A0001F921F92CDB7DEB7FC01862F8F70618121
:1021B000607F682B618388E0DE01119601900D92AB
:1021C0008A95E1F729813A814B815C816D817E811D
:1021D0008F81988528960FB6F894DEBF0FBECDBFCD
:1021E000DF91CF910895DC011196EC911197E29562
:1021F000EF70E150EB3008F039C0F0E08827EC5F79
:10220000FE4E8F4F0C9470BA2711271136110F1103
:102210000F1118112F112F112F110F110F111496CB
:102220006D917D918D919C9117970E94A2B8089510
:1022300014966D917D918D919C9117972AE030E0D5
:1022400040E050E00E9407BACA01B901EECF1496EF
:102250006C9170E090E080E00E94A0B80895149620
:102260006D917D918D919C911797089560E070E03C
:10227000CB010895DC011196EC911197E295EF7076
:10228000E150EB3008F037C0F0E08827E55BFE4E08
:102290008F4F0C9470BA5D115D117B115611561160
:1022A0006C116311631163115611561114966D91DF
:1022B0007D918D919C911797089514966C9170E083
:1022C00090E080E0089514966D917D918D919C91A0
:1022D00017970E946DBB089514966D917D918D9115
:1022E0009C9117972AE030E040E050E00E9407BA46
:1022F000CA01B901089560E070E0CB010895FC01C6
:10230000A7812A2F2E7FD1F0818182958F708150F5
:102310008330A0F4A695A150BB0B2BE531E00E94C1
:1023200087BA24E630E040E050E00E9407BADA01C4
:10233000C90187569F4FAF4FBF4F08958FEF9FEF53
:102340000895CF93DF93EC016115710539F48F8106
:1023500081708F8381E0DF91CF9108958981982FDB
:1023600092959F7029F180E09430A8F79B01770F38
:10237000440B550B2959310941095109A4E6B0E034
:102380000E9426BA2BE531E040E050E00E9407BAF7
:1023900037FF02C030E020E02536310514F024E696
:1023A00030E02F5F220F8F818170282B2F83D2CFB7
:1023B0008F7080628983DACFFC019181892F8295A9
:1023C0008F7021F0823029F080E008959F70906234
:1023D00091839B0177FF02C030E020E02E3681E040
:1023E000380714F02DE631E02683878130FB80F931
:1023F000878381E00895DC01ED91FC91309729F00D
:1024000090859F7081E0953009F080E00895DC01AF
:102410001496ED91FC911597309799F090859F70E7
:102420008EEF890F823010F091110BC041875287D7
:10243000638774871496ED91FC918085807F82601C
:1024400080870895DC0119968D919C91009739F051
:10245000DC01ED91FC910280F381E02D1994089547
:10246000DC01ED91FC91008CF18DE02D1994CF935E
:10247000DF93EC01E881F9810484F585E02D19955D
:1024800029893A892F5F3F4F3A8B298BDF91CF9172
:102490000895CF93DF93EC018E8581110DC081E00B
:1024A00090E049895A892C853D854217530708F0E9
:1024B00080E0DF91CF910895E881F9810484F5856A
:1024C000E02DCE0119958F3F910549F780E090E00E
:1024D000F0CFFC01848595856817790708F4CB0156
:1024E000928B818B0895DC011E962C911E972223DE
:1024F00039F0ED91FC910190F081E02D6FEF19948E
:102500000895FC0187859089089581E0089590E001
:1025100080E00895CF92DF92EF92FF920F931F9386
:10252000CF93DF93CDB7DEB7AF970FB6F894DEBF8A
:102530000FBECDBF7C016A010AE713E01A8309834D
:102540001C861B8688EE93E0A0E0B0E08D879E8716
:10255000AF87B88B82E593E09A878987188F0F8BB6
:10256000198E1A8E1B8E1C8E84E089A31BA70AA7C6
:102570001CA61DA61EA61FA68091090890910A08F8
:10258000A0910B08B0910C088EA39FA3A8A7B9A790
:102590008B839C83AD83BE8318861F82AE01465D0C
:1025A0005F4FCE0101960E94137681309105B1F400
:1025B000D701ED91FC910488F589E02D1DA30CA3B2
:1025C0008CA59DA5AEA5BFA58EA39FA3A8A7B9A7BF
:1025D000A601BE016C5D7F4FC7011995AF960FB67E
:1025E000F894DEBF0FBECDBFDF91CF911F910F9149
:1025F000FF90EF90DF90CF900895CF92DF92EF920F
:10260000FF920F931F93CF93DF93CDB7DEB7AF97B2
:102610000FB6F894DEBF0FBECDBF7C016A010AE79A
:1026200013E01A8309831C861B8688EE93E0A0E0E2
:10263000B0E08D879E87AF87B88B82E593E09A875D
:102640008987188F0F8B198E1A8E1B8E1C8E84E033
:1026500089A31BA70AA71CA61DA61EA61FA68091BC
:10266000090890910A08A0910B08B0910C088EA35C
:102670009FA3A8A7B9A78B839C83AD83BE8318862D
:102680001F82AE01465D5F4FCE0101960E94137618
:1026900081309105B1F4D701ED91FC910684F78565
:1026A000E02D1DA30CA38CA59DA5AEA5BFA58EA353
:1026B0009FA3A8A7B9A7A601BE016C5D7F4FC70164
:1026C0001995AF960FB6F894DEBF0FBECDBFDF9160
:1026D000CF911F910F91FF90EF90DF90CF900895D1
:1026E000CF93DF93EC01888D843061F00E94D97B19
:1026F000E88DF0E0EE0FFF1FE559F94F11821082CF
:1027000084E0888FDF91CF910895EF92FF921F931D
:10271000CF93DF93FC01208D243039F080E0DF91EE
:10272000CF911F91FF90EF9008957B01EC0110E095
:10273000812F0E949C7C81110FC0188F888D84305E
:1027400069F3FD86EC861A8E198E20E0A70162E0FF
:102750000E94ED7B81E0E3CF883179F31F5F143075
:1027600039F7ECCF0F931F93CF93DF931F92CDB721
:10277000DEB78C01DC01ED91FC910084F185E02D48
:102780001995892B79F0BE016F5F7F4FF801848521
:102790000E949E74898190E00F90DF91CF911F91EC
:1027A0000F9108958FEF9FEFF7CFFC0184850C9474
:1027B0000175CF93DF931F92CDB7DEB741E050E0B4
:1027C000BE016F5F7F4FFC0184850E940175181662
:1027D000190634F4898190E00F90DF91CF9108952C
:1027E0008FEF9FEFF9CFFC018485843011F00C94BA
:1027F000DF7490E080E00895CF93C62F0E943E0FD3
:1028000061EE8FE098E00E94C90F6C2F8FE098E096
:102810000E94C90FCF910C94FB8A1092B00781E0FF
:102820008093AF0710928A0761E084E10E945F897C
:1028300061E085E10E945F89E9EBF0E080818E7FB5
:10284000808380818D7F808388E48093B80085E4D5
:102850008093BC0008956BE47FE0811102C06DE4B9
:102860007FE08BE998E00C94826F64EB7CE08BE96D
:1028700098E00E94826FF0E0E0E0199584EF91E02B
:10288000089561E477E0811102C06CE377E08CE4A5
:1028900099E00C94826FEF92FF920F931F93CF9366
:1028A000DF93EC01A881B981109761F18C918823A5
:1028B00049F108811981F8018081882351F08D3216
:1028C00041F080538A3028F00F5F1F4F198308832F
:1028D000F0CFC8010E94DAB07C016CE270E0C80160
:1028E0000E94C6BE009751F419821882C701DF9179
:1028F000CF911F910F91FF90EF90089501969983CA
:102900008883F4CFF12CE12CF1CF4F925F926F923C
:102910007F92AF92BF92DF92EF92FF920F931F933D
:10292000CF93DF9300D000D0CDB7DEB77C01D62E99
:102930008091F505882309F4BEC0D70114969C91B7
:1029400080910402891708F4B6C08091F305909134
:10295000F405BAE06B13F0C08D559A4FFC0110825C
:10296000D70118960D911C910115110509F49FC00E
:10297000F801618572856115710591F44580568075
:10298000678070848091FD079091FE07A091FF07FA
:10299000B0910008481659066A067B0609F487C0FC
:1029A000D8011B964D915C911C974115510509F476
:1029B0007EC0F701248153968C91539790E0322F7B
:1029C000377002C0959587953A95E2F780FF6FC002
:1029D000A22EB12CC501887F9370892B39F45196B2
:1029E0008D919C91887F9370A82AB92AD8018D91E6
:1029F0009C91DC01ED91FC916115710509F486C093
:102A00000688F789E02D1995019709F050C06CE30D
:102A1000F801808191810E948F6EA50170E060E0D5
:102A20002AE0D8018D919C910E943F6EF80122818D
:102A3000808191816AE873E1222311F068E873E1F3
:102A40000E94826FD8011D966D917C911E978D9189
:102A50009C910E941C6F60E2F801808191810E942C
:102A60008F6ED8011F966D917C9150978D919C919E
:102A70000E941C6FF8012281808191816DE773E1D2
:102A8000222311F067E773E10E94826F63EA75E029
:102A9000D8018D919C910E941C6FF80180819181D9
:102AA000DC01ED91FC91008CF18DE02D19951092D7
:102AB000F4051092F305D70115968D919C91169708
:102AC000009709F44DC014963C91209105022317FC
:102AD00008F446C0DC01ED91FC910190F081E02DFD
:102AE0006D2D199526960FB6F894DEBF0FBECDBF9B
:102AF000DF91CF911F910F91FF90EF90DF90BF90EA
:102B0000AF907F906F905F904F9008950488F58903
:102B1000E02D2AE733E03A832983D80115964D90BA
:102B20005D906D907C9018974B825C826D827E8266
:102B3000BE016F5F7F4F67CF8F3491050CF0BBCF25
:102B4000BDE06B1709F4B7CF9C012F5F3F4F309367
:102B5000F4052093F3058D559A4FFC016083ABCFAC
:102B600081E090E0BFCFCF93DF9300D000D01F92E1
:102B70001F92CDB7DEB7E6E8F8E0128A118A80E04E
:102B800090E19587848784E890E0948B838B81E043
:102B9000868780E090E2908B87871C821B828BE582
:102BA00092E09A838983FE83ED838FEF9FEF98876E
:102BB0008F8362EB72E18BE998E00E94826F6091F3
:102BC0008E0570918F05CE0101960E94197186E8DD
:102BD00098E00E94301262EA72E18BE998E00E946C
:102BE000826F8BE998E00E948B6E0E94BA922896C1
:102BF0000FB6F894DEBF0FBECDBFDF91CF91089521
:102C0000FC0186819781009799F0FC0120852F7047
:102C1000223029F461857285838594850895253055
:102C200039F460E00E948884009711F0FC01F2CF33
:102C300060E070E0CB010895CF93DF93EB0163E098
:102C4000FC01808191810E948884009761F0FC01E1
:102C500020852F70223039F4818592858C239D2325
:102C6000DF91CF91089590E080E0FACF63E0FC011E
:102C7000808191810E948884009719F0FC018185F0
:102C800008958FEF0895EF92FF921F93CF93DF93F4
:102C9000192F7B01C82FD92FD7FF03C0D195C1951C
:102CA000D10961E08C2F0E948D8982E0E816F10441
:102CB00099F460E08C2F0E945F896FE272E18CE4EE
:102CC00099E00E94826F8CE499E0DF91CF911F918F
:102CD000FF90EF900C948B6E612FEF2851F460956C
:102CE000661F6627661F8C2F0E945F896BE272E168
:102CF000E6CF661F6627661F8C2F0E945F8966E2FB
:102D000072E1DDCF892B71F0FB01828193810E94FA
:102D1000508164EC7EE08BE998E00E94826F88EC41
:102D200090E0089590E080E0F2CF892B71F0FB01F4
:102D3000828193810E94ED806DEA7EE08BE998E0CC
:102D40000E94826F88EC90E0089590E080E0F2CFDE
:102D50008091780890917908892B51F00E94E49332
:102D6000882331F06DE97EE08BE998E00E94826F64
:102D7000109298081092970880E090E19093930841
:102D80008093920884E890E090939A088093990841
:102D900081E08093940880E090E29093960880937D
:102DA000950886E898E00E94731286E898E00E94F1
:102DB000301288EC90E00895EF92FF920F931F93EA
:102DC000CF93DF93CDB7DEB72C970FB6F894DEBF65
:102DD0000FBECDBF8C017B018AE793E09A83898384
:102DE0001B821C821D821E8298878F8319861A86F9
:102DF0001B861C8605301105ECF0BE01695F7F4F14
:102E0000F701808591850E944F10892B99F0CE01A2
:102E100007960E941E82BE01695F7F4FF70186817F
:102E200097810E944F10892B61F0CE0107960E9476
:102E3000F4820EC0CE0101960E941E82043011055C
:102E400054F7CE0101960E94F482033011058CF1F3
:102E5000BE01695F7F4FF701848195810E944F1009
:102E6000892B39F1CE0107960E948982BE01695FE4
:102E70007F4FF701828193810E944F10892B01F1CE
:102E8000CE0107960E94B38166E87EE08BE998E068
:102E90000E94826F88EC90E02C960FB6F894DEBF0B
:102EA0000FBECDBFDF91CF911F910F91FF90EF909B
:102EB0000895CE0101960E94898202301105B4F670
:102EC000CE0101960E94B38101301105E9F6CE01D1
:102ED00001960E94B3816DE87EE08BE998E00E9444
:102EE000826FD2CFCF93C1E068EE73E080E090E0D4
:102EF0000E94FE8A6C2F8BE998E00E947984CF5F54
:102F0000C43191F784EF91E0CF910895CF93C62F0C
:102F100063E0FC01808191810E948884FC01892BFF
:102F200019F19085892F8D70F9F4907F92609087C8
:102F300081859285A385B4858827AA27BB278C2BFA
:102F400081879287A387B48766EA75E08CE499E06D
:102F50000E94826F6C2F8CE499E00E9479848CE44B
:102F600099E0CF910C948B6ECF9108950F931F939E
:102F7000CF93DF938C01EB010297C4F08A819B8190
:102F80000E94DAB08093050299270E9429840230BA
:102F9000110549F08C819D810E94DAB08093040272
:102FA00099270E943384C8ECD0E002C0C0E9D1E088
:102FB00062E77EE08BE998E00E94826F60910502F3
:102FC0008BE998E00E9479846DE57EE08BE998E0DA
:102FD0000E94826F609104028BE998E00E947984DC
:102FE0008BE998E00E948B6ECE01DF91CF911F910B
:102FF0000F910895CF93DF93EB010297A4F168E45A
:103000007FE08A819B810E9428B1892B29F40E944C
:103010005F836F770E94B98364E47FE08A819B813C
:103020000E9428B1892B29F40E945F8360680E9466
:10303000B9836CE47EE08BE998E00E94826F0E9485
:103040005F836095661F6627661F70E08BE998E0D6
:103050000E9480848BE998E00E948B6E88EC90E05F
:10306000DF91CF9108950E94B315F8CF0F931F936E
:10307000CF93DF93EC01888199810E94EF84082F20
:1030800010E00430110584F40E941D73009721F0B4
:10309000FC012085207F2087BC01888199810E94C6
:1030A0005A840F5F1F4FEDCF0881198160E0C8017E
:1030B0000E948884FC018185888761E0C8010E94A4
:1030C00088849B838A8362E0C8010E9488849D83F0
:1030D0008C8364E0C8010E9488849F838E83DF9183
:1030E000CF911F910F910895CF93DF93EC017983D6
:1030F00068831A8619861B861E8A1D8A0E94FB1108
:10310000882329F0CE01DF91CF910C943618DF91FE
:10311000CF910895CF92DF92EF92FF920F931F937A
:10312000CF93DF93EC016A017B018E819F81892B14
:10313000D9F4888199810E94EF84082F10E005302E
:10314000110594F40E941D73009721F0FC01208565
:10315000207F20879F838E83BC01888199810E9474
:103160005A840F5F1F4FEBCFEE81FF81309749F1FB
:103170008085982F9F7019F5807F82608087EE810F
:10318000FF81C186D286E386F4866EEA75E08CE420
:1031900099E00E94826F2AE030E0B701A6018CE43A
:1031A00099E00E94966E8CE499E0DF91CF911F9197
:1031B0000F91FF90EF90DF90CF900C948B6E923038
:1031C000F1F2DF91CF911F910F91FF90EF90DF907F
:1031D000CF900895CF93DF93009709F484C0FC014A
:1031E0002081222309F47FC0EC0168ED7CE10E947C
:1031F0003BB1892B09F456C06CEB7CE1CE010E94F7
:103200003BB1892B09F451C061EA75E0CE010E94FF
:103210003BB1892B09F44CC06DE975E0CE010E94E9
:103220003BB1892B09F447C069E975E0CE010E94E2
:103230003BB1892B09F442C065E975E0CE010E94DB
:103240003BB1892BF1F161E975E0CE010E943BB100
:10325000892BD1F16DE875E0CE010E943BB1892B3D
:10326000B1F168E875E0CE010E943BB1892B91F184
:1032700064E875E0CE010E943BB1892B71F16CEDE1
:103280007CE1CE010E943BB1892B51F160E875E0F1
:10329000CE010E943BB1892B31F58EE090E0DF91A9
:1032A000CF91089582E090E0FACF81E090E0F7CFEF
:1032B00088E090E0F4CF85E090E0F1CF86E090E008
:1032C000EECF87E090E0EBCF89E090E0E8CF8AE0B6
:1032D00090E0E5CF8BE090E0E2CF8CE090E0DFCFB4
:1032E0008DE090E0DCCF90E080E0D9CF0F931F938A
:1032F000CF93DF938C01FC01C081D1816FE270E03C
:10330000CE010E940EBF0097D9F0FC011192CF01AF
:103310000E94EA18EC016AEB75E08CE499E00E94E7
:10332000826FBE018CE499E00E9480848CE499E075
:103330000E948B6ECE01DF91CF911F910F91089566
:10334000CE010E94EA18EC01892BA1F3F801118249
:103350001082F0CF8F929F92AF92BF92CF92DF9266
:10336000EF92FF920F931F93CF93DF93CDB7DEB70A
:1033700067970FB6F894DEBF0FBECDBF8C017B01FF
:103380004C018BE0880E911C9F8A8E8AF801128670
:1033900011861386168A158A672B09F463C0A090DC
:1033A0007506B0907606A114B10409F45BC06FE213
:1033B00070E0C7010E94C6BE6C01892B09F44AC0A7
:1033C000F701DE01119690E080E0BD0121912223FA
:1033D00041F02F3231F08431910519F02D9301968F
:1033E000F5CF860F971FFC011082C5010E943F8414
:1033F000F80191838083B6016F5F7F4F4AE050E010
:10340000C4010E94FFBECE0146960E947619F801C3
:10341000968B858B8E899F89892B09F41386C80129
:103420000E94FB11882319F0C8010E943618679684
:103430000FB6F894DEBF0FBECDBFDF91CF911F91C5
:103440000F91FF90EF90DF90CF90BF90AF909F9043
:103450008F900895B701C5010E943F84F8019183C0
:103460008083DDCFF80111821082D9CFEF92FF92D5
:103470000F931F93CF93DF93EC018B011D821C826E
:103480001A821B82E880F980E114F10409F472C009
:1034900080918E0590918F05892B09F46BC0672B65
:1034A00009F48701F80180858F708630A9F46CE7F4
:1034B00073E0C8010E943F84009719F0FC018185E8
:1034C0008A8366E675E0C8010E943F84009709F48C
:1034D00058C0FC0181858B836EE773E0C7010E94B1
:1034E0003F84009709F043C068E375E08CE499E0FD
:1034F0000E94826F6B818CE499E00E94798466E37C
:1035000075E08CE499E00E94826F6A818CE499E016
:103510000E9479848CE499E00E948B6EE880F980A7
:103520000E941D738C010097D1F0FC018085807F83
:10353000826080871186128613861486808191812D
:10354000009711F00E94AAAE8EE793E00E9466BE3B
:10355000F80191838083B801C7010E945A846EE705
:1035600073E0888199810E943F84009719F0099641
:103570009D838C83DF91CF911F910F91FF90EF90EE
:103580000895F801808191810E94DAB0A4CF1F9341
:10359000CF93DF93FC01162FC389D4898189928947
:1035A0009C012F5F3F4F328B218BC80FD91FCE015B
:1035B0000E94BFB9181721F0612FCE010E94C7B930
:1035C00081E090E0DF91CF911F910895FC01818906
:1035D0009289248535858217930740F4238934899D
:1035E000820F931F0E94BFB990E008958FEF9FEF65
:1035F00008959B0190E00496982F8827642F820FEE
:10360000931F0C948374CF93DF93C82FD0E024963C
:10361000DC2FCC27C60FD71F0E9408748FE00E94B2
:103620001D748D2F0E941D748C2F0E941D7480E0CC
:103630000E941D74C82F0E9406748C2FDF91CF91B9
:103640000895CF93DF93C82FD62F472F60E170E006
:103650000E94F91A4D2F61E170E08C2FDF91CF911C
:103660000C94F91A90E0982F882744E050E0845F8A
:103670009B4F0C945474FC018485843011F00C949D
:103680009C7C80E00895CF93DF93FC012485243057
:10369000D9F0EC010E943B1B843189F0882379F03A
:1036A000883169F021E08C3159F4E881F981008496
:1036B000F185E02DCE01199521E0892B09F420E058
:1036C000822FDF91CF91089580E0FBCF44E050E05E
:1036D000BC018FE090E00C94547444E050E0BC01D5
:1036E00085E090E00C94547444E050E0BC0181E02B
:1036F00090E00C94547408958F929F92AF92BF9271
:10370000CF92DF92EF92FF920F931F93CF93DF93AD
:10371000CDB7DEB72D970FB6F894DEBF0FBECDBF85
:103720007C0110E000E038EE832E33E0932EA12CD4
:10373000B12C42E0C42E43E0D42E1C821B828D8229
:103740009E82AF82B886DA82C9820D87CE01019649
:103750000E943B1B811135C0F7014481558120E057
:1037600061E0802F0E94ED7B80E590E00E94B387AE
:1037700063E070E0802F0E94031B833129F462E034
:1037800070E0802F0E94B687F70184819581000F39
:10379000111FF801E559F94F918380832D960FB6DB
:1037A000F894DEBF0FBECDBFDF91CF911F910F9177
:1037B000FF90EF90DF90CF90BF90AF909F908F9051
:1037C00008950F5F1F4F0430110509F0B6CFE6CF03
:1037D000CF92DF92EF92FF921F93CF93DF93FC0182
:1037E0001485143089F1EC0180E590E00E94B387E4
:1037F00068E070E0812F0E94B6870E94438D6B01C4
:103800007C01CE010E943B1B8823A1F062E370E0A3
:1038100080E090E00E94FE8A0E94438D6C197D0931
:103820008E099F09683E73408105910550F38C8590
:103830000E94D97BEC85F0E0EE0FFF1FE559F94FB0
:103840001182108284E08C87DF91CF911F91FF90CD
:10385000EF90DF90CF9008954F925F926F927F929A
:103860008F929F92AF92BF92CF92DF92EF92FF9290
:103870001F93CF93DF93CDB7DEB72D970FB6F89494
:10388000DEBF0FBECDBF7C019BE6A92E96E0B92E10
:1038900010E0D12CC12C28EE422E23E0522E612CB8
:1038A000712C32E0832E33E0932E1C821B824D82DA
:1038B0005E826F8278869A8289821D87D5012D91DA
:1038C0003D915D01F7018481958128173907B1F495
:1038D000CE0101960E943B1B843199F1CE010196E5
:1038E0000E943B1B8C3151F4CE0101960E94F313D0
:1038F000892B21F4CE0101960E94E81B1F5F143032
:10390000A1F6CD2841F4D701ED91FC910084F18519
:10391000E02DC70119952D960FB6F894DEBF0FBEA6
:10392000CDBFDF91CF911F91FF90EF90DF90CF90AF
:10393000BF90AF909F908F907F906F905F904F90CF
:103940000895CC24C394D12CD9CF8F929F92AF925B
:10395000BF92CF92DF92EF92FF920F931F93CF937C
:103960006C015B017A01FC01C485C430A1F481E0E3
:1039700090E0F60193838283F12CE12CC701CF9173
:103980001F910F91FF90EF90DF90CF90BF90AF907D
:103990009F908F9008958A014130584010F000E0C8
:1039A00018E080E590E00E94B3878C2F0E94CA88BF
:1039B0004C0163E070E08C2F0E94031B873111F0F3
:1039C0008C3129F58016910660F380E590E00E9425
:1039D000B3879801A50170E060E08C2F0E946A888F
:1039E00060E270E08C2F0E94B68762E070E08C2F5E
:1039F0000E94031B84FD13C063E070E08C2F0E94C3
:103A0000031B811107C08C2F0E94D97BB0CF10E01F
:103A100000E0DBCF80E590E00E94B387E6CF40E195
:103A200062E070E08C2F0E94F91A012B09F0A6CFFA
:103A30009ECF3F924F925F926F927F928F929F9212
:103A4000AF92BF92CF92DF92EF92FF920F931F93AC
:103A5000CF93DF93CDB7DEB72D970FB6F894DEBFC7
:103A60000FBECDBF6C015B014A010E942C1C8BE68E
:103A7000E82E86E0F82E312C10E000E098EE492E7A
:103A800093E0592E612C712C1C821B824D825E8228
:103A90006F82788682E093E09A8389833D86F7017E
:103AA000219131917F01F601848195812817390791
:103AB00071F4CE0101960E943B1B873141F4A401B1
:103AC000B501CE0101960E94A51C080F191F339461
:103AD000F4E03F12D9CFC8012D960FB6F894DEBF9F
:103AE0000FBECDBFDF91CF911F910F91FF90EF904F
:103AF000DF90CF90BF90AF909F908F907F906F900E
:103B00005F904F903F900895CF93DF9391E0909313
:103B1000F8058823B9F0C091B800D091BA0080911F
:103B2000BC008A7B8093BC0060E084E10E945F89D6
:103B300060E085E10E945F890E940D14D093BA0075
:103B4000C093B800DF91CF910895CF92DF92EF92AA
:103B5000FF920F931F93CF93FC01C1810E94E689CE
:103B60006B017C018091B007811164C081E080937A
:103B7000B0078093AF079FEF9093AE071092AD0709
:103B80001092AC0780938B0780918B07CC0FC82BCA
:103B9000C0938B0780918A07813009F081C0109211
:103BA0008A070E94E6896B017C0180918B078093D4
:103BB000BB008091B2079091B307A091B407B09178
:103BC000B507892B8A2B8B2BA1F00E94E6890091E7
:103BD000B2071091B3072091B4073091B5076C1963
:103BE0007D098E099F09061717072807390708F46A
:103BF00042C08091BC0083FDD8CF85EC8093BC008F
:103C00000E94E6896B017C018091B007813009F444
:103C100049C08091AD07811167C08091AD07ECE884
:103C2000F7E0A2E4B6E090E0981751F121912D93CE
:103C30009F5FFACF8091B2079091B307A091B4072C
:103C4000B091B507892B8A2B8B2B09F48BCF0E945F
:103C5000E6890091B2071091B3072091B407309123
:103C6000B5076C197D098E099F09061717072807E4
:103C7000390708F077CF8091B1070E94841D80E05A
:103C800010924106809340068FE098E00E94820FD8
:103C9000CF911F910F91FF90EF90DF90CF900895FB
:103CA00085EEACCF8091B2079091B307A091B40795
:103CB000B091B507892B8A2B8B2B09F4A5CF0E94D5
:103CC000E6890091B2071091B3072091B4073091B3
:103CD000B5076C197D098E099F0906171707280774
:103CE000390708F091CFC7CF81E099CFAF92BF924B
:103CF000CF92DF92EF92FF921F93CF93DF93EC016D
:103D00000E94438D6B017C0128EEC20E23E0D21E7F
:103D1000E11CF11C10E08BE4A82EB12C0E94438D15
:103D20006C157D058E059F0598F460EFCE010E940D
:103D3000FC13CE010E94A51D182F80FF0BC0ED853E
:103D4000FE85309709F01995C5010197F1F7E6CF87
:103D500081E08A83812FDF91CF911F91FF90EF90B7
:103D6000DF90CF90BF90AF9008951F93CF93DF93D4
:103D7000EC01162F0E94761ECE010E943E0F62EDCE
:103D80008FE098E00E94C90F612F70E060957095F8
:103D900084E0660F771F8A95E1F7612B8FE098E04A
:103DA0000E94C90F0E94FB8ACE010E94A51D8117A7
:103DB00011F084E08A83DF91CF911F910895CF9312
:103DC000DF93EC0163EC0E94FC13CE01DF91CF91F5
:103DD0000C94A51D0F931F93CF93DF93EC010E94CA
:103DE000761E80FD36C0CE010E94DF1E60E0CE014F
:103DF0000E94B51ECE010E94761ECE010E943E0F8B
:103E000064EB8FE098E00E94C90F0E94FB8ACE010C
:103E10000E94761E082F10E082FF16C082E08A837F
:103E20008881882341F0CE010E94DF1E682F6160E7
:103E3000CE010E94B51E15950795802F8170DF91E8
:103E4000CF911F910F9108958A81823049F71A828C
:103E5000E7CF80E0F4CFCF93DF93EC010E94DF1E29
:103E6000682F6460CE01DF91CF910C94B51E0F9343
:103E70001F93CF93DF93EC01162F042F0E94761E21
:103E8000002319F0CE010E942B1FCE010E943E0F8D
:103E900065EA8FE098E00E94C90F612F8FE098E0FB
:103EA0000E94C90FDF91CF911F910F910C94FB8A53
:103EB0006F927F928F929F92AF92BF92CF92DF923A
:103EC000EF92FF920F931F93CF93DF93FC01248512
:103ED00021118CC0872E762EEC010E94EA1E8823C9
:103EE00009F486C0CE010E94761E40E060EFCE014C
:103EF0000E94371F10E000E066246A94AA24A3946D
:103F0000B12CE02EE694E694E694F12C802F877095
:103F1000650101C0CC0C8A95EAF78B85082E000C50
:103F2000990B0817190734F5FE01EE0DFF1D93805C
:103F30009C20CE010E94761ECE010E943E0F68E7B3
:103F40008FE098E00E94C90F992011F080E8982E28
:103F5000692D8FE098E00E94C90F0E94FB8ACE0174
:103F60000E94761E982F907485FF0BC0992369F0EC
:103F70008EEF2AC09924939408171907D1F2912C37
:103F8000D8CF911102C087FF602EFE01EE0DFF1DFC
:103F9000938187FF28C0C92AC3820F5F1F4F003457
:103FA000110509F0AECF6B86FFEF6F1202C081E002
:103FB0008C872396E72DF82DCF0108962991219320
:103FC000E817F907D9F781E0DF91CF911F910F91A1
:103FD000FF90EF90DF90CF90BF90AF909F908F9029
:103FE0007F906F900895C094C922D6CF80E0ECCF27
:103FF0008FEFEACFEF92FF920F931F93CF93DF9350
:104000008C017B0140E065E50E94371FE70188E0F5
:10401000E80EF11C699140E0C8010E94371FCE15DF
:10402000DF05C1F7DF91CF911F910F91FF90EF90C6
:104030000895CF92DF92EF92FF920F931F93CF9349
:10404000DF938C01EB017A01FC01858196810E944E
:10405000EA1E8823C1F1BE01F801858196810E9484
:10406000FA1F40E06EEBF801858196810E94371FB0
:10407000E7016701F9E0CF0ED11CF801E580F68079
:10408000C7010E94761EC7010E943E0F66E98FE0BD
:1040900098E00E94C90F0E94FB8AC7010E94761E09
:1040A00061EEC7010E94FC13C7010E94A51D899300
:1040B000CC16DD0611F7F801858196810E94EA1E73
:1040C00091E0813009F090E0892FDF91CF911F912D
:1040D0000F91FF90EF90DF90CF900895CF93DF93F3
:1040E000EA010E941920982F882341F068E0CE0150
:1040F0000E94320F91E02885281390E0892FDF91EC
:10410000CF910895CF93DF9300D000D000D0CDB7EA
:10411000DEB7AE014F5F5F4F0E946E20882331F003
:104120008D818F33A9F020F48F31A1F080E007C09A
:104130008F3521F08F37D1F78CE001C08BE02996C5
:104140000FB6F894DEBF0FBECDBFDF91CF910895BB
:104150008AE0F5CF89E0F3CF85ED8093BC008091B4
:10416000B2079091B307A091B407B091B507079635
:10417000A11DB11D23E0B695A795979587952A9522
:10418000D1F72091BC0024FD03C01092B007089520
:104190004091B2075091B3076091B4077091B50791
:1041A000452B462B472B69F30097A105B10541F03C
:1041B00025E32A95F1F700000197A109B109E1CFA4
:1041C0008091B1070C94841D1F920F920FB60F922D
:1041D00011240BB60F922F933F934F935F936F93DE
:1041E0007F938F939F93AF93BF93EF93FF938091B0
:1041F000B900887F803609F44DC008F040C088328D
:1042000009F4A9C028F5803109F49DC0C8F48823B9
:1042100009F4FBC0883009F496C0FF91EF91BF917B
:10422000AF919F918F917F916F915F914F913F914E
:104230002F910F900BBE0F900FBE0F901F901895EF
:10424000883109F488C0803241F78093AE0714C0EA
:10425000803409F49DC040F48033B9F38833E9F623
:104260008093AE0785ECB0C0803509F485C08835F1
:1042700009F496C0883489F60E94AC20CECF8839E4
:1042800009F48CC038F5883729F050F4883611F0DD
:10429000803719F683E08093B00710923F0657C02D
:1042A000883809F47BC0803919F0803809F0B5CF1F
:1042B00080913F06803208F071C0E0913F0681E0B6
:1042C0008E0F80933F068091BB00F0E0E15EF94FD6
:1042D00080833DC0803B39F0E0F4803A09F479C036
:1042E000883A09F09ACF84E08093B00710921C06B8
:1042F00010921B06E0911906F0911A06199580910B
:104300001B0681110FC081E080931B061092F905F6
:1043100009C0803C09F4A6CF883C09F4A3CF883BB0
:1043200009F07BCFE0911C0681E08E0F80931C0684
:10433000F0E0E750FA4F80818093BB0090911C061B
:1043400080911B0629C080918B078093BB0085EC70
:104350008093BC0062CF9091AD078091AC07981715
:1043600058F5E091AD0781E08E0F8093AD07F0E046
:10437000E457F84F8081E9CFE091AD0781E08E0FDF
:104380008093AD078091BB00F0E0E457F84F808345
:104390009091AD078091AC079817C8F285E8D8CF07
:1043A000E091AD0781E08E0F8093AD078091BB0057
:1043B000F0E0E457F84F80838091AF0781115CCF24
:1043C00081E080938A0784EA8093BC001092B00752
:1043D00024CF85EC8093BC001092B00780913F06FB
:1043E000803230F4E0913F06F0E0E15EF94F108258
:1043F00060913F0670E0E0911D06F0911E068FE18E
:1044000096E0199510923F0608CF1092AE0734CF70
:104410004F925F926F927F92AF92BF92CF92DF9254
:10442000EF92FF920F931F93CF93DF9300D01F92D1
:10443000CDB7DEB72B013C0129833A834B835C83E4
:10444000A60195016E0D7F1D801F911F0E94E5B989
:1044500029813A814B815C81621773078407950734
:1044600008F52415350546055705A8F421E0822FE7
:104470000F900F900F900F90DF91CF911F910F91A0
:10448000FF90EF90DF90CF90BF90AF907F906F90B4
:104490005F904F90089521E046165706680679060A
:1044A00030F30FC0461657066806790650F421E02F
:1044B00089819A81AB81BC8184159505A605B705D4
:1044C000B0F220E0D4CF8F929F92AF92BF92CF9262
:1044D000DF92EF92FF920F931F93CF93DF937C01B4
:1044E0004A015901C091F605D091F705062F660FD4
:1044F000110B209709F45CC088858F70863009F015
:1045000055C061E873E0CE010E943F846C0182E0F7
:104510008816910449F066E873E0E3E08E16910492
:1045200029F0D0E0C0E006C06AE873E0CE010E9446
:104530003F84EC01C114D104D9F1F60180858F705C
:104540008430B1F561857285A801C7010E94FFBE64
:10455000A8016FE873E0C7010E94E1BE209779F1DE
:1045600088858F70843059F569857A85A801C701DF
:104570000E94E1BEA8016FE873E0C7010E94E1BE9E
:10458000A114B10429F0A801B501C7010E94E1BE40
:10459000C701DF91CF911F910F91FF90EF90DF90B6
:1045A000CF90BF90AF909F908F900895D0E0C0E0E3
:1045B000A8016DE973E1C7010E9472B1C9CFF2E0B1
:1045C0008F16910481F083E08816910429F06091A0
:1045D000640670916506CACFA80167E973E1C70157
:1045E0000E9454B1C7CFA80164E973E1F8CFCF921C
:1045F000DF92EF92FF920F931F93CF93DF93CDB78C
:10460000DEB7C154D1090FB6F894DEBF0FBECDBFDF
:104610006C01AB0130E020E060E4CE0101967C014A
:104620000E946322F70101900020E9F731978F0182
:104630000E191F09A801B701C6010E94F1BE892BFE
:1046400011F010E000E0C801CF5BDF4F0FB6F89427
:10465000DEBF0FBECDBFDF91CF911F910F91FF90B5
:10466000EF90DF90CF9008954F925F926F927F927C
:104670008F929F92AF92BF92CF92DF92EF92FF9272
:104680000F931F93CF93DF93CDB7DEB761970FB62C
:10469000F894DEBF0FBECDBF0E94438D9B01AC01DD
:1046A00060919F057091A0058091A1059091A20550
:1046B000AA24AA94BA2C650118E8E12E13E1F12E80
:1046C00000E010E00E940822882319F1E0906206C1
:1046D000F0906306D70112968C91823089F568E6D6
:1046E00073E18CE499E00E94826F8CE499E00E946F
:1046F0008B6E80916206909163060E94EA1E0E9472
:10470000438D60939F057093A0058093A1059093BE
:10471000A20561960FB6F894DEBF0FBECDBFDF9144
:10472000CF911F910F91FF90EF90DF90CF90BF90AE
:10473000AF909F908F907F906F905F904F90089573
:1047400080919D0590919E05892B09F0DDC083E144
:1047500090E00E940EAE8C018BED94E6F801928BF6
:10476000818BF682E5821482108289E0818381E068
:104770008283838310939E0500939D050E94438D41
:104780006B017C01F0E1CF0EF7E2DF1EE11CF11CB2
:10479000D8011596ED91FC9116978FEF83871486BB
:1047A0001382148215821682178210861186128651
:1047B00014961C9299249394BE01665F7F4FF80172
:1047C000858196810E94581F18160CF071C00E94B6
:1047D000438D6C157D058E059F0508F069C067E067
:1047E000CE010A960E94320F99898913E5CFD8012C
:1047F0008C91811138C015968D919C910E94EA1E72
:10480000BE01665F7F4FF801858196810E94FA1F85
:1048100040E064EBD80115968D919C910E94371F62
:10482000F801A580B680C5010E94761EC5010E94D0
:104830003E0F67E88FE098E00E94C90F60E88FE0C4
:1048400098E00E94C90F0E94FB8AC5010E94761E53
:10485000B82ED80115968D919C910E94EA1EB5FC48
:1048600002C0F8019082AE014F5F5F4FBE01665FEC
:104870007F4FC8010E941920D8011196BC908A85EB
:10488000803109F48DC2BE01665F7F4FC8010E946E
:1048900082208B1558F5F8018181D80111968C93EF
:1048A000119714968C9114978F5F14968C9384CFE4
:1048B00010E000E080919D0590919E0520919B0560
:1048C00030919C0502171307ECF4980143E0220F86
:1048D000331F4A95E1F76091990570919A05620F2F
:1048E000731F0E94318B0F5F1F4FE4CF8A85803189
:1048F00011F48CE0D2CFBE01665F7F4FC8010E94E9
:104900008220CBCFFC01128280919705909198056F
:1049100020919B0530919C05821793070CF4D6C01B
:104920000E94438D2B013C01E0916206F0916306E9
:10493000309759F08FEF8387148613821482158283
:104940001682178210861186128640919B0550911F
:104950009C05E0919305F091940590E080E0841728
:1049600095070CF48FC088248394912C8091620663
:1049700090916306009709F48EC020919B053091B9
:104980009C05A3E0220F331FAA95E1F760919905DA
:1049900070919A05620F731F0E94581F18160CF031
:1049A0007AC080919B0590919C0541970CF073C053
:1049B0000E94438D9B01AC01AA24AA94BA2C6501E4
:1049C00018E8E12E13E1F12E00E010E0C301B2017E
:1049D0000E94082281115FC0C0909905D0909A056D
:1049E000A0909B05B0909C05850173E0000F111FFE
:1049F0007A95E1F70C0D1D1D67E0C8010E94320F8A
:104A0000D80117969C91F12CE12C8913AFCFEA14B1
:104A1000FB040CF057C148E050E0B801C6010E9409
:104A200080BEB8E0CB0ED11C892B09F04BC0EE0C38
:104A3000FF1CE0919305F0919405EE0DFF1D808120
:104A4000918181609183808362E573E18CE499E0D8
:104A50000E94826F80919B0590919C0563E0880F76
:104A6000991F6A95E1F72091990530919A05820F77
:104A7000931F0E942D866BE473E18CE499E00E9401
:104A8000A66F74CF21913191DF0112972E7F2D9364
:104A90003C93019664CF69E573E18CE499E00E9450
:104AA000826F60919B0570919C058CE499E00E9457
:104AB00080848CE499E00E948B6E1092980510928D
:104AC00097051DCEEFEFEE1AFE0AA1CF00919905D2
:104AD00010919A059C0143E0220F331F4A95E1F79C
:104AE000020F131FD8012C91283209F0DBC0AE0150
:104AF0004F5F5F4FB80180919D0590919E050E9488
:104B00006E20811105C020E030E04EEF52EC3EC037
:104B10006A8170E0762F6627770F770F770F2981EC
:104B2000B8E02B9F90011124262B372BF8018081B0
:104B30008031D1F4688570E08F81AB01481B510949
:104B4000CA019695982F8827979587950E945CBAF9
:104B5000CB014097B90113E0660F771F1A95E1F773
:104B600060789C01260F371F213854EE35075CF220
:104B7000B901330F880B990B0E94A2B820E030E0F6
:104B800040E05CE30E9401B99B01AC01E091950516
:104B9000F09196058091970590919805BC01A3E04E
:104BA000660F771FAA95E1F7A0919905B0919A0534
:104BB0006A0F7B1F309709F0199500919D051091A0
:104BC0009E05E0909705F090980573E0EE0CFF1CB1
:104BD0007A95E1F78091990590919A05E80EF91E72
:104BE000D7018C91803109F463C0B701C8010E94DC
:104BF0008220D82E882309F451C0F801858196813E
:104C00000E94EA1E882309F449C0B701D80115960D
:104C10008D919C910E94FA1FF801408164E4858186
:104C200096810E94371FD80112968C918823B1F18A
:104C3000E7EFED0D4EEE842E42E0942EE33038F493
:104C4000F0E0EE0FFF1FE359FD4F80809180E114EB
:104C5000F10489F1F8018381882369F18081811150
:104C60002AC00E94438D2B013C01092C000CAA088C
:104C7000BB08AE014F5F5F4FB701C8010E9419200A
:104C8000898181110BC00E94438D681979098A09B5
:104C90009B09641575058605970558F3809197055E
:104CA000909198050196909398058093970527CD4C
:104CB0006CE0D62EA2CFB401990C880B990B0E9400
:104CC000FE8AECCF80919D0590919E05892B09F479
:104CD0004DCE88E0815008F449CEF801E80FF11D6F
:104CE00090819923B9F3AA0CBB1C809193059091F4
:104CF0009405A80EB91ED5018D929C9266E473E1CD
:104D00008CE499E00E94826F60919B0570919C05F4
:104D10008CE499E00E9480846FE373E18CE499E075
:104D20000E94826F80919B0590919C0523E0880FE3
:104D3000991F2A95E1F72091990530919A05820FE4
:104D4000931F0E942D868CE499E00E948B6E8091C7
:104D50009B0590919C0533E0880F991F3A95E1F7E8
:104D60006091990570919A05680F791FFB01808108
:104D7000883261F480919D0590919E050E94318B4F
:104D800080916206909163060E942B1F80919B0583
:104D900090919C05019690939C0580939B05E6CD90
:104DA000FCE0FB1508F477CDA4CD64E072E18BE95B
:104DB00098E00E94826F61EF71E18BE998E00E94B8
:104DC000826F63EE71E18BE998E00E94826F6BED78
:104DD00071E18BE998E00E94826F8BE998E00E9474
:104DE0008B6E6EEC71E18BE998E00E94826F6EEB46
:104DF00071E18BE998E00E94826F62EB71E18BE9CF
:104E000098E00E94826F6BE971E18BE998E00E9463
:104E1000826F69E871E18BE998E00E94826F64E734
:104E200071E18BE998E00E94826F65E671E18BE9A0
:104E300098E00E94826F66E571E18BE998E00E943C
:104E4000826F6EE471E18BE998E00E94826F63E407
:104E500071E18BE998E00E94826F69E371E18BE96F
:104E600098E00E94826F61E371E18BE998E00E9413
:104E7000826F65E271E18BE998E00E94826F6BE0DE
:104E800071E18BE998E00E94826F6CEE70E18BE932
:104E900098E00E94826F67ED70E18BE998E00E94D4
:104EA000826F6AEC70E18BE998E00E94826F6CEB94
:104EB00070E18BE998E00E94826F60EB70E18BE912
:104EC00098E00E94826F68EA70E18BE998E00E94A6
:104ED000826F6DE970E18BE998E00E94826F60E972
:104EE00070E18BE998E00E94826F68E870E18BE9DD
:104EF00098E00E94826F6DE770E18BE998E00E9474
:104F0000826F6EE670E18BE998E00E94826F65E641
:104F100070E18BE998E00E94826F8BE998E00C9435
:104F20008B6E009789F0FC0120852F70253061F48D
:104F30000E948884009741F0FC0120852F70243066
:104F400019F481859285089590E080E00895CF92CC
:104F5000DF92EF92FF920F931F93CF93DF9300D0D6
:104F600000D0CDB7DEB78091F50581119CC080914E
:104F700073069091740602970CF495C000918E050B
:104F800010918F050115110509F48DC062E072E0E2
:104F90008AE699E00E94851363E973E0C8010E94E4
:104FA0003F848C01009709F47EC00E94EF84E82EB4
:104FB000F12CE114F10409F476C070E060E0C8015E
:104FC0000E9491276C01EA94EF2809F47BC061E00C
:104FD000C8010E948884FC0101851285CE010196DA
:104FE0000E94C687CE0101960E94E48767E27AE0BC
:104FF0008BE998E00E94826FB6018BE998E00E94ED
:105000001C6F6AE973E08BE998E00E941C6FB8019D
:105010008BE998E00E9480846AE973E08BE998E06C
:105020000E941C6F69E677E08BE998E00E941C6F94
:105030008BE998E00E948B6ED0926009C0925F0964
:10504000109362090093610989E697E0892BE9F5DD
:1050500081E993E0909364098093630980916606E7
:1050600090916706009741F070E060E00E94912700
:10507000909365068093640680916406909165061E
:10508000009721F090936609809365091092680952
:105090001092670981E08093F5056EE07AE08BE974
:1050A00098E00E94826F26960FB6F894DEBF0FBE7E
:1050B000CDBFDF91CF911F910F91FF90EF90DF90C7
:1050C000CF90089502E012E089CF89E697E0C2CF41
:1050D0002F923F924F925F926F927F928F929F9208
:1050E000AF92BF92CF92DF92EF92FF920F93CF9346
:1050F000DF9300D01F92CDB7DEB77C017A8369833E
:105100005C834B83DB011C92FC016081662309F404
:10511000C2C130FFC0C1F9E06F9FB0011124655AD0
:10512000774FCD010E9472B14B815C816CE973E0D5
:1051300089819A810E94E1BEE981FA810190002073
:10514000E9F7319789819A81E81BF90B1C012E0E32
:105150003F1EAB81BC81AE1BBF0B1197BC83AB83E1
:10516000D7011196EC91E295EF70E150EC3008F028
:10517000B3C0F0E08827E054F74D8F4F0C9470BA1D
:10518000CC283B29A129082A242A0829B829B8298A
:10519000B829FC28F028412AF7018481282F30E023
:1051A00050E040E0002359F030E0A4E6B0E00E9477
:1051B00039BA2FEF30E040E050E00E9407BA5F9329
:1051C0004F933F932F938EE993E09F938F93FC81AE
:1051D000FF938B818F933F922F920E9419BF77C0CC
:1051E000F70187818F9386818F9385818F93848147
:1051F0008F9381EA93E0E9CFF70187818F938681CE
:105200008F9385818F9384818F9385EA93E0DDCF9F
:10521000F701C480D580E680F780C701B6012AE097
:1052200030E040E050E00E9407BA97FF07C0909539
:105230008095709561957F4F8F4F9F4F9F938F9370
:105240007F936F93C701B6012AE030E040E050E061
:105250000E9407BA5F934F933F932F9389EA93E09D
:105260009F938F93FC81FF938B818F933F922F921B
:105270000E9419BF2CC0C7010E947F11BC01F70119
:10528000C680D780D0FADD24D0F89481F580EB80F9
:10529000BC80292F30E050E040E077FD35C001119F
:1052A00035C07F936F931F921F921F929F931F92FF
:1052B000FF92DF92CF9280EB93E09F938F939C813C
:1052C0009F93AB81AF933F922F920E9419BF0FB66D
:1052D000F894DEBF0FBECDBF89819A810F900F90E9
:1052E0000F900F90DF91CF910F91FF90EF90DF9093
:1052F000CF90BF90AF909F908F907F906F905F9076
:105300004F903F902F900895002361F0292F30E0B7
:10531000A4E6B0E00E9439BA2FEF30E040E050E060
:105320000E9407BA5F934F933F932F931F92FF9270
:10533000DF92CF9283EB93E09F938F93BF92EF9294
:1053400095CFD70115968C9115971F928F9316962E
:105350009C91169717968C9181708F939F9386EBF3
:1053600093E09F938F93BC81BF93EB81EF9333CFF7
:10537000D70114968D909D90AD90BC90179720E02A
:1053800030E0A901C501B4010E949BB82401350198
:1053900087FF04C077FA709477F87094C301B20164
:1053A0000E946DBB6B01072E000C880B990B0E94AD
:1053B000A2B89B01AC01C301B2010E948EBA20E0E9
:1053C00030E048EC52E40E9401B90E94F8BB0E9410
:1053D0006DBB062F772E20E030E0A901C501B40196
:1053E0000E949BB887FF07C07F920F93DF92CF92F6
:1053F0008CEB93E0B6CF7F920F93DF92CF928DEB41
:1054000093E09F938F939C819F93AB81AF93E3CE67
:10541000D70114968C9114971F928F9315968C91A7
:1054200015971F928F9316968C911F928F9383EBF3
:1054300093E09F938F93BC81BF93EB81EF933F9257
:105440002F920E9419BF43CFD70117968C911797BF
:105450001F928F9314968C9114971F928F93159689
:105460008C9115971F928F9316968C911F928F9304
:1054700080EB93E09F938F93BC81BF93EB81EF937D
:10548000F5CED70114966D917C914B815C81C10161
:105490000E94FFBE21CF29803A8062CEEF92FF9218
:1054A0000F93CF93DF93CDB7DEB7A0970FB6F894E5
:1054B000DEBF0FBECDBF7C0100E020E033E040E264
:1054C00050E0BE016F5F7F4F0E946828BE016F5F92
:1054D0007F4F8CE499E00E941C6F63E479E08CE4D8
:1054E00099E00E94826FF701618162956F708CE490
:1054F00099E00E9479846CE379E08CE499E00E9461
:10550000826FF70161816F708CE499E00E94798469
:105510008CE499E00E948B6EA0960FB6F894DEBFE3
:105520000FBECDBFDF91CF910F91FF90EF90089507
:105530002F923F924F925F926F927F928F929F92A3
:10554000AF92BF92CF92DF92EF92FF920F931F9391
:10555000CF93DF93CDB7DEB76A970FB6F894DEBF6F
:105560000FBECDBF1C0109871A872B873C874D874B
:105570005E876F87788B22E1E216F10408F035C070
:10558000F701EF57FD4F30813D8BCE0109960E9408
:105590007F1197FD04C0BC01C1010E94A1119A8531
:1055A000892F8F70D1011196EC911197E07FE82B34
:1055B0001196EC93119789858C93E295EF70EC30FE
:1055C00008F063C0F0E08827E751F54D8F4F0C9449
:1055D00070BAD72C122B122B772CF72A0B2D412CBB
:1055E000802C802C802C412C412C1D8ACECF10E0A9
:1055F00092959F709D3008F010C4E92FF0E0882745
:10560000EB5FF44D8F4F0C9470BA452B442D642DF5
:10561000442D0D2D0D2D442D442D0D2F0D2F442DDA
:10562000442D1B2C92959F709D3008F014C1E92FDA
:10563000F0E08827E15EF44D8F4F0C9470BA452B53
:10564000F92BEC2BAF2B2F2B2C2BD02BFB2B2B2C1C
:105650002B2CBA2BBA2B1B2C8889F10187838F85C1
:10566000D10116968C9316978E8515968C93159767
:105670008D8514968C9314979295907F11968C91AA
:1056800011978F70982B11969C93FD89FF2309F435
:1056900063C0D10111968C9182958F702F2F30E0CD
:1056A0008217130609F458C065EB77E08CE499E0A3
:1056B0000E94826FF101618162956F708CE499E0C4
:1056C0000E94798462EB77E08CE499E00E94826F1B
:1056D0006D898CE499E00E94798460EB77E08CE43A
:1056E00099E00E94826FD1010C9119821A821B826B
:1056F0001C821D821E821F8218868D898295807F62
:105700009A819F70892B8A830983EE24EA94FE2C68
:1057100011961C91119712962C91129713963C9109
:10572000139714964C91149715965C9115971696AD
:105730006C91169717967C91CE0101960E94982A3B
:10574000F10120833183428353836483758386838D
:105750009783C1010E944E2A88E0F1016EC18F85B6
:105760009889F1018683878190FB80F987838E85F4
:1057700085838BCF8D859E85AF85B889B7FD0EC09B
:105780008F3F9105A105B10529F024F08FEF90E03E
:10579000A0E0B0E0D10114968C9377CF80E0FACFEF
:1057A0006D857E858F85988920E0673FBFEF7B07F9
:1057B0008B079B076CF02FEF6115EAE07E078105F0
:1057C000910534F42AE030E040E050E00E9407BA4E
:1057D000D10114962C9359CF8F859889F101868336
:1057E000878190FB80F987838E8585838D8584836F
:1057F0004CCF8D85CFCFCD84DE84EF84F88820E038
:1058000030E0A901C701B6010E949BB860E087FDA6
:105810000FC020E030E04FE753E4C701B6010E941B
:10582000A3BB6FEF181624F0C701B6010E9474BB2A
:10583000F10164832ACFD10111968C9111978F7059
:10584000806C11968C9311978D859E8515969C93EF
:105850008E9314971ACF62E478E08CE499E00E946A
:10586000826F6A8562956F708CE499E00E947984FA
:105870006FE378E08CE499E00E94826FF10161812E
:10588000BFC092959F70933091F09C30A1F24D85EE
:105890005E856F857889F1014483558366837783BC
:1058A0009295907F81818F70982B9183EECEC1016C
:1058B0000E94B185D10114968C9314978F85988995
:1058C00016968C93169717968C91179790FB80F9E4
:1058D00017968C9317978E8515968C93159711961E
:1058E0008C9111978F70806211968C93CECECE01E1
:1058F00009960E94B185D10114968C931497EFCF2D
:1059000092959F709D3008F065C0E92FF0E08827E0
:10591000E357F34D8F4F0C9470BA452BAC2CD62C1B
:10592000572CD62CD62C9A2CC62CC62CC62CBA2C6E
:10593000C12C1B2C6D857E858F8598890E94A2B80D
:1059400020E030E040E251E40E94FBBAF1016483C0
:1059500075838683978399CE6D8570E090E080E0B3
:105960000E94A0B8D10114966D937D938D939C9362
:1059700017978BCE6D857E858F8598890E94A2B8FA
:10598000E5CF6D857E858F859889EACF9295907F4A
:10599000F10181818F70982B91838D859E85AF85D4
:1059A000B88984839583A683B7836FCE9295907FC1
:1059B000D10111968C9111978F70982B11969C9311
:1059C0008D859E85AF85B889F10184839583A683F3
:1059D000B7835BCE6DE278E08CE499E00E94826F41
:1059E0006A8562956F708CE499E00E9479846AE21E
:1059F00078E08CE499E00E94826FD10111966C915D
:105A000062956F708CE499E00E9479848CE499E04F
:105A10000E948B6E3ACE11E0EBCD4D855E856F8591
:105A20007889F10144835583668377839295907FCB
:105A300081818F70982B918388E0DE01119601900F
:105A40000D928A95E1F729813A814B815C816D81C4
:105A50007E818F8198856A960FB6F894DEBF0FBE5F
:105A6000CDBFDF91CF911F910F91FF90EF90DF900D
:105A7000CF90BF90AF909F908F907F906F905F90EE
:105A80004F903F902F900895963009F4C1C048F48C
:105A90006D85913071F06FEF70E0933051F060E000
:105AA00008C0973009F4C0C09A506D857E85923049
:105AB000B0F784E68F8788898E7F888B1E868A85DB
:105AC0008F7080628A876D872E8530E0AFEFB0E0FF
:105AD0000E9439BAC12CD12C7601CA946115F4E622
:105AE0007F078105910544F424E630E040E050E072
:105AF0000E9407BA69017A01112309F475C0DA8A94
:105B0000C98A2D852E8B022F10E088898695A82FB3
:105B1000A150BB0BB88FAF8B119609F0A4C09601B2
:105B2000203831050CF087C08FE790E08C199D0973
:105B3000809FD001819FB00D909FB00D11242FEF59
:105B400030E00E9487BA21E83EE740E050E00E9442
:105B500007BAD10117962C93ABE9B0E0A7019601E3
:105B60000E9426BA3FE7432E512C612C712CA301D1
:105B700092010E9407BA2C593F4F4F4F5F4F590176
:105B8000AEEFB1E0A70196010E9426BAA3019201EF
:105B90000E9407BAD8010E9426BA2FEF30E040E0F9
:105BA00050E00E9407BA89012F3F310519F014F027
:105BB0000FEF10E06DE178E08CE499E00E94826FD5
:105BC000B5018CE499E00E9480846FE078E08CE479
:105BD00099E00E94826FB8018CE499E00E94808471
:105BE0008CE499E00E948B6E6DED77E08CE499E097
:105BF0000E94826F8CE499E00E948B6E66ED77E0E4
:105C00008CE499E00E94826FC1010E944E2A3DCD32
:105C10006D857E858F8598892AE030E040E050E0F0
:105C20000E9407BAB90145CF6D857E858F85988919
:105C30000E946DBB3ECFA70120583109410951098F
:105C4000ABE9B0E00E9426BA2FE730E040E050E038
:105C50000E9407BA2C593F4F4F4F5F4F5901D10156
:105C600017961C92A7CF2F89388DAAEBBFEF0E9401
:105C70007FBA24E6822E912CA12CB12CA50194018F
:105C80000E9407BA29013A01B4E64B0E511C611C6F
:105C9000711C26E430E0AF89B88D0E9487BAA50157
:105CA00094010E9407BA49015A01EEE18E0E911C3F
:105CB000A11CB11C29893A89203831050CF094C007
:105CC0008FE790E0821B930B809FD001819FB00DE6
:105CD000909FB00D1124A50194010E9431BA9B013F
:105CE000AC01AFEFB0E00E9426BA24E63AE640E00D
:105CF00050E00E9407BAD10117962C93A701960194
:105D0000240D351D461D571DAEEFB1E00E9426BA89
:105D100023EE30E040E050E00E9407BA298B3A8B36
:105D20004B8B5C8BE989FA89FA8FE98FAFEFB0E092
:105D3000A70196010E9426BA2FE730E040E050E02C
:105D40000E9407BA7901FE89AF2FB0E029893A890C
:105D50004B895C890E9426BA2FEF30E040E050E08A
:105D60000E9407BA89012F3F310519F014F00FEF97
:105D700010E069E078E08CE499E00E94826F2AE00C
:105D800030E0B301A2018CE499E00E94966E63E0DA
:105D900078E08CE499E00E94826F2AE030E0B5015F
:105DA000A4018CE499E00E94966E6BEF77E08CE49E
:105DB00099E00E94826FB7018CE499E00E94808490
:105DC00063EF77E08CE499E00E94826FB8018CE485
:105DD00099E00E9480846AEE77E08CE499E00E946A
:105DE000826F698D7A8DF8CEA7019601205831090E
:105DF00041095109ABE9B0E00E9426BA2FE730E033
:105E000040E050E00E9407BA2C593F4F4F4F5F4F80
:105E10007901D10117961C92ACCF64EC77E08CE449
:105E200099E00E94826F6A8562956F708CE499E0B8
:105E30000E94798461EC77E01DCDCF92DF92FF92D2
:105E40000F931F93CF93DF938C01EB016A01CB017A
:105E50000E94FB11F82E882309F44EC0D0FE05C025
:105E6000F8016081CE010E948617D1FE3CC0F80186
:105E7000818182958F7044815581668177818730D9
:105E800030F08930D0F096EF980F923090F0EC819E
:105E9000FD81309771F090859F702EEF290F223091
:105EA00010F0911106C08295807F90859F70892B9C
:105EB0008087CE010E94071216C0EC81FD813097C9
:105EC00091F080858F709EEF980F923010F08111C5
:105ED0000AC04187528763877487EC81FD81808582
:105EE000807F8360808764E578E08CE499E00E949D
:105EF000826FC8010E944E2A8F2DDF91CF911F9192
:105F00000F91FF90DF90CF900895CF92DF92EF92A4
:105F1000FF920F931F93CF93DF938C017B016A0154
:105F2000CB010E94FB11D82F8823E1F1D7011496F1
:105F30008D919C91009709F44AC0FC01C0852C2FDB
:105F40002F703EEF320F323010F0211135C0C59561
:105F5000C595C595C595D0FE76C0C7010E94361679
:105F6000F8018083CC2309F441C0C295C07F8181B0
:105F70008F70C82BC183D70114968D919C91009787
:105F800089F1FC0120852F70223019F581859285D9
:105F9000A385B485F80184839583A683B783C8015C
:105FA0000E944E2A8D2FDF91CF911F910F91FF906C
:105FB000EF90DF90CF900895253049F460E00E9483
:105FC0008884009721F0DC011896CC91C0CFC0E006
:105FD000C2CF253039F460E00E948884009711F028
:105FE000FC01D4CF80E090E0DC01D4CFD70114963F
:105FF000ED91FC9180858295807F8595859585952D
:106000008595823021F0833081F0D0E0CBCF41857F
:10601000528563857485F80181818F70806A8183E0
:106020004483558366837783BDCF418552856385DD
:106030007485F80181818F708067818344835583E3
:1060400066837783AFCFCC2389F2C295C07FF801F6
:106050008ECFCF93DF9300D000D01F921F92CDB789
:10606000DEB7FC01608398E0DE01119601900D928D
:106070009A95E1F729813A814B815C816D817E811E
:106080008F81988528960FB6F894DEBF0FBECDBFDE
:10609000DF91CF910895CF93DF93EB0163E0FC0193
:1060A000808191810E948884FC01892BA9F08085E0
:1060B0008D7091F4C095D095CF6FAE0170E060E027
:1060C00081859285A385B4858C239523A623B72348
:1060D00081879287A387B487DF91CF910895CF936B
:1060E000DF93EB0163E0FC01808191810E94888451
:1060F000FC01892BB9F09085892F8D7099F4907FE0
:1061000092609087CC27CE01B0E0A0E04185528517
:1061100063857485842B952BA62BB72B818792875B
:10612000A387B487DF91CF910895CF92DF92EF924A
:10613000FF920F931F93CF93DF9300D000D01F9255
:106140001F92CDB7DEB76C017B0160FF03C0E894FE
:10615000E0F8F3F8F3FC0DC00E948D10663971056C
:106160008105910530F08091730690917406059732
:10617000E9F4B70166277370C6010E946F306FE9BA
:1061800077E08CE499E00E94826F8FEF9FEF289672
:106190000FB6F894DEBF0FBECDBFDF91CF911F9138
:1061A0000F91FF90EF90DF90CF90089519821A829F
:1061B0001B821C821D821E821F8218868A818F701C
:1061C0008A8340E053E0B601CE0101960E94852FFC
:1061D00060E073E0C6010E941C16E82AF92A0981D2
:1061E0001A812B813C814D815E816F817885C6014A
:1061F0000E942C8ECCCF3F924F925F926F927F92F3
:106200008F929F92AF92BF92CF92DF92EF92FF92C6
:106210000F931F93CF93DF93CDB7DEB7CC5BD1093C
:106220000FB6F894DEBF0FBECDBF4C01C755DF4F90
:106230000883C95AD040C655DF4F1883CA5AD04088
:10624000C555DF4F2883CB5AD040C455DF4F388324
:10625000CC5AD040C355DF4F4883CD5AD040C255A9
:10626000DF4F5883CE5AD040C155DF4F6883CF5A95
:10627000D040C055DF4F7883C05BD040CF54DF4F54
:10628000F982E882C15BD0405C2C0E94438DC754E8
:10629000DF4F688379838A839B83C95BD040C6556F
:1062A000DF4F8881CA5AD0408F70682E712CC09001
:1062B0007306D0907406C954DF4FD982C882C75B79
:1062C000D040CF54DF4FE881F981C15BD040309797
:1062D00021F0808181110C94643BD4011B968C9138
:1062E000882341F0C4010B96CF54DF4F99838883F4
:1062F000C15BD0406114710411F00C94AD3BCF54DC
:10630000DF4FE881F981C15BD040309711F00C94E8
:10631000683BF401658876886114710411F40C946B
:10632000AD3BC655DF4F8881CA5AD0408F7011F0FF
:106330000C94AD3B662DCE0187559F4F0E94CC102B
:10634000C756DF4F2883C959D040C656DF4F388320
:10635000CA59D040C556DF4F4883CB59D040C456A8
:10636000DF4F5883CC59D040C356DF4F6883CD5997
:10637000D040C256DF4F7883CE59D040C156DF4F50
:106380008883CF59D040C056DF4F9883C05AD04041
:106390000C94AD3BCE0187559F4F0E944E2AF401CD
:1063A00080819181009711F40C94F03BFDE06F1611
:1063B000710409F0ABC00E94EF84082F10E0063092
:1063C0001105A4F40E941D73009739F0DC011896A2
:1063D0002C911897207F18962C93BC01F401808192
:1063E00091810E945A840F5F1F4FE9CF65E0D4016D
:1063F0008D919C910E9488848C01892BE1F410E09E
:1064000000E0C801C454DF4F0FB6F894DEBF0FBEE2
:10641000CDBFDF91CF911F910F91FF90EF90DF9053
:10642000CF90BF90AF909F908F907F906F905F9034
:106430004F903F900895C755DF4F8881C95AD0408B
:106440008031E8F6CE0187559F4F0E943A1116160B
:1064500017061806190624F4F80180858D70A1F03E
:10646000D80118968C9118978F7018968C936CE0C1
:1064700077E08CE499E00E94826F8CE499E00E94BE
:106480008B6E01E010E0BDCF0E94438D6B017C015B
:10649000CE0187559F4F0E943A11C60ED71EE81EA7
:1064A000F91EF801C186D286E386F486C755DF4F10
:1064B0008881C95AD0408295807F8260808761E060
:1064C00077E08CE499E00E94826FCE0187559F4F60
:1064D0000E943A11AB01BC012AE030E08CE499E063
:1064E0000E94966E6BEF76E08CE499E00E94826FDA
:1064F000D80119964D915D916D917C911C972AE080
:1065000030E08CE499E00E94966EB7CFC755DF4F1C
:10651000F880C95AD040B4E0FB1609F400C3BF1597
:1065200030F0FF2009F476C0B12CA12CB5C288EF61
:106530008F0D8230C8F788E0FE01E755FF4FDE017E
:10654000119601900D928A95E1F7C655DF4F88812B
:10655000CA5AD040807F09F435C3CE0187559F4F7A
:106560000E943A118B01672B09F42CC389E0F812C1
:1065700003C0119501951109B401CE0187559F4FB4
:106580000E941E8560E0CE0187559F4F0E942930F2
:106590006A962FAF6A976B963FAF6B976C964FAF2B
:1065A0006C976D965FAF6D976E966FAF6E976F96A7
:1065B0007FAF6F97A0968FAFA097A1969FAFA1973F
:1065C00092E06916710409F448C30CF0FEC2CC24B1
:1065D000C3946114710409F0A7CFC655DF4FE88159
:1065E000CA5AD040E295EF70E150EB3008F0BBC3DF
:1065F000F0E08827E150FD4C8F4F0C9470BA2F3695
:106600002F36B336B336B3368E366A366A366A36C6
:106610004C364C3619821A821B821C821D821E82C5
:106620001F8218868A818F708A83C655DF4F8881C2
:10663000CA5AD040807F09F477CFE9E06E16710422
:1066400009F42CC20CF013C16114710409F433C1B4
:1066500022E06216710409F067CFB12CA12CC12C85
:1066600033243A94B401CE0101960E941E858A819A
:10667000982F92959F70945F9F70923060F4C655EA
:10668000DF4F9881CA5AD04092959F70923019F48A
:106690008F7080628A83D40118969C91973071F430
:1066A000C655DF4F8881CA5AD040807E803211F0B3
:1066B000803421F48A818F7080628A83F401A185FD
:1066C000B285892F90E0109741F0ED91FC911197E0
:1066D000028CF38DE02DCD0119957C01C755DF4F5C
:1066E0000881C95AD040C655DF4F1881CA5AD040D8
:1066F000C555DF4F2881CB5AD040C455DF4F388174
:10670000CC5AD040C355DF4F4881CD5AD040C255F6
:10671000DF4F5881CE5AD040C155DF4F6881CF5AE4
:10672000D040C055DF4F7881C05BD040CE0101968C
:106730000E94982ACF57DF4F2883C158D040CE57A8
:10674000DF4F3883C258D040CD57DF4F4883C358FE
:10675000D040CC57DF4F5883C458D040CB57DF4F81
:106760006883C558D040CA57DF4F7883C658D04099
:10677000C957DF4F8883C758D040C857DF4F988329
:10678000C858D040CE0101960E944E2ACC2051F12B
:10679000C655DF4F8881CA5AD04082958F709FE0DE
:1067A000980F9F70923020F08A5F8F708230D0F403
:1067B0008A8182958F7081508230A0F42D8130E0E3
:1067C000AFEFB0E00E9439BA2FEF6115F4E67F0712
:1067D0008105910534F424E630E040E050E00E9469
:1067E00007BA2D8388E0FE013196DE01A755BF4F21
:1067F00001900D928A95E1F72AE0B22AD12CD401BA
:1068000018968C911897873009F003C4552009F425
:1068100017C31296ED91FC9190859F70953009F009
:106820000FC3C954DF4F88819981C75BD04005975A
:1068300009F406C3CF54DF4F48815981C15BD04072
:10684000BE0167557F4FCF010E94783E01E010E006
:10685000C755DF4F8881C95AD040853009F4ADC390
:1068600008F0F1C2833009F41CC3312C8AC38AE0DA
:106870006816710409F4BFC09BE06916710409F041
:1068800053CEB401CE0101960E941E85CE018755DC
:106890009F4F0E947F11BC01CE0101960E94A11161
:1068A00088E0FE013196DE01A755BF4F01900D92A1
:1068B0008A95E1F7EEC0C4010E94383F8C0161E087
:1068C00070E01816190614F070E060E08CE499E0AE
:1068D0000E9480846CE973E08CE499E00E941C6F54
:1068E000CE0187559F4F0E943A11AB01BC012AE0AF
:1068F00030E08CE499E00E94966E8CE499E00E946E
:106900008B6ECE0187559F4F101611060CF0D2C624
:106910000E943A11B12CA12C672B682B692B89F5A9
:1069200062E0CE0187559F4F0E942930CF56DF4F3E
:106930002883C159D040CE56DF4F3883C259D0404A
:10694000CD56DF4F4883C359D040CC56DF4F5883D4
:10695000C459D040CB56DF4F6883C559D040CA5682
:10696000DF4F7883C659D040C956DF4F8883C75957
:10697000D040C856DF4F9883C859D040AA24A3946A
:10698000BA2CCC24C394332433946CCE61E0CE0172
:1069900087559F4F0E942930C757DF4F2883C9581A
:1069A000D040C657DF4F3883CA58D040C557DF4F55
:1069B0004883CB58D040C457DF4F5883CC58D04081
:1069C000C357DF4F6883CD58D040C257DF4F78831D
:1069D000CE58D040C157DF4F8883CF58D040C057E2
:1069E000DF4F9883C059D040AA24A394BA2CCC245A
:1069F000C394312C37CEB401CE0101960E941E857E
:106A0000C255DF4F9881CE5AD0408A81282F2295D7
:106A10002F7041F0223049F0B12CA12CDD24D39409
:106A2000C12C37C18F7080628A83892F90E08536B0
:106A3000910514F084E690E08E8388E0FE013196A3
:106A4000DE01A755BF4F01900D928A95E1F762E0F4
:106A5000CE0187559F4F0E94CC10EA962FAFEA9740
:106A6000EB963FAFEB97EC964FAFEC97ED965FAFA1
:106A7000ED97EE966FAFEE97EF967FAFEF97C15819
:106A8000DF4F8883CF57D040C058DF4F9883C0581E
:106A9000D040A12CBAE0BB2ED12CC2CFB401CE0184
:106AA00001960E941E85C155DF4F6881CF5AD040A4
:106AB000C055DF4F7881C05BD0407170CE01019628
:106AC0000E94DC11C82E882309F457C188E0FE011A
:106AD0003196DE01A755BF4F01900D928A95E1F7DF
:106AE00062E0CE0187559F4F0E94CC10E2962FAFF7
:106AF000E297E3963FAFE397E4964FAFE497E596CE
:106B00005FAFE597E6966FAFE697E7967FAFE797BB
:106B1000E8968FAFE897E9969FAFE997BACFC4019F
:106B20000E94383F181619063CF562E0CE018755E1
:106B30009F4F0E942930AA962FAFAA97AB963FAFDE
:106B4000AB97AC964FAFAC97AD965FAFAD97AE96A7
:106B50006FAFAE97AF967FAFAF97E0968FAFE097EE
:106B6000E1969FAFE197AA24A394BA2CD12CCC2410
:106B7000C3943324339443CE61E0CE0187559F4FB5
:106B80000E942930A2962FAFA297A3963FAFA3975A
:106B9000A4964FAFA497A5965FAFA597A6966FAFA3
:106BA000A697A7967FAFA797A8968FAFA897A99605
:106BB0009FAFA997AA24A394BA2CD12CCC24C39418
:106BC000312C1DCE05E010E0D1CCB9E06B1671047C
:106BD00009F4D8C0EAE06E16710409F0A5CCC655D8
:106BE000DF4F8881CA5AD04082958F70823009F079
:106BF0001CC1C255DF4F6881CE5AD040060F111D0F
:106C000017FF02C010E000E00536110514F004E69D
:106C100010E0C255DF4F0883CE5AD04062E0CE016B
:106C200087559F4F0E94CC102A962FAF2A972B96FC
:106C30003FAF2B972C964FAF2C972D965FAF2D978C
:106C40002E966FAF2E972F967FAF2F9760968FAFB0
:106C5000609761969FAF61971CCFC12CBECCC35586
:106C6000DF4F6881CD5AD040060F111D17FF02C0BB
:106C700010E000E00F3F110519F014F00FEF10E0E5
:106C8000C355DF4F0883CD5AD040A12CEAE0BE2E79
:106C9000D12C33243A94B3CDC355DF4F6881798129
:106CA000CD5AD040060F171F17FF02C010E000E0BA
:106CB0000536110514F004E610E0012E000C220B3D
:106CC000330BC355DF4F088319832A833B83CD5A87
:106CD000D040DBCFC355DF4F688179818A819B81AA
:106CE000CD5AD0400E946DBB600F711F77FF02C06C
:106CF00070E060E06536710514F064E670E0072E20
:106D0000000C880B990B0E94A2B8C355DF4F688313
:106D100079838A839B83CD5AD040B7CFC355DF4F49
:106D200028813981CD5AD0404AE0409FC001419F1F
:106D3000900D1124820F931F97FF02C090E080E016
:106D4000893EF3E09F0714F088EE93E0092E000CD3
:106D5000AA0BBB0BC355DF4F88839983AA83BB83E0
:106D6000CD5AD04092CF88E0FE013196DE01A75582
:106D7000BF4F01900D928A95E1F7B12CA12CDD2433
:106D8000D39487CFC655DF4F8881CA5AD0408295A9
:106D90008F70823009F049C0C155DF4F6881CF5AEA
:106DA000D040C055DF4F8881C05BD040782F7170D4
:106DB000060F171F0E3621E012072CF417FF05C02F
:106DC0000DE611E002C010E000E0C155DF4F08837E
:106DD000CF5AD040C055DF4F8881C05BD04010FBF8
:106DE00080F9C055DF4F8883C05BD04062E0CE01A0
:106DF00087559F4F0E94CC1062962FAF6297639683
:106E00003FAF639764964FAF649765965FAF6597A2
:106E100066966FAF669767967FAF679768968FAFF6
:106E2000689769969FAF699734CE88E0FE013196E6
:106E3000DE01A755BF4F01900D928A95E1F7ECCD89
:106E40000FEF1FEF05CD863009F47CC0873009F0C5
:106E50000CCDC4010E943616F82E96E0891361C04D
:106E60006BED76E08CE499E00E94826F66E070E062
:106E70008CE499E00E9480848CE499E00E948B6EFF
:106E800062E0CE0187559F4F0E94293029AF3AAF6B
:106E90004BAF5CAF6DAF7EAF8FAF21969FAF2197A9
:106EA0003CC0C4010E943616853019F00DEF1FEF6B
:106EB000A8CA6CEE76E08CE499E00E94826F65E0EF
:106EC00070E08CE499E00E9480848CE499E00E9458
:106ED0008B6EB401CE0187559F4F0E941E8561E0E5
:106EE000CE0187559F4F0E94293022962FAF2297BF
:106EF00023963FAF239724964FAF249725965FAFF5
:106F0000259726966FAF269727967FAF27972896C7
:106F10008FAF289729969FAF29976894A0F8B0F86B
:106F2000A4CC63EC76E08CE499E00E94826F6F2D34
:106F300070E08CE499E00E9480848CE499E00E94E7
:106F40008B6EB4CFC4010E94383F1816190674F135
:106F5000B401CE0187559F4F0E941E8561E0CE018E
:106F600087559F4F0E94293029AB3AAB4BAB5CABA6
:106F70006DAB7EAB8FAB98AF6894A0F8B0F876E0BD
:106F8000372EC755DF4F8881C95AD040811132C092
:106F90006894A0F8C655DF4F8881CA5AD040807FD8
:106FA00069F16894B1F8D1101EC227C26FEA76E089
:106FB0008CE499E00E94826F79CFC4010E94383F2F
:106FC00018161906A4F462E0CE0187559F4F0E945F
:106FD000293029A73AA74BA75CA76DA77EA78FA743
:106FE00098AB6894A0F8B0F865E0362ECACF68E98F
:106FF00076E0DECF6894A0F8B0F8CCCF40E052E065
:10700000B401CE0187559F4F0E94852F8111C9CFB2
:10701000CACFAFEF3A12B1C0C4010E94383F332447
:107020003394181619060CF4ABC0312C60E976E0E5
:107030008CE499E00E94826FE32C032C000CFF0883
:10704000CD54DF4FF982E882C35BD040B7018CE4B6
:1070500099E00E94808469E876E08CE499E00E94DF
:10706000826F6C2D70E08CE499E00E9480848CE447
:1070700099E00E948B6ECF54DF4F48805980C15BEE
:10708000D0404114510409F484C064E07DE1C201A0
:107090000E943BB101E010E0892B09F44BC060E095
:1070A0007DE1C2010E943BB102E010E0892B09F4AE
:1070B00041C067ED75E0C2010E943BB105E010E000
:1070C000892BC1F163ED75E0C2010E943BB106E07E
:1070D00010E0892B79F165EC7CE1C2010E943BB1A3
:1070E0000AE010E0892B31F160EC7CE1C2010E94E2
:1070F0003BB10BE010E0892BE9F06AEC7CE1C201C6
:107100000E943BB10CE010E0892BA1F06AEC75E025
:10711000C2010E943BB10DE010E0892B59F066ECF2
:1071200075E0C2010E943BB110E000E0892B11F430
:107130000EE010E0C4010E943616E82EF12CE11496
:10714000F10431F4CD54DF4FE880F980C35BD040C7
:107150000115110509F436C0E016F106A1F063E748
:1071600076E08CE499E00E94826FB7018CE499E0AC
:107170000E9480848CE499E031C3332009F456CF17
:10718000CC24C39453CFCF54DF4F19821882C15BF4
:10719000D040C755DF4FE881C95AD040EA3008F0E7
:1071A00013C1F0E08827E852F74C8F4F0C9470BA67
:1071B000F139CD39C6391B39F139AD398A395D39E3
:1071C000F139F139D40119968D919C91009709F408
:1071D00016C9DC01ED91FC910488F589E02D72015E
:1071E000C755DF4F0881C95AD040C655DF4F1881B7
:1071F000CA5AD040C555DF4F2881CB5AD040C4551C
:10720000DF4F3881CC5AD040C355DF4F4881CD5A2B
:10721000D040C255DF4F5881CE5AD040C155DF4FC4
:107220006881CF5AD040C055DF4F7881C05BD040D5
:1072300019958C01E6C8C4010E943616853009F004
:1072400035CE64E676E08CE499E00E94826F65E0DA
:1072500070E08CE499E00E9480848CE499E00E94C4
:107260008B6EB401CE0187559F4F0E941E85F4019D
:107270008085853099F46CE0CE0187559F4F0E9440
:10728000293029A33AA34BA35CA36DA37EA38FA3AC
:1072900098A76894A0F8B0F8312C57C061E0CE01EF
:1072A00087559F4F0E942930298F3A8F4B8F5C8FD3
:1072B0006D8F7E8F8F8F98A3ECCFC4010E943616FE
:1072C000182F8630F9F463E576E08CE499E00E94AB
:1072D000826F66E070E08CE499E00E9480848CE428
:1072E00099E00E948B6E62E0CE0187559F4F0E940D
:1072F0002930298B3A8B4B8B5C8B6D8B7E8B8F8BE4
:10730000988FC7CF6BE376E08CE499E00E94826FA0
:10731000612F0ECE31101EC0B401CE0187559F4F94
:107320000E941E8561E0CE0187559F4F0E94293043
:1073300029873A874B875C876D877E878F87988BF5
:107340006894A0F8B0F856E0352E0FEF1FEFCC246C
:10735000C39429CE67E276E02BCE3320A1F062E021
:10736000CE0187559F4F0E94293029833A834B8352
:107370005C836D837E838F8398876894A0F8B0F8D0
:1073800045E0342EE2CF60E176E012CEC4010E94E7
:107390003616853009F07DCF89CD332019F06DEF99
:1073A00075E006CEC655DF4F8881CA5AD040807F2F
:1073B00031F4B401CE0187559F4F0E941E85689419
:1073C000A0F8F3E0BF2A68CFC655DF4F8881CA5ABC
:1073D000D040807F19F46894B0F85ECF23E0B22AE1
:1073E0005BCFDD2021F00CEF1FEF0C940132312C2C
:1073F0000FEF1FEFA114B10439F0A501B401CE01C4
:1074000087559F4F0E941D2FD40119968D919C91F5
:10741000009709F473C0CF54DF4FE880F980C15B57
:10742000D040DC01ED91FC910488F589E02DC75531
:10743000DF4F0881C95AD040C655DF4F1881CA5A5C
:10744000D040C555DF4F2881CB5AD040C455DF4FBF
:107450003881CC5AD040C355DF4F4881CD5AD040F7
:10746000C255DF4F5881CE5AD040C155DF4F688199
:10747000CF5AD040C055DF4F7881C05BD0401995BE
:107480008C01332021F0632DC4010E948617C9545A
:10749000DF4FE881F981C75BD040359721F0B50116
:1074A000C4010E94953063EE75E08CE499E00E947F
:1074B000826FB8018CE499E00E9480846CED75E0E5
:1074C0008CE499E00E94826F0E94438DAB01BC0165
:1074D000C754DF4FC880D980EA80FB80C95BD040A9
:1074E0004C195D096E097F098CE499E00E9476844D
:1074F0008CE499E00E948B6E0C940132F40180853B
:10750000853009F462C0863009F0BBCFC4010E9407
:10751000FC847C01009709F4B4CF712C612C97FF97
:1075200006C0F194E194F10866246394712CC701BC
:1075300001978634910508F0A4CFC755DF4F088125
:10754000C95AD04010E0DE2C61E08E2D0E948D895A
:10755000672859F10130110521F061E00C30110567
:1075600009F460E0062F10E08D2D0E945F8968EF1E
:1075700075E08CE499E00E94826FB7018CE499E099
:107580000E94808466EF75E08CE499E00E94826F2F
:10759000B8018CE499E00E9480848CE499E00E9418
:1075A0008B6E6894A0F8B0F87EC00130110551F0E0
:1075B00091E080E00C30110509F090E0092F182FC0
:1075C000602FD2CF01E010E0FBCFF2E06F16710424
:1075D00009F46CC02CE06216710429F06A946728E3
:1075E00009F04FCFDECFC4010E940016892B49F469
:1075F000D401ED91FC916081718185EC93E00E9452
:107600006690CE0187559F4F0E94F31020E030E036
:1076100048EC52E40E9401B90E946DBBCD54DF4F8B
:10762000688379838A839B83C35BD040CD54DF4FCB
:1076300048805980C35BD0400E94438DC72ED82E0E
:10764000E92EFF24C114D104E104F10421F4C12C7A
:10765000D12C7601C39462EF75E08CE499E00E942E
:10766000826FCD54DF4F68817981C35BD0408CE459
:1076700099E00E9480846DEE75E08CE499E00E94B0
:10768000826FB701A601662777272AE08CE499E08C
:107690000E943F6E8CE499E00E948B6EB601A201BD
:1076A000C4010E948A1801E010E0EBCE6894A0F8B3
:1076B000B1F8F9CF0E943A11672B682B692B09F0BA
:1076C00065C9B12CA12C93C96114710409F045C09E
:1076D0008081882311F40C948931CE018F549F4FFF
:1076E0000E9476193C01C655DF4F8881CA5AD040A6
:1076F0008F7071F5662DCE0187559F4F0E94CC107B
:10770000CF55DF4F2883C15AD040CE55DF4F388345
:10771000C25AD040CD55DF4F4883C35AD040CC55D4
:10772000DF4F5883C45AD040CB55DF4F6883C55ACA
:10773000D040CA55DF4F7883C65AD040C955DF4F75
:107740008883C75AD040C855DF4F9883C85AD04065
:107750006114710411F40C9489310E948D106B0135
:107760008B0167E377E08CE499E00E94826FB601B9
:107770008CE499E00E94808460E377E08CE499E0F7
:107780000E94826FD401ED91FC91608171818CE443
:1077900099E00E941C6F6AE277E08CE499E00E9415
:1077A000826FCF54DF4F68817981C15BD0408CE418
:1077B00099E00E941C6F64E277E08CE499E00E94FB
:1077C000826F083C110514F00C94CA3166E177E031
:1077D00085EA98E00E94826F85EA98E00E948B6EAD
:1077E0000FEF1FEF0C9401322F923F924F925F9256
:1077F0006F927F928F929F92AF92BF92CF92DF92C1
:10780000EF92FF920F931F93CF93DF93CDB7DEB725
:10781000A3970FB6F894DEBF0FBECDBF5C011B016E
:10782000D0907605DD2009F4B8C0809169068F5F9D
:1078300080936906E0917506F0917606309709F419
:10784000A4C086809780609075067090760661145B
:10785000710409F496C08114910409F492C0D40112
:1078600018968C918F70853091F7C4010E94EF8437
:10787000823068F3B401CE0101960E947418CE01E3
:1078800001960E94FB11882309F45EC060E074E059
:10789000CE0101960E941C16892B09F455C0188E42
:1078A000198E1A8E1B8E1C8E1D8E1E8E1F8E898D1C
:1078B0008F70898F40E053E0BE016F5F7F4FCE0134
:1078C00048960E94852F6BE777E08CE499E00E9450
:1078D000826F60E074E0CE0101960E944B308A8591
:1078E0009B85009789F1DC01ED91FC910488F58975
:1078F000E02DCC24C394F12CE12C088D198D2A8D18
:107900003B8D4C8D5D8D6E8D7F8D19958F3F9807CA
:10791000D9F0E981FA8160817181892BE9F48CE4E5
:1079200099E00E941C6F69E777E08CE499E00E947F
:10793000826F61E777E08CE499E00E94826F8CE4CB
:1079400099E00E948B6ED12CF40182809380CE014D
:1079500001960E94221277CF8CE499E00E941C6F5E
:107960006FE677E08CE499E00E94826F6BE677E047
:107970008CE499E00E94826F8CE499E00E948B6E07
:10798000E3CF8CE499E00E948B6E80916906815070
:1079900080936906D1101092760565E0D5018D912E
:1079A0009C910E9488844C01009709F489C0FC01D5
:1079B000D084D594D594D594D5944184528463844D
:1079C00074840E94438DDD2009F47AC0461A570A58
:1079D000680A790A188E198E1A8E1B8ED88E198D08
:1079E0001F70106A198F4C8E5D8E6E8E7F8EC30154
:1079F000B20128EE33E040E050E00E9407BA28A32D
:107A000039A34AA35BA3672B682B692B09F5E12CEB
:107A100090E1F92E0D2D2A8D3B8D4C8D5D8D6E8D57
:107A20007F8DC5010E942C8E2AE030E048A159A12B
:107A30006AA17BA18CE499E00E94966E60E977E0F0
:107A40008CE499E00E94826F8CE499E00E948B6E36
:107A500077FE36C0F2E04F1651046104F0E87F066D
:107A60007CF1E12C80E1F82E088D198D2A8D3B8D5B
:107A70004C8D5D8D6E8D7F8DC5010E942C8E19827F
:107A80001A821B821C821D821E821F8218861A8106
:107A90001F701A83D982CC24C394F12CE12C0D2DB4
:107AA0002B813C8140E05E816F817885C5010E9419
:107AB000FB30D40118968C9118978F7018968C9380
:107AC000B1E02B163104B9F460E073E0C5010E9407
:107AD0001C16009781F020917306309174062630B1
:107AE000310549F4BC01C5010E94953060E073E0A6
:107AF000C5010E944B30F501818592850097D9F42C
:107B000090E080E0A3960FB6F894DEBF0FBECDBF25
:107B1000DF91CF911F910F91FF90EF90DF90CF9069
:107B2000BF90AF909F908F907F906F905F904F909D
:107B30003F902F900895DC01ED91FC910484F58530
:107B4000E02D1995892BE1F2F50181859285DC0103
:107B5000ED91FC910480F581E02DB1011995D2CF12
:107B6000AF92BF92CF92DF92EF92FF920F931F934B
:107B7000CF93DF93CDB7DEB767970FB6F894DEBF2C
:107B80000FBECDBFE0917506F0917606309709F4EF
:107B90009EC0809169068F5F809369060681178178
:107BA000E0907506F0907606E114F10431F10115CC
:107BB000110519F1F80180858F708530A9F7C8018A
:107BC0000E94EF84823080F3B801CE0101960E94BA
:107BD0007418CE0101960E94FB11882331F062E0F7
:107BE00070E0CE0101960E94F43BF80102811381FE
:107BF000CE0101960E942212D3CF80916906815056
:107C0000809369068091730690917406059709F434
:107C10005EC00E94438D9B01AC0160918005709114
:107C200081058091820590918305AA24AA94BA2C9B
:107C3000650118EEE12E13E0F12E00E010E00E9445
:107C40000822082F882309F442C010E060919005B3
:107C50007091910561157105D1F1111138C0FB01C9
:107C600080858F708530D9F4CE0101960E947418FA
:107C700061E070E0CE0101960E94F43B892B59F03F
:107C80000E94438D609380057093810580938205E7
:107C900090938305102FCE0101960E942212E0914D
:107CA0009005F0919105309791F0828193819093A6
:107CB000910580939005892B49F6E0917506F09126
:107CC00076068681978190939105809390056796BB
:107CD0000FB6F894DEBF0FBECDBFDF91CF911F91DD
:107CE0000F91FF90EF90DF90CF90BF90AF900895ED
:107CF0004F925F926F927F928F929F92AF92BF92BC
:107D0000CF92EF92FF920F931F93CF93DF93CDB754
:107D1000DEB767970FB6F894DEBF0FBECDBF0097F2
:107D200009F4A4C0FC0120852F70253009F09EC005
:107D30002A015B0186809780809169068F5F80931E
:107D400069068114910409F48CC0F40180858F7058
:107D5000843009F082C061857285809175069091AA
:107D600076060E943F843C01009709F476C0FC012E
:107D700080858F70853009F070C0B301CE01019607
:107D80000E947418A114B104A9F0CE0101960E94BA
:107D9000FB11882379F0C12C7201F501008111815A
:107DA000228133814481558166817781CE0101969C
:107DB0000E94FB3060E0C3010E9488840097D1F1EB
:107DC000FC0120852F702230A9F581859285A3853D
:107DD000B4850797A105B10569F561E0C3010E946B
:107DE0008884A201B5010E94783EA114B10489F5EE
:107DF000882379F180916906815080936906CE01CC
:107E000001960E94221281E067960FB6F894DEBFB9
:107E10000FBECDBFDF91CF911F910F91FF90EF90DB
:107E2000CF90BF90AF909F908F907F906F905F901A
:107E30004F900895A114B10461F4CE0101960E94FF
:107E4000FB11882331F0CE0101960E94383F892B27
:107E500089F6CE0101960E942212F401828093805D
:107E600070CF8091690681508093690680E0CCCF05
:107E7000FF920F931F93CF93DF9300D000D01F92F8
:107E80001F92CDB7DEB78C0119821A821B821C8229
:107E90001D821E821F8218868A818F708A83D80174
:107EA000ED91FC91608171818CE499E00E941C6FDE
:107EB00069E677E08CE499E00E94826FC8010E9435
:107EC000FB11811119C060E677E08CE499E00E9413
:107ED000826F8CE499E00E948B6E0FEF1FEFC80158
:107EE00028960FB6F894DEBF0FBECDBFDF91CF91BD
:107EF0001F910F91FF900895C8010E943616F80156
:107F00009085973039F0853049F1D0F48130E9F02F
:107F1000823021F1D80119968D919C91009721F121
:107F2000DC01ED91FC910688F789E02D199501E0BF
:107F3000892B09F400E0802F0E94411410E0CFCF7C
:107F4000863019F08A50833028F761E477E08CE4BA
:107F500099E00E94826F01E010E0C1CF80E00E94B2
:107F6000411410E000E0BBCF40E052E0B801CE0188
:107F700001960E94852FF8018085873071F160F4A9
:107F8000833009F451C0843061F061E577E08CE41E
:107F900099E00E94826FE5CF883009F445C08930AE
:107FA000A1F7CE0101960E94B1858C0166E477E0CD
:107FB0008CE499E00E94826FB8018CE499E00E9401
:107FC00080848CE499E00E948B6E91E080E0012B2C
:107FD00009F490E0092F182F82CF0280F381E02D61
:107FE00080858F70853031F56EE577E08CE499E01F
:107FF0000E94826F50E040E070E060E0F801828112
:1080000093810E94783EF82E082F10E06BE577E010
:108010008CE499E00E94826F8F2D0E9441148CE4C1
:1080200099E00E948B6E5BCFCE0101960E943A11BF
:108030008B01BCCF10E000E0B9CF2F923F924F925E
:108040005F926F927F928F929F92AF92BF92CF92E8
:10805000DF92EF92FF920F931F93CF93DF93CDB7F1
:10806000DEB7CB55D1090FB6F894DEBF0FBECDBF3A
:108070000E94438D9B01AC01609188057091890538
:1080800080918A0590918B05AA24AA94BA2C650147
:1080900010E3E12E15E7F12E00E010E00E94082227
:1080A000882309F411C2E0917506F09176063097A5
:1080B00009F40AC2809169068F5F80936906268061
:1080C000378010E02114310409F446C1F1018085A4
:1080D0008F708530F9F460E0C1010E948884FC0152
:1080E00081859285A385B4850597A105B10591F495
:1080F000B101CE0101960E947418CE0101960E9432
:10810000FB116A968FAF6A97811108C0CE01019664
:108110000E942212F10122803380D4CF25961CAE1A
:108120001DAE1EAE1FAE259729961CAE1DAE1EAE0F
:108130001FAE299740E052E0BE016F5F7F4FCE0136
:108140008F5B9F4F0E94852FCE0101960E940016E3
:1081500065966CAF7DAF8EAF9FAF6597CE010196F0
:108160000E94FC844C01CE018F5B9F4F0E94F31054
:1081700069966CAF7DAF8EAF9FAF6997CE010196C8
:108180000E943616182F63962EAD3FAD6397B90146
:10819000330F880B990B0E94A2B820E030E048EC26
:1081A00052E40E94FBBA2B013C01CE0101960E94D1
:1081B000383F6C969FAF8EAF6C976CE972E18CE4A0
:1081C00099E00E94826F42E069966CAD7DAD8EAD04
:1081D0009FAD69970E94818666E972E18CE499E01F
:1081E0000E94826F42E0C301B2010E94818660E971
:1081F00072E18CE499E00E94826F612F70E08CE460
:1082000099E00E94808465960EAD1FAD65970115BB
:10821000110509F49AC00E94438DBB27A92F982FFE
:10822000872F0097A105B10521F481E090E0A0E03F
:10823000B0E09C01AD0144275527B80190E080E0F3
:10824000AA24AA94BA2CC12CD12C17E2E12E19E051
:10825000F12E00E010E00E940822882379F1F1015C
:108260006081718185EA98E00E941C6F60E872E18C
:1082700085EA98E00E94826FF1016081718184ED4E
:1082800093E00E94669065961FAE1EAE6597659658
:108290004CAD5DAD6EAD7FAD6597CE0101960E9490
:1082A0008A1862E070E0C4010E944316CE01019674
:1082B0000E9422126A961FAD6A972CCF20E030E010
:1082C00048E152E4C301B2010E94A3BB18163CF47A
:1082D000F1016081718180EE93E00E9466906C965E
:1082E0002EAD3FAD6C97232B19F461E070E0DBCF2E
:1082F00020E030E040E85FE369966CAD7DAD8EAD87
:108300009FAD69970E948EBA9B01AC01C301B20177
:108310000E949BB870E060E087FDC5CFA301920189
:1083200069966CAD7DAD8EAD9FAD69970E949BB88F
:108330001816DCF661E772E18CE499E00E94826F26
:108340008CE499E00E948B6EB1CF67E672E18CE419
:1083500099E00E94826FAACF809169068150809334
:1083600069060E94438D6093880570938905809308
:108370008A0590938B050E948D104B015C010E9431
:10838000438D2B013C010E94B784882309F466C009
:108390008091DA07811162C030E020E041E050E0D6
:1083A00060E4CE0101960E94632240E450E06DEB50
:1083B00076E1CE0101960E9454B16FE873E0CE01E0
:1083C00001960E94BBBE40E450E06EE372E1CE0134
:1083D00001960E9454B1B501A401CE018F5B9F4F5D
:1083E0000E94F80FBE016F5B7F4FCE0101960E9485
:1083F000118E30E020E041E050E060E4CE010196D3
:108400000E94632240E450E06DEB76E1CE010196DC
:108410000E9454B16FE873E0CE0101960E94BBBE8A
:1084200040E450E067E372E1CE0101960E9454B14E
:10843000C301B20128EE33E040E050E00E94E5B90C
:10844000BA01A901CE018F5B9F4F0E94F80FBE01B8
:108450006F5B7F4FCE0101960E94118E112309F4AC
:108460004DC061E672E18CE499E00E94826F0E9447
:108470008D10AB01BC018CE499E00E94768469E523
:1084800072E18CE499E00E94826F60916906062E89
:10849000000C770B8CE499E00E94808467E472E121
:1084A0008CE499E00E94826F40918405509185058B
:1084B00060918605709187058CE499E00E9476842E
:1084C0008CE499E00E948B6EC55ADF4F0FB6F8948A
:1084D000DEBF0FBECDBFDF91CF911F910F91FF90F7
:1084E000EF90DF90CF90BF90AF909F908F907F9054
:1084F0006F905F904F903F902F90089567E572E1E5
:108500008CE499E00E94826F0E948D10AB01BC0147
:108510008CE499E00E9476846FE472E1B2CF6F92AE
:108520007F929F92AF92BF92CF92DF92EF92FF9293
:108530000F931F93CF93DF93CDB7DEB7E2970FB6BC
:10854000F894DEBF0FBECDBF78AB6FA75AAB49AB77
:10855000672B09F484C2FA01309719F020812111A8
:1085600009C0FC012385222329F09C01255F3F4F90
:108570003AAB29AB5C01E9A9FAA93097E1F4F5011E
:10858000E588F688E114F10401F510E000E0CFA4DD
:10859000D8A83601600E711EF3018081882309F48A
:1085A00058C0082E000C990B0E945EBEF301808318
:1085B0000F5F1F4FECCF8081882309F3CE01C19656
:1085C0000E9476197C01892BD1F2FEE0EF16F104AE
:1085D000E1F62FA538A919821A821B821C821D82FE
:1085E0001E821F8218868A818F70806C8A833E83E8
:1085F0002D836EE0CE0101960E94CC1029A33AA3F0
:108600004BA35CA36DA37EA38FA398A7E9A8FAA8A8
:10861000CC24C39409811A812B813C814D815E81D8
:108620006F817885C5010E94FB30E2960FB6F89401
:10863000DEBF0FBECDBFDF91CF911F910F91FF9095
:10864000EF90DF90CF90BF90AF909F907F906F9012
:108650000895C114D10481F1F6018081882361F16C
:108660008D3209F46DC090ED980F9A3008F468C00F
:1086700008E010E0853211F10EEF1FEF8B37F1F0BB
:1086800007E110E08332D1F094E6692E98E0792E6C
:1086900001E010E0C3010E944BB1AC01B301C6017F
:1086A0000E9464B1892B51F00F5F1F4FF9E06F0EEC
:1086B000711C0931110571F70FEF1FEF19A21AA2F2
:1086C0001BA21CA21DA21EA21FA218A68AA18F7007
:1086D0008AA309A385E0E816F104A9F1E6E0EE1605
:1086E000F10411F407E110E09E2C6E2DCE0181966D
:1086F0000E94CC10298F3A8F4B8F5C8F6D8F7E8FAD
:108700008F8F98A301151105A9F104F50E3F1F4F96
:108710000CF0A5C1CE018F960E944B14092E000CBF
:10872000AA0BBB0B0097A105B10509F4D6C02AA17D
:108730002F70206A2AA38DA39EA3AFA3B8A7CDC094
:1087400010E000E0BBCF08E110E0CECF073111050B
:1087500009F441C108311105E9F660E0CE018196C6
:108760000E942930298B3A8B4B8B5C8B6D8B7E8BD7
:108770008F8B988F19821A821B821C828A818F703C
:1087800080668A83EFA5F8A9309709F48EC08081AE
:10879000882309F48AC06FA478A8F3018081882314
:1087A00059F08D3249F080538A3030F0FFEF6F1A64
:1087B0007F0A78AA6FA6EFCFC3010E94DAB06C01DE
:1087C0006EE270E0C3010E94C6BE009709F45AC071
:1087D000FC01018100330CF455C00A330CF055C084
:1087E000002E000C110B005311096CE270E0C30164
:1087F0000E94C6BE009709F04BC018AA1FA601151B
:10880000110509F449C02AE02C9DC0012D9D900D51
:1088100011241C141D041CF0119501951109080F59
:10882000191F012E000C220B330B0D831E832F8387
:108830003887692DCE0101960E94CC1029873A878E
:108840004B875C876D877E878F87988BDA80D29481
:108850008FE0D8223E01F9E26F0E711C10E000E0BB
:108860008FA598A9892B29F10330110511F10F5F0C
:108870001F4FCE018F960E944B14F3018193919369
:108880003F01EECF10E000E0B0CF09E010E0ADCF47
:10889000019698AB8FA7B3CF8601DD0C220B330B6B
:1088A0008A818F70806A8A83C0CF00E010E09801CF
:1088B000BCCFFAE0EF16F104E9F08BE0E816F10422
:1088C00069F1E9E0EE16F10491F5CE0101960E94FE
:1088D0003A11CE0181960E94DC11E9A8FAA8CC24B5
:1088E000C39409A11AA12BA13CA14DA15EA16FA126
:1088F00078A598CECE0101960E943A118AA1982FB0
:1089000092959F7039F0923041F7653608F064E631
:108910006EA3E3CF8F7080628AA3F7CFCE0101965A
:108920000E943A11CE0181960E94A111D6CF81E01A
:1089300090E0D11002C090E080E0800F911F823063
:10894000910539F164F4019741F688E0FE01319612
:10895000DE01919601900D928A95E1F7BECF8330AA
:10896000910539F1049709F0B8CF1BA509A5CE01EF
:1089700001960E943A118AA18F7080628AA36FA328
:1089800088A570FB80F988A70EA31DA36DA57EA501
:10899000C9CF19A5CE0101960E943A118AA18F7004
:1089A00080638AA36FA388A570FB80F988A71EA3A4
:1089B00094CF1BA509A5CE0101960E943A118AA168
:1089C0008F7080628AA36FA388A570FB80F988A747
:1089D0000EA31DA382CF60E0CE0181960E942930B4
:1089E00029833A834B835C836D837E838F8398874F
:1089F0007E01F9E0EF0EF11C10E000E08FA598A9D0
:108A0000892B71F00430110591F00F5F1F4FCE01DB
:108A10008F960E944B14F701819391937F01EECFC3
:108A20000330110589F00430110509F056CF9F85F8
:108A30002D853B8549858AA18F7080658AA34FA3C8
:108A40003EA32DA398A749CF9D852B8539858AA163
:108A50008F7080648AA33FA32EA39DA33ECF90E096
:108A600080E0E3CD2F923F924F925F926F927F9280
:108A70008F929F92AF92BF92CF92DF92EF92FF922E
:108A80000F931F93CF93DF93CDB7DEB7C955D109AD
:108A90000FB6F894DEBF0FBECDBF3C01562E6296D6
:108AA000EFAE62976396FFAE639764960FAF6497DD
:108AB00065961FAF659766962FAF669767963FAF2F
:108AC000679768964FAF689769965FAF69976A96A0
:108AD000CFAE6A972D2C4A2C3B2C009709F45EC12F
:108AE000FC0180858295807F859585958595859506
:108AF000843009F43EC12CF4882309F443C180E09A
:108B00002DC0853009F444C08630C9F76DEE73E09E
:108B1000C3010E943F844C01009709F46FC0B12C3F
:108B2000A12CD12CC12C6296EFAC62976396FFAC5E
:108B3000639764960FAD649765961FAD65976696CB
:108B40002FAD669767963FAD679768964FAD68976C
:108B500069965FAD6997652D0E943245C75ADF4F10
:108B60000FB6F894DEBF0FBECDBFDF91CF911F913E
:108B70000F91FF90EF90DF90CF90BF90AF909F90BC
:108B80008F907F906F905F904F903F902F900895BF
:108B9000809169068F5F8093690686809780811433
:108BA000910431F1A42CB32C6A96CFAC6A97D22CE5
:108BB0006296EFAC62976396FFAC639764960FADD5
:108BC000649765961FAD659766962FAD6697679615
:108BD0003FAD679768964FAD689769965FAD6997A7
:108BE000652DC4010E943245F40182809380D7CF65
:108BF0008091690681508093690681CF61EF73E0AF
:108C0000C3010E943F847C0166EF73E0C3010E94B0
:108C10003F846C01552039F0F1E05F1609F48AC0F9
:108C200010E000E00CC06BEF73E0C3010E943F84D2
:108C30004C0160E074E0C3010E943F848C01811408
:108C4000910409F443010115110509F48301E114AC
:108C5000F10421F46A96EFAC6A97F22CC114D104A6
:108C600011F4C42CD32C8114910409F494C0F401A0
:108C700080858F70843009F08EC0818492840115C4
:108C8000110509F493C0F80180858F70843009F0D4
:108C90008DC001851285E114F10409F4CBC0811463
:108CA000910409F492C064EC73E18CE499E00E94B1
:108CB000826FF701618572858CE499E00E941C6FD8
:108CC0006FEB73E18CE499E00E94826FB4018CE455
:108CD00099E00E941C6F8CE499E00E948B6ECE019B
:108CE0008F5A9F4F0E944E2AC114D10409F0FAC036
:108CF000F70180858F70843009F0F2C0618572853C
:108D0000CE0101960E94AA19CE0101960E94FB1184
:108D1000882359F08114910409F46BC050E040E0BD
:108D2000B401CE0101960E948F42CE0101960E94AD
:108D30002212D6C065E074E0C3010E943F844C015A
:108D40006AE074E0C3010E943F848C0181149104A5
:108D500009F0CDC06BEF73E0C3010E943F844C016A
:108D60000115110509F465CF892B09F070CF430176
:108D70006ECF10E000E0912C812CD12CC12CF12C75
:108D8000E12C5DCF10E000E0912C812CD12CC12C86
:108D9000F12CE12C5CCF912C812C71CFCA2CDB2CD7
:108DA0006A96EFAC6A97F22C912C812C00E020E0BF
:108DB00033E040E150E0BE016F5B7F4FCE018F5A40
:108DC0009F4F0E9468288C0166CF65EB73E18CE4AD
:108DD00099E00E94826FF701618572858CE499E0C9
:108DE0000E941C6F60EB73E18CE499E00E94826F3B
:108DF00076CFCC24C394F12CE12C62960FAD629710
:108E000063961FAD639764962FAD649765963FADEB
:108E1000659766964FAD669767965FAD679768965C
:108E20006FAD689769967FAD6997CE0101960E94F4
:108E3000FB307BCFC114D10409F452C001151105D8
:108E400009F44EC0F60180858F70843009F044C06B
:108E500069EA73E18CE499E00E94826FF601618512
:108E600072858CE499E00E941C6F64EA73E18CE4E3
:108E700099E00E94826FB8018CE499E00E941C6F17
:108E80008CE499E00E948B6EF6016185728540E466
:108E900050E0CE0101960E94FFBE0E94B784882355
:108EA000D9F08091DA07811117C06FE270E0CE012E
:108EB00001960E94C6BE892B51F4F60121853285A8
:108EC00043E050E060E4CE0101960E946322B801C5
:108ED000CE0101960E94118EE114F10409F008CF31
:108EE00081E03CCE0115110509F0ACCF01CF892BF3
:108EF00009F0ADCE9ECE8F929F92AF92BF92CF924D
:108F0000DF92EF92FF920F931F93CF93DF93CDB732
:108F1000DEB7A8970FB6F894DEBF0FBECDBF84E0D2
:108F2000E0E1F2E0DE01119601900D928A95E1F701
:108F3000FE0135968CE1DF011D928A95E9F73497A1
:108F40004F01DB01685F7F4F1D91812F90E0E4E0CE
:108F500095958795EA95E1F7805D9D4FFC018081AD
:108F6000F4018083E12FEF70F0E0E05DFD4F808140
:108F7000F4018183F2E08F0E911C6A177B0721F7C1
:108F8000198A1A8A80918E0590918F05892B09F490
:108F900078C0052FE42ED32E122F8CE499E00E9486
:108FA0008B6E6AE37AE08CE499E00E94826F42E083
:108FB000612F7D2D8E2D902F0E94818668E37AE0AF
:108FC0008CE499E00E94826FBE016F5F7F4F8CE45A
:108FD00099E00E941C6F66E37AE08CE499E00E94BD
:108FE000826F8CE499E00E948B6EBE016F5F7F4FB1
:108FF00080917706909178060E943F844C0120E092
:1090000030E04EEF52EC612F7D2D8E2D902F0E947F
:109010009BB88823B1F120E030E04AEA52E4612FA6
:109020007D2D8E2D902F0E949BB8882351F120E03A
:1090300030E0A901612F7D2D8E2D902F0E949BB8CD
:109040008823F9F019A21AA21BA21CA28AA18F7070
:109050008067F82E212F812F9D2DAE2DB02F8DA34F
:109060009EA3AFA3B8A7B12CA12CD12CC12CE9A0F1
:109070000BA11CA13EA14FA158A56FEFC4010E94F6
:109080003245A8960FB6F894DEBF0FBECDBFDF9174
:10909000CF911F910F91FF90EF90DF90CF90BF90F5
:1090A000AF909F908F9008956F927F928F929F9232
:1090B000AF92BF92CF92DF92EF92FF920F931F93E6
:1090C000CF93DF93CDB7DEB7A0970FB6F894DEBF8E
:1090D0000FBECDBF8C01862E7A01DC018D919C9153
:1090E0001197892B09F460C01496ED91FC9130978B
:1090F00009F45AC080818071BFEF6B1357C0B1F47F
:1091000081E0A0960FB6F894DEBF0FBECDBFDF9111
:10911000CF911F910F91FF90EF90DF90CF90BF9074
:10912000AF909F908F907F906F900895433051053E
:1091300039F3818082942FE0822266E775E08CE427
:1091400099E00E94826FD80113966C918CE499E0AB
:109150000E94798464E775E08CE499E00E94826F54
:10916000D8011496ED91FC9161816F708CE499E0C7
:109170000E94798461E775E08CE499E00E94826F37
:10918000682D8CE499E00E9479848CE499E00E9437
:109190008B6ED8011496ED91FC9181818F708812AD
:1091A00007C080818F7E808380E0ABCF8111FCCFB0
:1091B000198E1A8E1B8E1C8E1D8E1E8E1F8E18A24F
:1091C0008A8D8F708A8FD8011496ED91FC918181E0
:1091D0008F70881579F1B3E0EB16F10459F16FE661
:1091E00075E08CE499E00E94826FF80163818CE461
:1091F00099E00E9479846DE675E08CE499E00E9424
:10920000826FD8011496ED91FC9161816F708CE4AE
:1092100099E00E9479846AE675E08CE499E00E9406
:10922000826F682D8CE499E00E9479848CE499E047
:109230000E948B6EF80120813181FCE0F81508F462
:1092400016C1E82DF0E08827E75DF64B8F4F0C94B0
:1092500070BA36497349F4490B4A174AF449CD4963
:10926000F4491A4A254AE149284A344AD801149651
:10927000CD90DC90F60181818F70853009F4F7C0C4
:1092800050F48230C1F06DE174E0C9010E943F8466
:109290003C01912C4BC08730D1F08A30A1F766E1B8
:1092A00074E0C9010E943F843C01D6019C9092FA6F
:1092B000992490F83BC060E174E0C9010E943F84AA
:1092C0003C01D6019C9090FA992490F82FC06FE051
:1092D00074E0C9010E943F843C01F601908091FA3C
:1092E000992490F823C062E274E0C9010E943F848F
:1092F0003C01D8011496ED91FC91808180FB99246A
:1093000090F8982F9E7F80FF916090836114710484
:1093100069F461E0CE0149960E942930298B3A8B8D
:109320004B8B5C8B6D8B7E8B8F8B988FF801A08025
:10933000B18061EF73E0C5010E943F846C0166EF6C
:1093400073E0C5010E943F845C01892B81F4C11444
:10935000D10469F460E0CE0149960E942930298346
:109360003A834B835C836D837E838F839887D80198
:109370001496ED91FC916114710409F07CC0898D03
:10938000811179C0B82DBF708B2E8181807F882A92
:10939000818280818F7E8083B3CE67E274E0C901D1
:1093A0000E943F843C01D8011496ED91FC9180818C
:1093B00081FB992490F8982F9D7F81FF9260908384
:1093C000B5CF6DE274E0C9010E943F843C01D80131
:1093D0001496ED91FC91808182FB992490F8982F4E
:1093E0009B7F82FF9460EBCF6DE174E0C9010E9426
:1093F0003F843C01892B09F04CCF62E0CE014996B5
:109400000E94293029873A874B875C876D877E8742
:109410008F87988B3ECF63E374E0C9010E943F843D
:109420003C01D8011496ED91FC9190804CCF68E3FB
:1094300074E0F3CF6EE374E0C9010E943F843C0105
:10944000D8011496ED91FC9149CF64E474E0F4CF17
:109450006BE474E0C9010E943F843C01D80114967A
:10946000ED91FC91908023CF61E574E0F3CF912CD6
:10947000712C612C5BCF83E0E816F104B9F0982DD4
:109480009F70892E8181807F882A818280818F7E52
:109490008083E98CFA8C0B8D1C8D2D8D3E8D4F8D2C
:1094A00058A1692DC3010E9432452ACE81818F7057
:1094B000881509F425CE829490EF8922882A81822A
:1094C0008081806168CF8F929F92AF92BF92CF923E
:1094D000DF92EF92FF920F931F93CF93DF93CDB75D
:1094E000DEB767970FB6F894DEBF0FBECDBF61152C
:1094F000710599F1FA017B016C01E60FF71F1082EB
:109500000E948D104B018B0165E07AE08CE499E0BC
:109510000E94826FB4018CE499E00E94808462E032
:109520007AE08CE499E00E94826FB6018CE499E0C5
:109530000E941C6F6FEF79E08CE499E00E94826FCB
:109540000A3F1105ECF462EF79E085EA98E00E94A9
:10955000826F85EA98E00E948B6E67960FB6F8944A
:10956000DEBF0FBECDBFDF91CF911F910F91FF9056
:10957000EF90DF90CF90BF90AF909F908F90089525
:10958000B7018CE499E00E941C6F8CE499E00E9482
:109590008B6E809173069091740663E070E005977E
:1095A00049F062E070E0C6010E94F722009781F462
:1095B00061E070E0C6010E94F722009749F467EE6F
:1095C00079E08CE499E00E94826F8CE499E0C3CF4B
:1095D000C80ED91E68E574E0C6010E94D1BE892B71
:1095E00069F4F70101900020E9F73197EE19FF09BE
:1095F000329720F0C7010E945270AFCF6FE270E047
:10960000C6010E94C6BE8C01009741F0FC01108289
:109610008181843209F4A1CF0F5F1F4FF601808151
:10962000843209F49ACFB601CE0101960E94AA199C
:10963000CE0101960E94FB11882331F0A801B701E9
:10964000CE0101960E948F42CE0101960E94221205
:1096500084CF2F923F924F925F926F927F928F9220
:109660009F92AF92BF92CF92DF92EF92FF920F93B1
:109670001F93CF93DF93CDB7DEB7C556D1090FB691
:10968000F894DEBF0FBECDBFDC0114962D913C9146
:10969000232B09F4FEC59B012250310922303105EC
:1096A00008F091C23B014C01FC018281803409F435
:1096B000F7C208F04AC0843008F085C28091750571
:1096C0008F5F80937505A3016FEFC4010E9454481A
:1096D000D40112960C9112970695017013961C9165
:1096E00013978AEC810F803108F043C061E674E083
:1096F0008D919C910E943F847C010097D1F1FC01E7
:1097000080858F708530A9F580918B09181324C04E
:1097100080918C09803401F580918D0990918E099A
:109720005C01990FCC08DD0860E0C7010E948884C5
:10973000FC0181859285A385B485A816B906CA0661
:10974000DB060CF065C0512C3EC0823409F4A8C27F
:1097500008F439C28058AFCF10938B0980E480930E
:109760008C09812F0E94C98990938E0980938D095D
:10977000D7CF212F30E0F901E75BF64E8491F90154
:10978000E755F64E1491F901E151F64EF490FF20A1
:1097900009F43BC081110E94F888EF2DF0E0EE0F34
:1097A000FF1FE05BFA4FA591B491EC911E2331E0CD
:1097B00020E009F430E0832F922F552453940817AA
:1097C000190609F0C0CFF3E06F16710409F488C0E0
:1097D000D4011496ED91FC91E181EF70E150EC30F1
:1097E00008F07EC0F0E08827E750F44B8F4F0C94D0
:1097F00070BA1A4C964D504C864C964D9F4C964DD7
:10980000D34C004D194D5B4D7D4D90E080E0D5CFA0
:1098100061E0C7010E94888455245394FC0181852E
:109820009285A385B4858A159B05AC05BD050CF012
:10983000CACF89CF0E94438D9B01AC014427552795
:10984000D4011496ED91FC916281738190E080E0E7
:10985000AA24AA94BA2CC12CD12C18EEE12E13E024
:10986000F12E00E010E00E9408228823C9F1F401E3
:109870000081118163E374E0C8010E943F84892B59
:1098800041F468E374E0C8010E943F84892B09F425
:109890000EC142E050E063E0C4010E94544820C081
:1098A0000E94438D9B01AC0144275527D401149697
:1098B000ED91FC916281738190E080E0AA24AA94EA
:1098C000BA2CC12CD12C1CE2E12EFF24F39400E031
:1098D00010E00E94082242E050E064E0811184C060
:1098E000D4011496ED91FC91808183FB992790F926
:1098F000951509F4D2C1982F907E09F439C1982F9B
:10990000907E90528F71892B808358C10E94438D25
:109910009B01AC0144275527D4011496ED91FC918D
:109920006281738190E080E0AA24AA94BA2CC12CB1
:10993000D12C16E9E12EF12C00E010E0CACF0E94F4
:10994000438D9B01AC0144275527D4011496ED911A
:10995000FC916281738190E080E0AA24AA94BA2CE1
:10996000C12CD12C18EEE12E13E0F12E00E010E016
:109970000E940822882309F4B3CFF40100811181E9
:109980006EE374E0C8010E943F84892B41F464E4D3
:1099900074E0C8010E943F84892B09F488C042E02A
:1099A00050E068E079CF0E94438D9B01AC014427D1
:1099B0005527D4011496ED91FC916281738190E05A
:1099C00080E0AA24AA94BA2CC12CD12C1CE2E12E4E
:1099D000FF24F39400E010E00E94082242E050E0EF
:1099E00069E0882309F47CCFC4010E9454480E9496
:1099F000438DD4011496ED91FC917383628370CFF3
:109A00000E94438D9B01AC0144275527D401149635
:109A1000ED91FC916281738190E080E0AA24AA9488
:109A2000BA2CC12CD12C16E9E12EF12C00E010E06B
:109A3000D3CF0E94438D9B01AC0144275527D4010D
:109A40001496ED91FC916281738190E080E0AA24EC
:109A5000AA94BA2CC12CD12C18EEE12E13E0F12ED1
:109A600000E010E00E940822882309F439CFF401B5
:109A7000008111816BE474E0C8010E943F84892B4E
:109A800039F461E574E0C8010E943F84892B21F01C
:109A900042E050E06BE000CF6DE274E0C8010E944C
:109AA0003F8442E050E066E0892B09F4F5CE42E0C5
:109AB00050E06DE0F1CE0E94438D9B01AC01442744
:109AC0005527D4011496ED91FC916281738190E049
:109AD00080E0AA24AA94BA2CC12CD12C1CE2E12E3D
:109AE000FF24F39400E010E00E940822882309F488
:109AF000F7CE42E050E06CE077CF0E94438D9B01AF
:109B0000AC0144275527D4011496ED91FC91628154
:109B1000738190E080E0AA24AA94BA2CC12CD12CA5
:109B200016E9E12EF12C00E010E0DECF0E94438D1B
:109B30009B01AC0144275527D4011496ED91FC916B
:109B40006281738190E080E0AA24AA94BA2CC12C8F
:109B5000D12C18E5E12E12E0F12E00E010E00E9479
:109B60000822882309F4BCCE42E050E060E094CEA5
:109B70000E94438DD4011496ED91FC911597738347
:109B80006283E181EF70552009F445C0E230F1F0C5
:109B900050F4EE23E9F1D4011496ED91FC9180810B
:109BA00050FA83F9B1CEE53089F0A3016AE0E730DD
:109BB00091F7C4010E9454488111EDCF8091750541
:109BC00081508093750590E080E065C3F4010081C9
:109BD000118167E274E0C8010E943F84892BA9F4D7
:109BE0006EE374E0C8010E943F84892B71F464E441
:109BF00074E0C8010E943F84892B39F46FE074E05F
:109C0000C8010E943F84892B19F0A30166E0D1CFDF
:109C1000A30161E0CECFE150ED3008F0BCCFF0E021
:109C20008827EA5EF14B8F4F0C9470BA234ECB4DD0
:109C3000264E264ECB4D294ECB4D4A4E4A4E4A4ECD
:109C40004A4E4A4E264EA30162E0B3CFA30165E01F
:109C5000B0CF0D911C9167E274E0C8010E943F846F
:109C6000892BA9F46EE374E0C8010E943F84892B1C
:109C700071F464E474E0C8010E943F84892B39F4D4
:109C80006FE074E0C8010E943F84892B19F0A301A2
:109C900067E08FCFA30160E08CCF8F71806434CEFA
:109CA000B3E06B16710409F48ECF61E674E0F40141
:109CB000808191810E943F848C01D40113968C9104
:109CC00090918B098913CEC090918C09903409F042
:109CD000C9C080918D0990918E093C010115110533
:109CE00009F4F0C0F80120852F70253009F0EAC092
:109CF000C8010E94EF84A4968FAFA497843008F423
:109D0000BDC063E0C8010E948884DC0119968D9172
:109D10009C913AE0D32ED89EF001D99EF00D1124EB
:109D2000A396FFAFEEAFA39762E0C8010E948884BC
:109D3000DC0119968D919C91D89E7001D99EF00CF2
:109D4000112457010F2C000CCC08DD0861E0C8017C
:109D50000E948884A6969FAF8EAFA69760E0C80148
:109D60000E948884FC0121843284438454849301BA
:109D7000072C000C440B550B2219330944095509D3
:109D8000A396AEADBFADA397BD01BB0F880B990BDA
:109D90006A197B098C099D090E94D5B9A696EEAD7A
:109DA000FFADA69721853285438554852219330955
:109DB000440955090E9407BAA20EB31EC41ED51E3F
:109DC000A496FFADA497F53009F46BC081E090E054
:109DD000A396EEADFFADA397AF01FF0F660B770B18
:109DE0004A155B056C057D050CF464C0B601A50140
:109DF00057010F2C000CCC08DD084A155B056C05DB
:109E00007D050CF45CC05A016B01A496FFADA497CC
:109E1000F23009F06BC06301770CEE08FF0860E0D8
:109E2000C8010E948884FC0181859285A385B48540
:109E3000C816D906EA06FB060CF447C261E0C80161
:109E40000E948884FC0181859285A385B4858C1548
:109E50009D05AE05BF050CF0B6CE81E090E0A0E018
:109E6000B0E036C280938B0990E490938C090E94F5
:109E7000C98990938E0980938D092FCF8AE0869DA2
:109E80005001879DB00C11240B2C000CCC08DD0870
:109E9000F12CE12C20E038E2A3963FAF2EAFA39740
:109EA00095CF64E0C8010E948884DC0119968D91E9
:109EB0009C918ECF66246A9423E0722E99CF712CE8
:109EC000612CA3CF2AE0289F5001299FB00C1124B8
:109ED0000B2C000CCC08DD08F12CE12C20E038E242
:109EE000A3963FAF2EAFA39781E090E0D4011496E4
:109EF000ED91FC91428153819301241B350B37FF77
:109F000003C0319521953109821793070CF4C1C024
:109F10008081982F929596959770963008F0BCC0E6
:109F20009F5F9295990F907E8F71892BB4C0F70136
:109F300061857285DB018C91811157C2A114B10436
:109F400009F474C0D50118968C9118978F708430DD
:109F500009F06CC019966D917C91CE0101960E941A
:109F6000AA19CE0101960E94FB11882309F45AC058
:109F70006114710409F461C0E114F10431F0F701D6
:109F800080858F70843009F441C025961CAE1DAECB
:109F90001EAE1FAE259729961CAE1DAE1EAE1FAE7F
:109FA000299723961FAD23971F7023961FAF2397E2
:109FB00081E022968FAF2297CC24C394F12CE12C20
:109FC00001E024962FAD249725963FAD259740E0DC
:109FD00027965FAD279728966FAD289729967FAD76
:109FE0002997CE0101960E94FB301CC00115110576
:109FF00029F0F80180858F70843019F068E674E0EC
:10A00000F4C161857285FB01808196CF618572857F
:10A01000FB018081882331F050E040E0CE010196C1
:10A020000E948F42CE0101960E942212D401149602
:10A03000ED91FC9173826282C6CD0115110531F05C
:10A04000D80118968C918F708430E9F025961CAE5B
:10A050001DAE1EAE1FAE259729961CAE1DAE1EAEC0
:10A060001FAE299723961FAD23971F7023961FAF0E
:10A07000239782E022968FAF2297CC24C394F12CB1
:10A08000E12C02E09ECFF80161857285DB018C91A5
:10A09000C1CF80818F7180838081803AB8F0C70101
:10A0A000FF0CAA0BBB0B8A159B05AC05BD0571F017
:10A0B000A396EEADFFADA397CF01FF0FAA0BBB0B8D
:10A0C0008A159B05AC05BD0509F07DCD46155705E4
:10A0D00009F479CD6D961CAE1DAE1EAE1FAE6D9708
:10A0E0006B968FAD6B978F7080666B968FAF6B970B
:10A0F0006D968CAD9DADAEADBFAD6D9765968CAFD9
:10A100009DAFAEAFBFAF65976996ACAEBDAECEAEFC
:10A11000DFAE69976FE375E08CE499E00E94826F8F
:10A12000D40113966C918CE499E00E9479846DE3DC
:10A1300075E08CE499E00E94826FCE018F5A9F4FA8
:10A140000E944E2A6DEE73E0F401808191810E949D
:10A150003F84B12CA12CD12CC12C6296EFAC62971C
:10A160006396FFAC639764960FAD649765961FADD9
:10A17000659766962FAD669767963FAD6797689629
:10A180004FAD689769965FAD69976FEF0E94324552
:10A19000D4010D911C9161EF73E0C8010E943F84CE
:10A1A0007C0166EF73E0C8010E943F848C01009738
:10A1B000E1F1FC0180858F708430B9F5618572858D
:10A1C00040E450E0CE0101960E94FFBE6FE270E0D5
:10A1D000CE0101960E94C6BE892B59F4D80119966A
:10A1E0002D913C9143E050E060E4CE0101960E9445
:10A1F000632200E020E032E040E150E0BE016F5B0E
:10A200007F4FCE018F5A9F4F0E9468280E94B784CB
:10A21000882359F08091DA07811107C0BE016F5B76
:10A220007F4FCE0101960E94118EE114F10409F4D2
:10A23000FDCEF70180858F70843009F0F7CE6185FF
:10A240007285CE0101960E94AA19CE0101960E9444
:10A25000FB11882309F4E6CECC24C394F12CE12C25
:10A2600062960FAD629763961FAD639764962FADAC
:10A27000649765963FAD659766964FAD669767960E
:10A280005FAD679768966FAD689769967FAD699780
:10A29000A8CE8FEF9FEFCB59DF4F0FB6F894DEBFFC
:10A2A0000FBECDBFDF91CF911F910F91FF90EF9027
:10A2B000DF90CF90BF90AF909F908F907F906F90E6
:10A2C0005F904F903F902F90089580E090E0DC01E8
:10A2D000F40124813581F90142815381052E000C5E
:10A2E000660B770B481759076A077B0709F46BCC95
:10A2F0003C01D4010D911C9161EF73E0C8010E94F3
:10A300003F845C0166EF73E0C8010E943F846C01EA
:10A31000A114B10419F4892B09F488CE62E274E027
:10A32000C8010E943F847C016DE174E0C8010E9475
:10A330003F848C0165E475E08CE499E00E94826FB3
:10A34000F40163818CE499E00E94798463E475E010
:10A350008CE499E00E94826FB3018CE499E00E9442
:10A3600080848CE499E00E948B6EC114D10409F4BE
:10A37000E5CDD60118968C9118978F70843009F02E
:10A38000DDCD19966D917C9140E450E0CE010196AF
:10A390000E94FFBE0E94B784882309F4CFCD80912C
:10A3A000DA078111CBCD6FE270E0CE0101960E94F9
:10A3B000C6BE892B51F4F6012185328543E050E079
:10A3C00060E4CE0101960E9463226114710409F4D5
:10A3D0000DCEE114F10439F0D70118968C918F70ED
:10A3E000843009F4A4CD65E674E0CE0101960E94A4
:10A3F000118EA4CD8F929F92AF92BF92CF92DF9297
:10A40000EF92FF920F931F93CF93DF9300D000D072
:10A41000CDB7DEB720918C0530918D05232B09F443
:10A42000C7C020917F052111C3C04C0180917F05D9
:10A430008F5F80937F05809169068F5F80936906A7
:10A440000E94438D9B01AC0160917B0570917C055E
:10A4500080917D0590917E05AA24AA94BA2C65016D
:10A460001BE0E12EF12C00E010E00E94082288237E
:10A4700009F452C0E0918C05F0918D050681178199
:10A4800001151105B9F1F80180858F70863071F5DD
:10A490006DEE73E0C8010E943F840097D1F0FC018B
:10A4A00020852F702530A9F4E680F780E114F104AF
:10A4B000E9F0FA82E982B801CE0101960E94361ACB
:10A4C000B401CE0101960E94294BF701E280F3808E
:10A4D000EDCF1A83098370E060E0CE0101960E94FF
:10A4E000361AB401CE0101960E94294BF80102816F
:10A4F0001381C6CFF3E08F16910451F00E94438D73
:10A5000060937B0570937C0580937D0590937E0519
:10A5100010928B0910928C0983E088169104F1F156
:10A520000E94438D9B01AC01609177057091780585
:10A530008091790590917A05AA24AA94BA2C650194
:10A5400018E8E12E13E1F12E00E010E00E9408224D
:10A55000882321F1E0918C05F0918D05068117810A
:10A560000115110589F0F80180858F70863041F45E
:10A570001A83098370E060E0CE0101960E94361ACA
:10A58000F80102811381ECCF0E94438D609377051F
:10A59000709378058093790590937A058091690688
:10A5A00081508093690680917F05815080937F055B
:10A5B00026960FB6F894DEBF0FBECDBFDF91CF91C8
:10A5C0001F910F91FF90EF90DF90CF90BF90AF90D1
:10A5D0009F908F9008954F925F926F927F92AF926B
:10A5E000BF92CF92DF92EF92FF920F931F93CF9380
:10A5F000DF93CDB7DEB767970FB6F894DEBF0FBE17
:10A60000CDBF6AE273E18CE499E00E94826F8CE432
:10A6100099E00E948B6E0E94438D2B013C0180913A
:10A620006906882349F10E94438D9B01AC01AA244D
:10A63000AA94BA2C650110E1E12E17E2F12E00E098
:10A6400010E0C301B2010E940822811115C00E94CE
:10A65000D37080917906811162C0809173069091C8
:10A660007406059711F00E94B03D0E941D4082E0E3
:10A6700090E00E94FA51D3CF80916906882351F06F
:10A6800067E073E185EA98E00E94826F85EA98E0CE
:10A690000E948B6E61EF72E18CE499E00E94826F00
:10A6A0008CE499E00E948B6E809192058F5F80937D
:10A6B0009205E0917506F09176063097D1F106810A
:10A6C000178101151105A9F1D80118968C918F7089
:10A6D0008530B9F7C8010E94EF84882391F3F8010F
:10A6E00060817181CE0101960E94AA19CE01019666
:10A6F0000E94FB11882359F08A859B85009739F0C9
:10A70000DC01ED91FC910284F385E02D1995CE01D9
:10A7100001960E942212F80102811381D2CF80910A
:10A72000770690917806892B09F497CF0E943423FD
:10A7300094CF109291051092900569EE72E18CE42D
:10A7400099E00E94826F8CE499E00E948B6E64E62F
:10A7500070E080E090E00E94FE8A1092F505109271
:10A760006A0661ED72E18CE499E00E94826F0E94BA
:10A770008D10AB01BC018CE499E00E94768480913D
:10A780008E0590918F050E94638710928F0510921D
:10A790008E0510928D0510928C05109276061092FF
:10A7A00075061092F7051092F60510926706109242
:10A7B0006606109265061092640610927806109252
:10A7C00077066CEC72E18CE499E00E94826F0E9443
:10A7D0008D10AB01BC018CE499E00E9476848CE47E
:10A7E00099E00E948B6E10926806809192058150CC
:10A7F0008093920567960FB6F894DEBF0FBECDBF6B
:10A80000DF91CF911F910F91FF90EF90DF90CF904C
:10A81000BF90AF907F906F905F904F900895809120
:10A82000DA078F5F8093DA07A89583E090E00E94B3
:10A83000FA510E94D3708091DA0781508093DA0731
:10A840000895CF92DF92EF92FF920F931F93CF93D1
:10A85000DF93FC012485243059F090E080E0DF9103
:10A86000CF911F910F91FF90EF90DF90CF900895BF
:10A870006A018B01EC01F12C8F2D0E949C7C8111CF
:10A8800027C0FC868C85843041F3209102023091F0
:10A8900003022F5F3F4F21F1309303022093020206
:10A8A000409102025091030220E061E00E94ED7BA2
:10A8B000F80182818F3FB9F483818F3FF9F484815D
:10A8C0008F3FE1F485818F3FC9F484E08C87C5CF49
:10A8D0008B7F8831B1F2F394F4E0FF12CDCFD2CF69
:10A8E00020E030ECD9CF811109C08381811106C0ED
:10A8F0008481811103C08581882339F3C114D10477
:10A9000021F3FC8480E590E00E94B387B8016E5F7C
:10A910007F4F8F2D0E94321BB6018F2D0E94211B6D
:10A9200064E070E08F2D0E94B6870E94438D6B011A
:10A930007C01F4E9CF0EF1E1DF1EE11CF11CCE0138
:10A940000E943B1B873149F161E070E080E090E0BC
:10A950000E94FE8A0E940F54CE010E943B1B882356
:10A9600009F4B3CF0E94438DC616D706E806F90650
:10A9700030F78C850E94D97BEC85F0E0EE0FFF1F4D
:10A98000E559F94F1182108284E08C8766ED74E1FD
:10A990008FEA98E00E94A66F60CF6BEC74E18FEABB
:10A9A00098E00E94A66F81E090E059CFA89583E0DF
:10A9B00090E00C94FA515F926F927F928F929F92E7
:10A9C000AF92BF92CF92DF92EF92FF920F931F93BD
:10A9D000CF93DF93CDB7DEB76D970FB6F894DEBF98
:10A9E0000FBECDBF80918E0590918F05892B09F404
:10A9F000E5C3809169068111E1C3809169068F5F8B
:10AA00008093690664EE7DE08BE998E00E94826F96
:10AA10008BE998E00E948B6E00918E0510918F0556
:10AA20006CE674E0C8010E943F84909376068093A0
:10AA3000750662E774E0C8010E943F849093F705B1
:10AA40008093F6056DEA74E0C8010E943F849093FC
:10AA50008D0580938C0569E774E0C8010E943F84EE
:10AA600090936706809366060E94A7276EE774E0BE
:10AA700080918E0590918F050E943F849093780677
:10AA800080937706009709F4BBC1209179062111C4
:10AA9000B7C1DC011696ED90FC9080916206909112
:10AAA0006306892B51F081E08093790664ED7DE0A7
:10AAB0008BE998E00E94826F55C06BE97DE08CE4E1
:10AAC00099E00E94826F8CE499E00E948B6E65E9A8
:10AAD0007DE08CE499E00E94826F0E948D10AB01B2
:10AAE000BC018CE499E00E9476848CE499E00E9499
:10AAF0008B6E8FE090E00E940EAE8C0188E1F80131
:10AB00008183128210821686158610924106109259
:10AB100040061092B7071092D9070E940D1481E7E2
:10AB2000A82E8FE0B82EB0921A06A092190692E7CE
:10AB3000C92E9FE0D92ED0921E06C0921D061093FA
:10AB4000630600936206012B09F0B1C063E87DE063
:10AB500085EA98E00E94826F85EA98E00E948B6EF9
:10AB60001092790610929C0510929B05CC24C394F8
:10AB7000D12CE114F10409F443C1809179068823B2
:10AB800009F43EC1D70118968C9118978F708630C2
:10AB900009F089C00D911C91FE0131965F014801B9
:10ABA000F0E18F0E911C3501D8018C910E94A91003
:10ABB000582EF80181810E94A9105294A0EF5A22C8
:10ABC000582AD5015D925D010E5F1F4F80169106D8
:10ABD00059F760E07DE08BE998E00E94826F609118
:10ABE0009B0570919C058BE998E00E94808469EF39
:10ABF0007CE08BE998E00E94826F80919B059091A8
:10AC00009C05F3E0880F991FFA95E1F720919905CB
:10AC100030919A05820F931F0E942D868BE998E050
:10AC20000E948B6E20919B0530919C05213131054E
:10AC3000D4F56091990570919A0548E0C901E3E067
:10AC4000880F991FEA95E1F7860F971F415058F139
:10AC5000FC01E40FF11D50815523C1F3220F331F76
:10AC60004091930550919405240F351FF901D1822D
:10AC7000C08228E0F301DC0101900D922A95E1F7F2
:10AC8000DC018C91883231F48091620690916306E8
:10AC90000E942B1F80919B0590919C05019690939B
:10ACA0009C0580939B05F701E280F38062CF88E8E2
:10ACB00090E00E940EAE90939A058093990567E705
:10ACC0007DE08CE499E00E94826F0E948D10AB01C0
:10ACD000BC018CE499E00E9476848CE499E00E94A7
:10ACE0008B6E82E290E00E940EAE9093940580936A
:10ACF00093056AE67DE08CE499E00E94826F0E94F1
:10AD00008D10AB01BC018CE499E00E9476848CE448
:10AD100099E00E948B6E8091990590919A05892BFC
:10AD200031F08091930590919405892B79F462E537
:10AD30007DE085EA98E00E94826F0E948D10AB0151
:10AD4000BC0185EA98E00E94768406CF8BE797E401
:10AD500090939605809395051092410610924006B7
:10AD60001092B7071092D9070E940D14B0921A06DC
:10AD7000A0921906D0921E06C0921D06809162060E
:10AD8000909163060E943E0F81E00E940B8A811120
:10AD900030C06FE37DE08CE499E00E94A66F0091E3
:10ADA000620610916306C8010E943E0F40E060EF0A
:10ADB000C8010E94371F0E94FB8AE0916206F09151
:10ADC000630681E080836FE17DE08CE499E00E947E
:10ADD000A66F80916206909163060E94EA1E882306
:10ADE00009F461CE63E17DE08CE499E00E94A66FF6
:10ADF0005ACE65E07DE08CE499E00E94A66FB0CE6B
:10AE00001092910510929005E0917506F0917606EA
:10AE1000309709F4D6C0E680F7800091750610914E
:10AE200076060115110509F4C5C0E114F10409F411
:10AE3000C1C0D70118968C918F70853091F7C701EA
:10AE40000E94EF84823068F3B701CE0101960E9420
:10AE50007418CE0101960E94FB11882309F448C0A2
:10AE60008A859B85009749F5CE0101960E94FC8456
:10AE70008C01912C812C97FF06C011950195110929
:10AE800088248394912CCE0101960E943616C82EF8
:10AE9000D12C89858530A9F1863051F5B02E61E03D
:10AEA000802F0E948D8961E0892809F461C0CA94CD
:10AEB000CD2809F061C060E05FC0DC01ED91FC913C
:10AEC0000484F585E02D1995892B49F08A859B85A9
:10AED000DC01ED91FC910284F385E02D19958A85C2
:10AEE0009B85DC01ED91FC910680F781E02D1995A1
:10AEF000D7011296ED90FC90CE0101960E9422128D
:10AF00008CCFCD2829F462E0CE0101960E948617ED
:10AF100060E071E0CE0101960E946F308D819E81CC
:10AF2000892B31F060E072E0CE0101960E946F3013
:10AF300061E0802F0E948D8960E0802F0E945F89F0
:10AF40006CEC7DE08CE499E00E94826FB8018CE4A7
:10AF500099E00E94808467EC7DE08CE499E00E9497
:10AF6000826F65EC7DE08CE499E00E94826FC0CF37
:10AF7000CA94CD2809F09FCFC62ED12C8B2D0E94CC
:10AF80005F8960EC7DE08CE499E00E94826FB801FB
:10AF90008CE499E00E9480846EEB7DE08CE499E083
:10AFA0000E94826FB6018CE499E00E9480846CEB71
:10AFB0007DE0D9CFF80186819781909391058093A8
:10AFC00090058CE499E00E948B6EE0918C05F091E5
:10AFD0008D05309709F48AC0809169068F5F809350
:10AFE0006906068117810115110509F47AC0D80197
:10AFF00018968C918F70863009F069C0198F088F70
:10B0000070E060E0CE0148960E94361A8C8D9D8DCE
:10B01000892B09F45CC080918E0590918F05892B56
:10B0200009F455C0E88CF98CF70180858F70863063
:10B0300099F56DEE73E0C7010E943F840097F1F02F
:10B04000DC0118962C9118972F702530B9F41696BC
:10B05000CD90DC90C114D104F9F0DA82C982B70135
:10B06000CE0101960E94361AED81FE811082118276
:10B0700012821382F601C280D380ECCFFA82E98279
:10B0800070E060E0CE0101960E94361A62E070E046
:10B09000CE0101960E94294BEC8DFD8D108211820C
:10B0A000128213828A8D843068F462E0823008F064
:10B0B00060E08B8D0E948D89EC8DFD8D8181807F7C
:10B0C000818305C0803441F060E0823431F0D801E2
:10B0D00012960D911C9187CF62E08B8D0E948D8915
:10B0E000F6CF809169068150809369066CEE7CE012
:10B0F0008BE998E00E94826F64EE7CE08BE998E037
:10B100000E94826F81E02091750630917606232B94
:10B1100009F480E00E942B146BED7CE08BE998E051
:10B120000E94826F81E020918C0530918D05232B48
:10B1300009F480E00E942B1464ED7CE08BE998E038
:10B140000E94826F81E02091660630916706232B72
:10B1500009F480E00E942B146BEC7CE08BE998E012
:10B160000E94826F81E02091770630917806232B30
:10B1700009F480E00E942B148BE998E00E948B6E0A
:10B1800066EC7CE08BE998E00E94826F0E948D1053
:10B19000AB01BC018BE998E00E9476848BE998E0D2
:10B1A0000E948B6E81E080936A068BE698E00E9495
:10B1B000E81B809169068150809369066D960FB6F1
:10B1C000F894DEBF0FBECDBFDF91CF911F910F91DD
:10B1D000FF90EF90DF90CF90BF90AF909F908F90B7
:10B1E0007F906F905F900895CF93DF93EC01FB0108
:10B1F0002481358140815181628173810E94966EE4
:10B20000CE01DF91CF910895AF92BF92CF92DF929E
:10B21000EF92FF921F93CF93DF9300D000D0CDB772
:10B22000DEB76C017C0110E08AE0A82EB12C13304F
:10B2300061F1F701828190E0B0E0A0E089839A8318
:10B24000AB83BC83BE82AD82BE016F5F7F4F8CE457
:10B2500099E00E94F45862E973E10E94826F1F5FD7
:10B26000FFEFEF1AFF0A143011F726960FB6F89485
:10B27000DEBF0FBECDBFDF91CF911F91FF90EF904A
:10B28000DF90CF90BF90AF900895F601858190E058
:10B29000B0E0A0E089839A83AB83BC83BE82AD8299
:10B2A000BE016F5F7F4F8BE998E00E94F45860E920
:10B2B00073E1D3CF0F931F93CF93DF9300D000D0D0
:10B2C000CDB7DEB70E94D5266DE37AE08BE998E032
:10B2D0000E94826FCE0101960E94C687CE01019620
:10B2E0000E9404590AE713E01A8309838091090830
:10B2F00090910A08A0910B08B0910C088B839C8355
:10B30000AD83BE83CE0101960E9404591A8309833E
:10B310001B821C821D821E8280E590E00E94B38702
:10B3200044E050E0BE016D5F7F4F81E090E00E94FD
:10B330002474CE0101960E9404591A8309831B824A
:10B340001C821D821E8280E590E00E94B38744E04B
:10B3500050E0BE016D5F7F4F85E090E00E94247455
:10B36000CE0101960E94045963E67AE08BE998E0E9
:10B370000E94826F88EC90E026960FB6F894DEBFAC
:10B380000FBECDBFDF91CF911F910F910895CF9246
:10B39000DF92EF92FF921F93CF93DF9300D000D004
:10B3A000CDB7DEB769E07AE08BE998E00E94826F62
:10B3B00080E8E82E88E0F82E10E090E1C92ED12C2C
:10B3C000F70181917F01803130F461E874E08BE90D
:10B3D00098E00E941C6F153041F1F7013197808190
:10B3E00090E0B0E0A0E089839A83AB83BC83DE82E7
:10B3F000CD82BE016F5F7F4F8BE998E00E94F458C9
:10B4000067E07AE00E94826F1F5F1630C9F62696C9
:10B410000FB6F894DEBF0FBECDBFDF91CF911F9165
:10B42000FF90EF90DF90CF9008958091850890E095
:10B43000B0E0A0E089839A83AB83BC83DE82CD82B7
:10B44000BE016F5F7F4F8BE998E00E94F4580E9425
:10B450008B6EDACFEF92FF920F931F93CF93DF9310
:10B4600000D000D01F92CDB7DEB77B01CE0107968A
:10B470009F938F9301979F938F9301979F938F93A0
:10B4800001979F938F9301979F938F9301979F931A
:10B490008F938E010F5F1F4F1F930F9383E894E0EC
:10B4A0009F938F93DB0113968C9113978F93129632
:10B4B0008C918F930E9486BF0FB6F894DEBF0FBEAB
:10B4C000CDBF0697ECF46AED7EE085EA98E00E9435
:10B4D000826FD70112966D917C9185EA98E00E9467
:10B4E0001C6F80E991E027960FB6F894DEBF0FBE7F
:10B4F000CDBFDF91CF911F910F91FF90EF900895F5
:10B500008091780890917908892B09F44BC00E94AA
:10B510006C80882309F446C0A0917808B09179081E
:10B5200052961C921E92519754961C921E925397BB
:10B5300084E890E01D969C938E931C971E961C9217
:10B540001E9780E090E350969C938E931F97ED9109
:10B55000FC9111970088F189E02D64E070E0CD0145
:10B5600019958091780890917908DC01ED91FC9112
:10B570000280F381E02D46E050E0B801199586E0A5
:10B58000F801A0E8B8E001900D928A95E1F780916A
:10B59000780890917908DC01ED91FC910488F58997
:10B5A000E02D19950E94C7596CEE7EE08BE998E07A
:10B5B0000E94826F88EC90E096CFCF93DF93CDB757
:10B5C000DEB72E970FB6F894DEBF0FBECDBF8091C9
:10B5D000690681116BC061E37EE08BE998E00E940F
:10B5E000826F8BE998E00E948B6E109298081092FF
:10B5F000970880E090E1909393088093920884E804
:10B6000090E090939A088093990881E08093940841
:10B6100080E090E2909396088093950886E898E001
:10B620000E94E61A8B37910509F0C4C01C821B8268
:10B630008BE592E09A83898386E898E09E838D83E8
:10B640008FEF9FEF98878F8380918E0590918F0564
:10B65000892B11F00E94EB52CE0101960E94958732
:10B6600090938F0580938E0586E898E00E943012B3
:10B6700080918E0590918F05892BD9F465E27EE04B
:10B6800085EA98E00E94826F85EA98E00E948B6EBE
:10B690006AEF74E0CE0109960E94C96DCE01099649
:10B6A0000E944693CE0109960E948A6D90E080E048
:10B6B00014C062E17EE08BE998E00E94826F8BE922
:10B6C00098E00E948B6E0E94DB54809178089091E4
:10B6D0007908892B59F481E090E02E960FB6F89402
:10B6E000DEBF0FBECDBFDF91CF9108950E946C8069
:10B6F000882389F3A0917808B091790852961C921A
:10B700001E92519754961C921E92539784E890E093
:10B710001D969C938E931C971E961C921E9780E0FC
:10B7200090E350969C938E931F97ED91FC91119707
:10B730000088F189E02D60E670E0CD0119956091F7
:10B7400078087091790840E0CE0109960E94086E51
:10B75000BE01675F7F4F8AE798E00E94906CCE0140
:10B7600009960E948A6D8091780890917908DC0191
:10B77000ED91FC910488F589E02D199564EF7DE049
:10B780008CE499E00E94826F6AE778E0CE01099626
:10B790000E94C06DBE01675F7F4F8CE499E00E94FC
:10B7A000746F8CE499E00E948B6ECE0109960E9422
:10B7B0008A6D91CF86E898E00E944912892BA1F00A
:10B7C00086E898E00E9473126AEF74E0CE01019659
:10B7D0000E94C96DCE0101960E944693CE0101964A
:10B7E0000E948A6D0E94BA9286E898E00E94301208
:10B7F00061E07EE08BE998E00E94826F8BE998E03F
:10B800000E948B6E53CF0E94DD5A892B49F486EF3C
:10B810009FEF909374068093730684EF91E00895F0
:10B8200088EC90E00895BF92CF92DF92EF92FF9262
:10B830000F931F93CF93DF9300D000D0CDB7DEB727
:10B840008C016B01FB0184819581892BD9F1E0800A
:10B85000F1806FE370E0C7010E94C6BE009791F1CE
:10B860009C012E193F09790137FD2CC06AEF74E065
:10B87000CE0101960E94C96DF601848195810097E1
:10B88000B9F08E159F0508F47C01F6016081718185
:10B89000FB01EE0DFF1DB0801082CE0101960E94CB
:10B8A000646DF60180819181E80EF91EF701B08286
:10B8B000BE016F5F7F4FC6010E94906CCE01019662
:10B8C0000E948A6D67E974E0C6010E940B6C8823B0
:10B8D00019F1F801128A118A80E090E19587848736
:10B8E00084E890E0948B838B81E0868780E090E20F
:10B8F000908B878781E090E026960FB6F894DEBFA4
:10B900000FBECDBFDF91CF911F910F91FF90EF90B0
:10B91000DF90CF90BF90089564EA74E0C6010E9462
:10B920000B6C882369F0F801128A118A148A138A31
:10B9300084E890E095878487168680E090E3D8CFEE
:10B9400090E080E0D9CFFF920F931F93CF93DF93C6
:10B9500000D000D0CDB7DEB78C01BC01CE0101967E
:10B960000E94C06DBE016F5F7F4F8CE499E00E9422
:10B97000746F8CE499E00E948B6ECE0101960E9458
:10B980008A6D6FE47FE0CE0101960E94926DBE0148
:10B990006F5F7F4FC8010E94F06BF82ECE010196B9
:10B9A0000E948A6DFF2069F0B801CE0101960E94C5
:10B9B000C06DCE0101960E944693CE0101960E9471
:10B9C0008A6D26960FB6F894DEBF0FBECDBFDF910D
:10B9D000CF911F910F91FF9008955F926F927F9288
:10B9E0008F929F92AF92BF92CF92DF92EF92FF928F
:10B9F0000F931F93CF93DF93CDB7DEB7C956D1090D
:10BA00000FB6F894DEBF0FBECDBF4C018B01F42EF4
:10BA1000642F8CE499E00E94798465EE79E08CE4EF
:10BA200099E00E94826FB801CE0101965C010E94EC
:10BA3000C06DB5018CE499E00E94746F8CE499E0CC
:10BA40000E948B6EC5010E948A6D92E0F91265C258
:10BA500063EE79E0C5010E94926DB501C8010E94B4
:10BA6000206CF82EC5010E948A6DFF2009F4CAC21D
:10BA700020E04DE251E0B40189E498E00E94247096
:10BA8000E0906406F09065066CED79E0CE018C598B
:10BA90009F4F0E94926D65ED79E0CE01825A9F4FD3
:10BAA0000E94926DCE018E5A9F4F0E94C687689663
:10BAB0001FAD689767960FAD67976696DFAC669780
:10BAC0006596CFAC65976AEF74E0CE0181960E94CF
:10BAD000C96DBE016F5D7F4FC5010E94C06D6C2DA9
:10BAE000C5010E94DB6C60EB74E00E940C6D6D2D53
:10BAF0000E94DB6C60EB74E00E940C6D602F0E9472
:10BB0000DB6C60EB74E00E940C6D612F0E94DB6CBB
:10BB1000BC01CE01885A9F4F0E94C06DC5010E9492
:10BB20008A6DCE0181960E948A6D60ED79E0CE012A
:10BB3000845B9F4F0E94926D6AEF74E0CE018A5B36
:10BB40009F4F0E94C96D08E718E0D80118966C91C4
:10BB500070E084E0759567958A95E1F7C5010E94CC
:10BB600040804D815E8169817A81CE018A5B9F4FE1
:10BB70000E94506CC5010E948A6DF80160856F704B
:10BB800070E0C5010E9440804D815E8169817A81AB
:10BB9000CE018A5B9F4F0E94506CC5010E948A6D46
:10BBA0000F5F1F4FF8E00E371F0779F66AEC79E058
:10BBB000CE01805C9F4F0E94926D69EA79E0CE01D0
:10BBC00081960E94926DBE016F5D7F4FCE01C89637
:10BBD0000E94C06DBE01605C7F4FCE01C8960E947E
:10BBE000266DBE016A5B7F4F0E94266DBE01645BBD
:10BBF0007F4F0E94266DBE01685A7F4F0E94266DBE
:10BC0000BE01625A7F4F0E94266D8C014AE0B50149
:10BC100080E590E00E94B7B1F50101900020E9F7BE
:10BC20003197AF014A195B09B501C8010E94506CF8
:10BC3000811103C0C8010E94C96CBE016C597F4FBD
:10BC4000C8010E94266DB7010E940C6DBC01C401A1
:10BC50000E94746FC4010E948B6ECE01C8960E9430
:10BC60008A6DCE0181960E948A6DCE01805C9F4FC5
:10BC70000E948A6DCE018A5B9F4F0E948A6DCE0121
:10BC8000845B9F4F0E948A6DCE01885A9F4F0E940D
:10BC90008A6DCE01825A9F4F0E948A6DCE018C59C7
:10BCA0009F4F0E948A6DC4010E948B6E64E670E013
:10BCB00080E090E00E94FE8AD401ED91FC9104881E
:10BCC000F589E02DC401199501E010E082C02296AB
:10BCD0006EAD7FAD229750E040E0CE0181960E948C
:10BCE0008F42892B09F448C118AE19AE1AAE1BAEAB
:10BCF0001CAE1DAE1EAE1FAE89AD8F7089AF40E089
:10BD000053E0BE016F5D7F4FCE01C8960E94852F24
:10BD100000E020E033E040E250E0B501CE01C896FB
:10BD20000E946828BC01C6010E94646D08EC10E105
:10BD300025C1EE2009F4EFC046E050E070E060E07D
:10BD4000C8010E948D6BD8016D917C91CE018196C6
:10BD50000E94AA19CE0181960E94FB1100E911E010
:10BD6000882399F189A5873061F4CE0181960E94DC
:10BD7000383F61E0892B09F462E0CE0181960E9490
:10BD8000861718AE19AE1AAE1BAE1CAE1DAE1EAE97
:10BD90001FAE89AD8F7089AF40E053E0BE016F5D8B
:10BDA0007F4FCE01C8960E94852F00E020E033E04F
:10BDB00040E250E0B501CE01C8960E946828BC015F
:10BDC000C6010E94646D08EC10E1CE0181960E94CC
:10BDD0002212C801C759DF4F0FB6F894DEBF0FBE5D
:10BDE000CDBFDF91CF911F910F91FF90EF90DF902A
:10BDF000CF90BF90AF909F908F907F906F905F900B
:10BE00000895F801608171810E943F847C01892B33
:10BE100009F040C104E911E0DCCFEE2009F47BC059
:10BE200049E050E070E060E0C8010E948D6B4AE09C
:10BE3000B401C5010E94086E41E050E06CE973E076
:10BE4000C8010E94506C4D815E8169817A81C80170
:10BE50000E94506C65E879E08CE499E00E94826F62
:10BE6000B801CE0181960E94C06DBE016F5D7F4F0B
:10BE70008CE499E00E94746F8CE499E00E948B6ED0
:10BE8000CE0181960E948A6D6DE779E0CE018196A0
:10BE90000E94926DF801848195812DA13EA18217A7
:10BEA0009307E1F4892BA1F1E080F18069A07AA0E9
:10BEB000D7018D917D01882359F1082E000C990B33
:10BEC0000E9456BE6C01F30181913F01082E000CC7
:10BED000990B0E9456BEC816D90651F3CE01819621
:10BEE0000E948A6D552041F021E048EC50E0B401F9
:10BEF00089E498E00E942470D8018D919C910E9461
:10BF00005270009711F484E991E08C01C5013DC0A5
:10BF100055245394E3CF01E97ECFB1E0FB1270C00A
:10BF200062EA79E0C5010E94926DB501C8010E94E4
:10BF3000F06B582EC5010E948A6D552049F1EE2004
:10BF400051F346E050E070E060E0C8010E948D6B64
:10BF50004AE0B401CE01805C9F4F0E94086EF80158
:10BF600060817181CE0181960E94AA19CE018196CD
:10BF70000E94FB118111ABCE00E911E0CE01819648
:10BF80000E942212CE01805C9F4F0E948A6D21CFB9
:10BF90006BE879E0C5010E94926DB501C8010E946D
:10BFA000F06BF82EC5010E948A6DF11036CF60E764
:10BFB00079E0C5010E94926DB501C8010E94F06B45
:10BFC000182FC5010E948A6D00E0112309F401CFEA
:10BFD00080E00E941F8468E479E08BE998E00E9489
:10BFE000826F8BE998E00E948B6E6AEF74E0C50166
:10BFF0000E94C96DC5010E944693C5010E948A6DC9
:10C0000000E063CE6BE979E0C5010E94926DB50155
:10C01000C8010E94F06BF82EC5010E948A6DF110D4
:10C0200088CE65E979E0C5010E94926DB501C8012D
:10C030000E94F06BF82EC5010E948A6DFF2001F36B
:10C04000EE2009F468CF45E050E070E060E0C80100
:10C050000E948D6B60EB74E0C8010E940B6C88231A
:10C0600039F0E0907506F0907606E114F10491F451
:10C070006AEF74E0C8010E940B6C811107C08091C7
:10C08000750690917606009709F0BBCEE0908E057C
:10C09000F0908F0520E048EC50E2B40189E498E08C
:10C0A0000E942470C4010E948B6E1C821B828BE54F
:10C0B00092E09A8389839E828D828FEF9FEF98878B
:10C0C0008F83B701C5010E941971F0CDAF92BF9265
:10C0D000CF92DF92EF92FF920F931F93CF93DF9354
:10C0E000CDB7DEB7C859D1090FB6F894DEBF0FBE81
:10C0F000CDBF8E010F5B1F4FD8011D921C92FE0118
:10C10000ED5BFF4F8EE1DF011D928A95E9F780918B
:10C11000780890917908892B09F49AC10E946C8063
:10C12000882309F495C1A0917808B09179085296B6
:10C130001C921E92519754961C921E92539784E81B
:10C1400090E01D969C938E931C971E961C921E97B2
:10C1500080E090E350969C938E931F97ED91FC9115
:10C1600011970088F189E02D60E270E0CD0119950A
:10C170004FE150E0B80180917808909179080E94D1
:10C18000C3807C018091780890917908DC01ED9161
:10C19000FC910488F589E02D1995E114F10409F466
:10C1A00057C1F801EE0DFF1D1082809185081F9286
:10C1B0008F93809184081F928F93809183081F92A0
:10C1C0008F93809182081F928F93809181081F9294
:10C1D0008F93809180081F928F9382EB94E09F93BE
:10C1E0008F931F9280E48F93FE0131966F01FF932E
:10C1F000EF930E9419BF67E270E18BE998E00E941B
:10C20000826FB8018BE998E00E941C6FB6018BE940
:10C2100098E00E941C6F8BE998E00E948B6E7E0173
:10C22000F1E6EF0EF11CD70113961C921E921297A5
:10C2300088EE93E0A0E0B0E0F70184839583A683C5
:10C24000B78384E0848782E093E0918380831686BD
:10C250001586108B0787128A118A80E590E0948BEF
:10C26000838B178A66E57FE08CE499E00E94826FF9
:10C270006AE778E0CE0187589F4F0E94C06DBE01EB
:10C2800067587F4F8CE499E00E94746F8CE499E0CA
:10C290000E948B6ECE0187589F4F0E948A6D61EE7F
:10C2A00074E0CE0185579F4F0E94C96D61EE74E026
:10C2B000CE0187589F4F0E94C96DBE0167587F4FBE
:10C2C000CE018D579F4F0E94C06D6AE778E0CE0186
:10C2D0008D579F4F0E94266DBE0165577F4F0E946C
:10C2E000266DBC01CE018F569F4F0E94C06DCE01BE
:10C2F0008D579F4F0E948A6DCE0187589F4F0E9495
:10C300008A6DCE0185579F4F0E948A6D83EE94E01F
:10C31000CD57DF4F99838883C358D040C957DF4F2B
:10C3200019821882C758D040C757DF4F1982188228
:10C33000C958D040CF56DF4F88819981C159D0402C
:10C34000CB57DF4F99838883C558D04061E270E1B5
:10C350008CE499E00E94826F0E948D10AB01BC01B9
:10C360008CE499E00E9476848CE499E00E948B6EC4
:10C3700064E670E080E090E00E94FE8A83EA9CE53B
:10C38000D7011E969C938E931D9768E878E680E50A
:10C3900093E70E9423B28C010FB6F894DEBF0FBE64
:10C3A000CDBF892BA1F183E090E00E940EAED801B1
:10C3B0001D969C938E931C97FC01F182E082128261
:10C3C000C7010E94431B882319F0C7010E94E81B84
:10C3D000D70151966D917C9152975396AD90BC9038
:10C3E0006115710509F44BC0CE0187589F4F0E941B
:10C3F000B86FA501BE0167587F4FC7010E94215445
:10C40000181619060CF487C1C8010E94297368EB3D
:10C410007FE08CE499E00E94826FEE24EA94FE2C87
:10C42000CE018F569F4F0E948A6DC701C856DF4FBD
:10C430000FB6F894DEBF0FBECDBFDF91CF911F9135
:10C440000F91FF90EF90DF90CF90BF90AF90089545
:10C4500040E250E069E570E1C8010E9472B16BE30F
:10C4600070E18BE998E00E94826FB8018BE998E057
:10C470000E941C6F8BE998E00E948B6E96CEF701AC
:10C4800067857089A501C7010E94FD12B9CF81EBB4
:10C490009FE09F938F931F930F930E94AAB2D7019F
:10C4A00056961C921E925597D8011C96ED91FC91C0
:10C4B000A080B1800F900F900F900F9093E3C92E42
:10C4C000D12CD501ED91FC910084F185E02DC501C1
:10C4D000199541975CF4B1E0CB1AD10839F064E1C9
:10C4E00070E080E090E00E94FE8AEBCF6E01E7E909
:10C4F000CE0ED11CDF92CF9281E69FE09F938F9367
:10C500001F930F930E94C7B20F900F900F900F9040
:10C510000F900F900197D1F4D6018D919C91F70166
:10C52000968B858B6AEF74E0CE0185579F4F0E94F2
:10C53000C96D80E0C12CFAE0CF1270C08A3009F0DA
:10C5400071C0CE0185579F4F0E948A6DD7015596C5
:10C55000ED90FC90B8ECEB16F10409F0BAC065E17F
:10C5600070E18BE998E00E94826F64EF71E080E0F7
:10C5700090E00E94FE8AED961FAE1EAEED97EF96FC
:10C580001FAE1EAEEF978FEF9FEFC158DF4F99831D
:10C590008883CF57D04085E492E0EB969FAF8EAF73
:10C5A000EB97CF57DF4F19830883C158D040F894D9
:10C5B00080918E0590918F05892B11F00E94EB528E
:10C5C000CE0187589F4F0E94958790938F05809347
:10C5D0008E057894C8010E94297380918E059091F0
:10C5E0008F05892B09F063C06AEF74E0CE0185578F
:10C5F0009F4F0E94C96DCE0185579F4F0E94469361
:10C60000CE0185579F4F0E948A6D6EEF7FE085EACD
:10C6100098E00E94826FF12CE12C02CF9DE0C912BC
:10C6200001C0C82EC8010E946EB2D82ED7011D9637
:10C63000AD90BC90A114B10499F1BAE08B1779F0D8
:10C64000EDE08E1761F0FFEF8F1749F0682FCE01F4
:10C6500085579F4F0E947C6C8C2DCD2C6CCFC15781
:10C66000DF4F88819981CF58D040892B91F0BE014E
:10C6700065577F4FCE0187589F4F0E94C06DCE01F6
:10C6800087589F4FF5011995CE0187589F4F0E94FB
:10C690008A6D6AEF74E0CE0185579F4F0E945A6DF4
:10C6A000FFEFDF12D9CFC8010E9429734ACF0E9441
:10C6B000DB5480916A06882329F00E945F8367FF1C
:10C6C0000E94B31567EF7FE08BE998E00E94826FCC
:10C6D000A7CEE0E3EE16E1E0FE0651F463EE7FE064
:10C6E0008BE998E00E94826FC8010E94297398CE5E
:10C6F0006BEC7FE085EA98E00E94826FC8010E949F
:10C700002973B70185EA98E00E94808485EA98E061
:10C710000E948B6E85CED7011F96BC901F975096B6
:10C72000AC90DF92CF9284EB9FE09F938F931F9307
:10C730000F930E94AAB2DF92CF928FEA9FE09F935D
:10C740008F931F930F930E94AAB2D8011C96ED916C
:10C75000FC9181E08283DF92CF928CEA9FE09F93ED
:10C760008F931F930F930E94AAB2D8011C96ED914C
:10C77000FC911282AF92BF9286E79FE09F938F93C6
:10C780001F930F930E94AAB20FB6F894DEBF0FBE9C
:10C79000CDBFB12C8DE6C82E8FE0D82E8B2D94E026
:10C7A0008902F0011124A3E8B0E0AC0FBD1FEA0F2D
:10C7B000FB1F80819181009709F469CE228133812A
:10C7C00021153105C1F33F932F939F938F93DF92F0
:10C7D000CF921F930F930E94AAB2B3940FB6F8940E
:10C7E000DEBF0FBECDBFDACF0F931F93CF93DF9382
:10C7F000EB0102970CF49DC00A811B8168E47FE085
:10C80000C8010E9428B1892B51F481E00E941F8445
:10C8100088EC90E0DF91CF911F910F91089564E42F
:10C820007FE0C8010E9428B1892B11F480E0EECF8F
:10C8300064E27FE08BE998E00E94826F0E945F8350
:10C8400063FB662760F981E0682770E08BE998E078
:10C850000E9480848BE998E00E948B6E809178081A
:10C8600090917908892B09F454C00A811B810E9498
:10C870006C80882309F44DC0F80101900020E9F78D
:10C880003197E01BF10BB09708F043C0A0917808F6
:10C89000B091790852961C921E92519754961C9210
:10C8A0001E92539784E890E01D969C938E931C975C
:10C8B0001E961C921E9780E090E350969C938E9358
:10C8C0001F97ED91FC9111970088F189E02D60E2AE
:10C8D00070E0CD011995B8018091780890917908A0
:10C8E0000E941C6F8091780890917908DC01ED918D
:10C8F000FC910190F081E02D60E01995809178081D
:10C9000090917908DC01ED91FC910488F589E02D86
:10C9100019956A817B818BE998E00E941C6F6DE11B
:10C920007FE08BE998E00E94826F8BE998E00E949B
:10C930008B6E809173069091740602977CF10E9431
:10C940006660883C910539F424E030E03093740649
:10C95000209373065FCF8F3F9807C9F462E07FE0B2
:10C960008CE499E00E94826F8CE499E00E948B6EC7
:10C970001092680683E090E09093740680937306AB
:10C980008BE698E00E94E81B89EC90E043CF209171
:10C990006A062111D9CF2FE030E0D8CF65EF7EE0D5
:10C9A00085EA98E00E94826F85EA98E00E948B6E8B
:10C9B00084EF91E02FCF0895FC0124813581621727
:10C9C000730748F480819181009729F0860F971FA3
:10C9D000FC018081089580E008950895AF92BF9290
:10C9E000CF92DF92EF92FF920F931F93CF93DF933B
:10C9F0006C017B018B01040F151FEB015E01AE186A
:10CA0000BF08C017D10759F06991D601ED91FC918B
:10CA10000190F081E02DC6011995892B79F7C501A8
:10CA2000DF91CF911F910F91FF90EF90DF90CF900A
:10CA3000BF90AF900895FC01538D448D252F30E0B9
:10CA4000842F90E0821B930B541710F0CF9608951B
:10CA500001970895FC01918D828D981761F0A28D48
:10CA6000AE0FBF2FB11D5D968C91928D9F5F9F730E
:10CA7000928F90E008958FEF9FEF0895FC01918DC4
:10CA8000828D981731F0828DE80FF11D858D90E031
:10CA900008958FEF9FEF0895FC01918D228D892FCE
:10CAA00090E0805C9F4F821B91098F7399270895B6
:10CAB0008FEA98E00E944C6521E0892B09F420E080
:10CAC000822F0895FC01A48DA80FB92FB11DA35A80
:10CAD000BF4F2C91848D90E001968F739927848F9E
:10CAE000A689B7892C93A089B1898C9183708064C1
:10CAF0008C93938D848D981306C00288F389E02D62
:10CB000080818F7D80830895EF92FF920F931F9312
:10CB1000CF93DF93EC0181E0888F9B8D8C8D9813F0
:10CB20001AC0E889F989808185FF15C09FB7F894FC
:10CB3000EE89FF896083E889F98980818370806448
:10CB400080839FBF81E090E0DF91CF911F910F9193
:10CB5000FF90EF900895F62E0B8D10E00F5F1F4FA2
:10CB60000F731127E02E8C8D8E110CC00FB607FCB1
:10CB7000FACFE889F989808185FFF5CFCE010E943F
:10CB80006265F1CFEB8DEC0FFD2FF11DE35AFF4FE6
:10CB9000F0829FB7F8940B8FEA89FB8980818062CD
:10CBA000CFCFCF93DF93EC01888D8823B9F0AA898A
:10CBB000BB89E889F9898C9185FD03C0808186FD58
:10CBC0000DC00FB607FCF7CF8C9185FFF2CF8081A7
:10CBD00085FFEDCFCE010E946265E9CFDF91CF9155
:10CBE000089580E090E0892B29F00E94586581111A
:10CBF0000E94000080E090E0892B49F080E090E006
:10CC0000892B29F00E94000081110E94000080E021
:10CC100090E0892B49F080E090E0892B29F00E9478
:10CC2000000081110E94000080E090E0892B49F013
:10CC300080E090E0892B29F00E94000081110C9483
:10CC4000000008950F931F93FC016285738584850E
:10CC500095850281138124813581601B710B820BC4
:10CC6000930B0685178520893189601B710B820B18
:10CC7000930B1F910F910895DC01ED91FC910190B0
:10CC8000F081E02D19948FEF9FEF0895FC016289E8
:10CC90007389848995890895EF920F931F93CF9399
:10CCA000DF93FC01248D222341F0213051F1DF91EB
:10CCB000CF911F910F91EF90089522893389448974
:10CCC000558986899789A08DB18D821B930BA40B02
:10CCD000B50B892F9A2FAB2FBB278C010F5F1F4FEE
:10CCE0006281738184819581CFB7F894DCB7E1E0EC
:10CCF000ECBFEE24E394E2E0FEEF1995DCBFCFBF7A
:10CD0000D6CFF0E0E0E0DF91CF911F910F91EF904F
:10CD10001994FC01138E128E41110CC082899389E3
:10CD2000A489B589868B978BA08FB18F148E81E0F3
:10CD300090E0089590E080E00895CF92DF92EF9226
:10CD4000FF92CF93DF93DC01CB01642FCFB7F89430
:10CD50006D01EE24FF24CBBEDCB741E04CBFA9013E
:10CD6000E1E0FEEF1995DCBFCFBFDF91CF91FF90DF
:10CD7000EF90DF90CF900895CF93DF93FC01248D47
:10CD8000211110C0EC01828D938D892B49F06689A9
:10CD90007789808D918D30E020E045E00E949D668E
:10CDA0001B8E1A8EDF91CF9108951F93CF93DF933F
:10CDB000FC01248D211145C0162FEC01828D938D2D
:10CDC000892B49F466897789808D918D30E020E048
:10CDD00043E00E949D664A8D5B8DCA018170992750
:10CDE000FE01E80FF91F158F892B69F02D8D3E8DFF
:10CDF0006E897F89888D998D640F751F811D911DA6
:10CE000041E00E949D668A8D9B8D01969B8F8A8F43
:10CE100081159140B1F46E897F89888D998D30E0BC
:10CE200020E045E00E949D661B8E1A8E8E899F89A8
:10CE3000A88DB98D9F5FAF4FBF4F8E8B9F8BA88FF3
:10CE4000B98F81E090E0DF91CF911F910895DC01CF
:10CE5000ED91FC910280F381E02D40E01994FB01FB
:10CE600024813581428153812417350750F4A081F4
:10CE7000B181A20FB31F8C93848195810196958314
:10CE8000848380E00895CF93DF93EC01E881F981FA
:10CE90000284F385E02DCE0119950196B9F7DF9153
:10CEA000CF910895CF92DF92EF92FF920F931F934D
:10CEB000CF93DF937C016A018B01D0E0C0E0CC15F9
:10CEC000DD0581F0D701ED91FC910284F385E02D21
:10CED000C70119958F3F980729F0F80181938F01B9
:10CEE0002196EDCFCE01DF91CF911F910F91FF9051
:10CEF000EF90DF90CF900895CF93C62FDC01ED9196
:10CF0000FC910088F189E02D1995DC01ED91FC91EF
:10CF10000190F081E02D6C2FCF911994062E000C1A
:10CF2000770BFC01778366830895CF93DF93EC0141
:10CF30008E819F81019611F5E881F9810088F18940
:10CF4000E02DCE011995DC01ED91FC910084F18575
:10CF5000E02D1995892BB1F0E881F9810284F385E0
:10CF6000E02DCE0119958132910534F3E881F981E4
:10CF70000684F785E02D682FCE01199581E0DF91B9
:10CF8000CF91089580E0FBCFCF93DF931F92CDB771
:10CF9000DEB76983DC01ED91FC910280F381E02D25
:10CFA00041E050E0BE016F5F7F4F19950F90DF9118
:10CFB000CF910895EF92FF920F931F93CF93DF933A
:10CFC000EC018B017A010E94438D688B798B8A8BEF
:10CFD0009B8B8C819D81DC01ED91FC910280F38122
:10CFE000E02DA701B801DF91CF911F910F91FF9024
:10CFF000EF9019941F93CF93DF93EC01162F0E94AB
:10D00000438D688B798B8A8B9B8B8C819D81DC0116
:10D01000ED91FC910190F081E02D612FDF91CF9196
:10D020001F911994CF92DF92EF92FF92CF93DF93EB
:10D03000EC018E819F818F3F980759F02FEF3FEFD2
:10D040003F832E83DF91CF91FF90EF90DF90CF90C1
:10D0500008950E94438D6B017C01A4EFCA0EA1E0EC
:10D06000DA1EE11CF11CE881F9810088F189E02DCC
:10D07000CE011995DC01ED91FC910084F185E02D44
:10D080001995892B39F40E94438D6C157D058E0509
:10D090009F0548F3E881F9810088F189E02DCE01F0
:10D0A0001995DC01ED91FC910284F385E02DDF916F
:10D0B000CF91FF90EF90DF90CF9019940E9451BED6
:10D0C0000F931F93CF93DF93EC0188819981009791
:10D0D00059F02A813B812617370730F081E0DF9134
:10D0E000CF911F910F9108958B016F5F7F4F0E9429
:10D0F00070BD009759F0998388831B830A832C8124
:10D100003D81232B59F7FC011082E8CF80E0E7CF67
:10D11000EF92FF920F931F93CF93DF93009751F4F9
:10D12000CFEFDFEFCE01DF91CF911F910F91FF90F5
:10D13000EF900895DC011C96ED90FC90F7010081C2
:10D140001181D801ED91FC910688F789E02DC80185
:10D150001995882329F3D801ED91FC910084F1857C
:10D16000E02DC8011995D801ED91FC91892B61F34F
:10D170000284F385E02DC8011995EC01019681F236
:10D18000F8018789882329F06C2F8FEA98E00E94A4
:10D190007984D70112968C91882321F2C532D1056A
:10D1A00009F6D801ED91FC910084F185E02DC801CC
:10D1B000199502975CF0D801ED91FC910688F789EA
:10D1C000E02DC80119958111ECCFAACFD1E0C0E0C4
:10D1D000D801ED91FC910284F385E02DC8011995E9
:10D1E0008F3F980709F49CCF9C01215431092A31C3
:10D1F000310570F48D2F8295807F829FC00D1124A0
:10D20000D11104C00C2E000CDD0B8CCFD0E0E0CF90
:10D210009C01215631092A31310560F3C0978A30CB
:10D22000910570F79D2F9295907F989FC00D1124C6
:10D23000E7CFCF92DF92EF92FF920F931F93CF939E
:10D24000DF936C018B0186E090E00E940EAEEC0152
:10D250009093F9068093F806F60101900020E9F713
:10D26000CF018C199D090E940EAE7C01B6010E946F
:10D27000DABEF60101900020E9F73197EC19FD09BB
:10D28000EE0DFF1D1082F982E8821B830A838091D4
:10D29000FA069091FB069D838C83D093FB06C09386
:10D2A000FA06DF91CF911F910F91FF90EF90DF90E1
:10D2B000CF900895FC01868197818F3F980729F0D0
:10D2C0002FEF3FEF378326830895808591850C9457
:10D2D0006EB21F93CF93DF93182F66E270E00E9427
:10D2E000031BC82F67E270E0812F0E94031B9C2F55
:10D2F000DF91CF911F910895CF93FC01C08D80E500
:10D3000090E00E94B38760E270E08C2F0E94B687A5
:10D3100062E070E08C2F0E94031B84FD1AC062E063
:10D3200070E08C2F0E94031B83FF0CC048E162E079
:10D3300070E08C2F0E94F91A0E947B1B90E080E025
:10D34000CF9108950E947B1B80E590E00E94B387F7
:10D35000DFCF40E162E070E08C2F0E94F91A0E945A
:10D360007B1B81E090E0ECCFFF920F931F93CF9354
:10D37000DF93EB01FC01178A168A2A81211109C06B
:10D380002B81211106C02C81211103C02D81222364
:10D39000F1F041155105D9F08A01FC01F08C80E5CE
:10D3A00090E00E94B387BE016E5F7F4F8F2D0E9479
:10D3B000321BB8018F2D0E94211B0E947B1B81E034
:10D3C00090E0DF91CF911F910F91FF90089590E031
:10D3D00080E0F7CFAF92BF92CF92DF92FF920F9390
:10D3E0001F93CF93DF938C015B01EA01FC01C68898
:10D3F000D788F08C80E590E00E94B3878F2D0E9443
:10D40000CA888C179D0720F48F2D0E94CA88EC01D2
:10D410009E01A501B6018F2D0E946A880E947B1B88
:10D42000F801868997898C0F9D1F978B868BCE017B
:10D43000DF91CF911F910F91FF90DF90CF90BF9020
:10D44000AF9008957F928F929F92AF92BF92CF92AA
:10D45000DF92EF92FF920F931F93CF93DF93CDB79D
:10D46000DEB7A6970FB6F894DEBF0FBECDBF8C0116
:10D47000762E942E852E20E2A22ECE0101967C01DE
:10D48000DC01EA2D1D92EA95E9F76801F3E4CF0E7D
:10D49000D11C8AE793E09AA389A38FEF8BA38CA377
:10D4A0008DA38EA343E450E0BE016F5D7F4FC601A4
:10D4B0000E94B469019609F4BFC081E089838A8320
:10D4C00086E0B82EBB821C82D80114966D917D91A6
:10D4D0008D919C9117970E9478BA6D837E838F837C
:10D4E000988789869A8680E890E09C878B874CE1B4
:10D4F00050E0B701C6010E94EA69FE0137968AE151
:10D50000DF011D928A95E9F74801B8E08B0E911C66
:10D51000F401D70101900D92BA94E1F740E150E097
:10D52000B701C6010E94EA69F7011192AA94E9F7CE
:10D5300096E0A92EB12C40E250E0B701C6010E944E
:10D54000EA69F1E0AF1AB108B1F783E6898392E89E
:10D550009A8393E59B838C8385E38D8381E08E831F
:10D560007F829DE3988797E099878A8786E0F40118
:10D57000DE011B9601900D928A95E1F78CE0898B74
:10D580008A8B61EF74E0CE0143960E94DABED80127
:10D590001B966C91CE0149960E94E688F80164853D
:10D5A000CE014B960E94E688D8011D966C91CE0163
:10D5B0004D960E94E6884EE150E0B701C6010E94F8
:10D5C000EA69B3E07B121EC082E3898384E08A8328
:10D5D000F80196859B8397859C8390899D8391898B
:10D5E0009E8396E39F838887828D8987838D8A8730
:10D5F000848D8B87858D8C874CE050E0B701C60108
:10D600000E94EA6987E3898386E08A8391E09B83AD
:10D6100093E09C838D838FE08E838AE38F838BE3FB
:10D6200088878FEF898749E050E0B701C6010E94E3
:10D63000EA69C6010E947C69A6960FB6F894DEBF1F
:10D640000FBECDBFDF91CF911F910F91FF90EF9053
:10D65000DF90CF90BF90AF909F908F907F90089574
:10D66000AF92BF92CF92DF92EF92FF920F931F93F0
:10D67000CF93DF93DC01CD90DC901197C114D104DE
:10D6800039F01496CD91DC918C017601209761F4EC
:10D69000DF91CF911F910F91FF90EF90DF90CF908E
:10D6A000BF90AF90089575015701BFEFAB1ABB0A49
:10D6B000F7018081082E000C990B0E941FB1892B65
:10D6C00091F72197CC0DDD1D8881082E000C990B58
:10D6D0000E941FB1892B29F0CE15DF0510F021978C
:10D6E000F3CFAE014F5F5F4F4E195F09D80115961A
:10D6F0005C934E931497CE14DF0420F4B701C60157
:10D700000E948DBED801ED91FC91119714968D91D8
:10D710009C91E80FF91F1082BBCFCF93DF93DC0100
:10D720001496ED91FC916E177F0728F54115510570
:10D7300011F19F01261B370B4217530708F49A017A
:10D74000DB01EC0188819981E21BF30BFD83EC8303
:10D75000AF01461B570B260F371FBC01620F731F0B
:10D760008A0F9B1F0E94FFBEE881F9818C819D81F9
:10D77000E80FF91F1082DF91CF910895DF92EF92A9
:10D78000FF920F931F93CF93DF93FC01E480F5800A
:10D79000E114F10451F48FEF9FEFDF91CF911F91CE
:10D7A0000F91FF90EF90DF900895EC010190F081D0
:10D7B000E02DEE0DFF1DD080108208811981062E0C
:10D7C000000C770BC8010E940EBF0E0D1F1DF80143
:10D7D000D082009701F328813981821B930BDDCF22
:10D7E000FB0144815581FC012481358124173507D3
:10D7F00078F080819181009759F0FB0160817181FF
:10D800006115710529F00E94F1BE21E0892B09F014
:10D8100020E0822F0895FC0124813581232B39F4E7
:10D8200021E0FB018081882349F020E007C080814E
:10D8300091810E94D1BE21E0892BB9F7822F0895F2
:10D84000FC0124813581FB01448155812417350772
:10D85000E1F4FC0180819181FB016081718100977D
:10D86000D1F061157105A1F4232BC1F0FC01808179
:10D8700090E008C0232B91F0FB01808190E091950E
:10D880008195910921E0892B09F020E0822F0895EC
:10D890000E94D1BEF7CF6115710561F721E0F6CF87
:10D8A000EF92FF920F931F93CF93DF936115710552
:10D8B00041F480E0DF91CF911F910F91FF90EF90A5
:10D8C000089541155105B1F07B01EC010C811D81DA
:10D8D000040F151FB8010E946068882351F3288146
:10D8E00039818C819D81B701820F931F0E94DABE1E
:10D8F0001D830C8381E0DECFCF93DF931F921F92B5
:10D90000CDB7DEB769831A8241E050E0BE016F5F98
:10D910007F4F0E94506C0F900F90DF91CF91089530
:10D920000F931F93CF93DF938C01EB01FC01808158
:10D9300091810097E1F06881798161157105A9F005
:10D94000428153812C813D814217530770F00E9420
:10D95000DABE8C819D81F801958384831D821C82AF
:10D96000DF91CF911F910F9108950E94AAAE8881F7
:10D970009981F801918380838A819B81938382833B
:10D980008C819D8195838483198218821B821A82DF
:10D99000E5CFCF93DF93EC0188819981009711F057
:10D9A0000E94AAAE198218821D821C821B821A82D2
:10D9B000DF91CF910895EF92FF920F931F93CF9332
:10D9C000DF9300D01F92CDB7DEB77C01862F4AE0EF
:10D9D0008E010F5F1F4FB80190E00E94B7B1F801B0
:10D9E00001900020E9F73197AF01401B510BB801BE
:10D9F000C7010E94506C811103C0C7010E94C96C0D
:10DA0000C7010F900F900F900F90DF91CF911F9152
:10DA10000F91FF90EF900895CF93DF93EC01611584
:10DA2000710539F4CE010E94C96CCE01DF91CF910E
:10DA30000895FB0101900020E9F73197AF01461BE3
:10DA4000570B0E94506C882369F3EFCFCF93DF937D
:10DA5000EC01FB0144815581608171810E94506C11
:10DA6000811103C0CE010E94C96CCE01DF91CF911C
:10DA70000895EF92FF920F931F93CF93DF93EC01E2
:10DA80007B018A01BA010E94606881110BC0CE013E
:10DA90000E94C96CCE01DF91CF911F910F91FF9031
:10DAA000EF9008951D830C83B701888199810E94AE
:10DAB000DABEF0CFFB0101900020E9F73197AF010A
:10DAC000461B570B0C94396DCF93DF93EC01611516
:10DAD000710531F00E945A6DCE01DF91CF9108950A
:10DAE0000E94C96CF9CFCF93DF93EC01FB0186173D
:10DAF000970749F0608171816115710541F044819A
:10DB000055810E94396DCE01DF91CF9108950E9419
:10DB1000C96CF9CFFC0180819181009711F00C94C0
:10DB2000AAAE0895EF92FF920F931F93CF93DF93C6
:10DB3000EC018B01198218821B821A821D821C82C1
:10DB4000CB010E944BB17C01BC01CE010E946068F8
:10DB5000811109C0CE01DF91CF911F910F91FF90EC
:10DB6000EF900C94C96CFD82EC82B8018881998198
:10DB7000DF91CF911F910F91FF90EF900C9444B1E2
:10DB8000FC011182108213821282158214820C947D
:10DB9000736DFC011182108213821282158214822D
:10DBA000FB0101900020E9F73197AF01461B570BAD
:10DBB0000C94396D0F931F93CF93DF93EC010E9468
:10DBC000438D688779878A879B87E881F9810284FA
:10DBD000F385E02DCE01199597FF15C00E94438D66
:10DBE000088519852A853B85601B710B820B930B79
:10DBF0000C811D812E813F81601771078207930779
:10DC000020F38FEF9FEFDF91CF911F910F91089538
:10DC1000EF92FF920F931F93CF93DF93EC017B0161
:10DC2000042F6AEF74E00E94C96DC7010E94DA6D8B
:10DC3000002E000C110B97FD0BC00817190741F0BF
:10DC4000682FCE010E947C6CC7010E94DA6DF3CF71
:10DC5000CE01DF91CF911F910F91FF90EF9008952A
:10DC6000FB0101900020E9F73197AF01461B570BEC
:10DC7000DC01ED91FC910280F381E02D19948F92EB
:10DC80009F92AF92BF92EF92FF920F931F93CF9309
:10DC9000DF93CDB7DEB7A1970FB6F894DEBF0FBE06
:10DCA000CDBF7C01FA01CB0119A2223008F42AE091
:10DCB0008E010F5D1F4F822E912CB12CA12CBF0124
:10DCC000A50194010E94E5B9F901CA016A300CF579
:10DCD000605DD8016E938D01232B242B252B79F7C2
:10DCE00090E080E0109721F0BD01C7010E94306EE6
:10DCF000A1960FB6F894DEBF0FBECDBFDF91CF91D6
:10DD00001F910F91FF90EF90BF90AF909F908F90D9
:10DD10000895695CDECF68EF74E00C94306EDC012E
:10DD2000ED91FC910190F081E02D1994CF92DF925A
:10DD3000EF92FF920F931F93CF93DF93211531053D
:10DD400081F4DC01ED91FC910190F081E02D642FD4
:10DD5000DF91CF911F910F91FF90EF90DF90CF90C7
:10DD600019942A30310501F52AE077FF1DC06A01B8
:10DD70007B01EC016DE20E948F6E8C0144275527D8
:10DD8000BA014C195D096E097F092AE0CE010E9493
:10DD90003F6E800F911FDF91CF911F910F91FF90E8
:10DDA000EF90DF90CF900895DF91CF911F910F9169
:10DDB000FF90EF90DF90CF900C943F6E8F929F92E8
:10DDC000AF92BF92CF92DF92EF92FF920F931F9389
:10DDD000CF93DF937C018B014C0182E0880E911C74
:10DDE0005701E5E0AE0EB11CD0E0C0E0F401619156
:10DDF0004F01C8010E9479846C016EE2C8010E9443
:10DE00008F6E8C0D9D1DC80FD91F8A149B0471F74E
:10DE1000F7016581C8010E9479848C0F9D1FDF91F5
:10DE2000CF911F910F91FF90EF90DF90CF90BF9017
:10DE3000AF909F908F9008956115710511F00C942B
:10DE4000306E90E080E008950F931F93CF93DF939F
:10DE5000EC018B0161EE74E00E941C6F011511054D
:10DE6000C1F1F80161918F01662399F1603240F0B0
:10DE7000623231F06C3521F0CE010E948F6EF1CF0D
:10DE80006CE5CE010E948F6EF801319780818C3055
:10DE9000D1F044F48930D9F08A30B9F0883009F7EC
:10DEA00062E6EACF823259F024F462E78D3021F342
:10DEB000D8CF8F3231F06CE58C35F1F2D2CF62E2FF
:10DEC000DBCF6FE2D9CF66E6D7CF6EE6D5CF64E77A
:10DED000D3CF62E2CE010E948F6E90E080E0DF91AE
:10DEE000CF911F910F910895DB0114964D915C9194
:10DEF00015976D917C91DC01ED91FC910280F3818D
:10DF0000E02D1994EF92FF920F931F93CF93DF931D
:10DF10008C017B01D0E0C0E0F701EC0FFD1F6491A4
:10DF2000662361F0D801ED91FC910190F081E02D24
:10DF3000C8011995892B11F02196EECFCE01DF9102
:10DF4000CF911F910F91FF90EF9008950F931F9322
:10DF5000CF93DF93EC010E94826F8C01CE010E946F
:10DF60008B6E800F911FDF91CF911F910F910895BC
:10DF7000DC018AE793E08D939D9384E0FB0101909F
:10DF80000D928A95E1F708951F920F920FB60F92A6
:10DF900011240BB60F922F933F934F935F936F9380
:10DFA0007F938F939F93AF93BF93EF93FF938FEAEA
:10DFB00098E00E946265FF91EF91BF91AF919F91B0
:10DFC0008F917F916F915F914F913F912F910F9022
:10DFD0000BBE0F900FBE0F901F9018951F920F92BF
:10DFE0000FB60F9211240BB60F922F938F939F931E
:10DFF000EF93FF93E091BF08F091C0088081E0911A
:10E00000C508F091C60882FD1DC090818091C808A6
:10E010008F5F8F732091C908821741F0E091C80883
:10E02000F0E0E155F74F958F8093C808FF91EF918D
:10E030009F918F912F910F900BBE0F900FBE0F905D
:10E040001F9018958081F2CFDF92EF92FF920F938D
:10E050001F93CF93DF9300D000D0CDB7DEB78B01F5
:10E060007A01D22E6AEF74E0CE0101960E94C96D4A
:10E070009E012F5F3F4F4D2DB701C8010E94709444
:10E08000CE0101960E948A6D26960FB6F894DEBFE7
:10E090000FBECDBFDF91CF911F910F91FF90EF90F9
:10E0A000DF900895CF92DF92EF92FF920F931F932C
:10E0B000CF93DF93CDB7DEB7EC970FB6F894DEBF02
:10E0C0000FBECDBFDC012C91222309F469C06CE99D
:10E0D00073E00E9481B19A8389837E01B3E0EB0EE5
:10E0E000F11C01E010E0D02EC12E6CE973E090E04D
:10E0F00080E00E9481B1F701819391937F010E31FD
:10E10000110521F00F5F1F4F892B69F70091F80669
:10E110001091F906E980FA800115110589F1D801FD
:10E120006D917C91C7010E94D1BE892B29F5D80140
:10E130001296ED91FC91BE016F5F7F4F8D2D9C2D4E
:10E1400019958C018FEA98E00E948B6E64EE74E161
:10E150008FEA98E00E94826FC801EC960FB6F8949F
:10E16000DEBF0FBECDBFDF91CF911F910F91FF900A
:10E17000EF90DF90CF900895F80104811581CCCF06
:10E1800068EE74E18FEA98E00E94A66F8FEA98E04B
:10E190000E948B6E64EE74E18FEA98E00E94826FB9
:10E1A00010E000E0D9CFCF938FEA98E00E944C6551
:10E1B000892BE9F18FEA98E00E942A65C82F8A30FE
:10E1C00089F08D3079F0883001F568E08FEA98E0C9
:10E1D0000E948F6E8091FC06882331F381508093DA
:10E1E000FC06E2CFE091FC06F0E0E454F94F108227
:10E1F00068EF74E08FEA98E00E941C6F8CEB96E069
:10E200000E9452701092FC06CFCF682F8FEA98E0E0
:10E210000E948F6EE091FC06EB3330F681E08E0FAA
:10E220008093FC06F0E0E454F94FC083BDCFCF915A
:10E2300008958F929F92AF92BF92CF92DF92EF920A
:10E24000FF920F931F93CF93DF936115710509F42C
:10E2500096C0DB011896EC911897E295E07FE59562
:10E26000E595E595E595E73008F089C0EC010E2EBF
:10E27000000CFF0B8827E05CFE488F4F0C9470BAAF
:10E280004771587161717871C271D4710D726BEF01
:10E2900074E0CE01DF91CF911F910F91FF90EF902D
:10E2A000DF90CF90BF90AF909F908F900C94306E86
:10E2B00019968C9165E075E0882359F360E075E06C
:10E2C000E8CF19964D915D916D917C911C972AE054
:10E2D00030E0CE01DF91CF911F910F91FF90EF9031
:10E2E000DF90CF90BF90AF909F908F900C94966EE0
:10E2F0001996CD90DD90ED90FC901C9720E030E0D9
:10E30000A901C701B6010E949BB887FF09C061E956
:10E3100073E0CE010E941C6FF7FAF094F7F8F094C6
:10E32000C701B6010E9474BB4B015C01BC01A40192
:10E33000CE010E94768460EB74E0CE010E941C6FD7
:10E34000C501B4010E94A0B89B01AC01C701B60190
:10E350000E948EBA2DEC3CEC4CE45DE30E948FBA37
:10E3600020E030E040E251E40E9401B90E9474BB19
:10E37000AB0170E060E02AE0CE010E943F6E90E0C9
:10E3800080E01DC019966D917C91CE01DF91CF91F7
:10E390001F910F91FF90EF90DF90CF90BF90AF90C3
:10E3A0009F908F900C94246F16960D911C916BE5A5
:10E3B000CE010E948F6E019679F48FEF9FEFDF916F
:10E3C000CF911F910F91FF90EF90DF90CF90BF9072
:10E3D000AF909F908F9008950115110579F0B801C5
:10E3E000CE010E941971019641F3D80112960D9148
:10E3F0001C910115110511F06CE2DACF6DE5CE012B
:10E400000E948F6E21E030E0019611F030E020E0B4
:10E4100088279927821B930BD2CF16960D911C91BA
:10E420006BE7CE010E948F6E019639F2011511053E
:10E4300029F1D8016D917C91CE010E94246F019643
:10E4400009F4BBCF6AE3CE010E948F6E019609F4F6
:10E45000B4CFB801CE010E941971019609F4ADCF75
:10E46000D80112960D911C910115110539F06CE23D
:10E47000CE010E948F6E0196C9F69FCF6DE7BFCF88
:10E48000CF93DF93EC01E881F9810284F385E02DDD
:10E49000CE0119958F3F980769F0E881F9818132A3
:10E4A00091059CF30684F785E02D682FCE01199520
:10E4B00090E080E0DF91CF910895CF92DF92EF92CC
:10E4C000FF920F931F93CF93DF937C016B01DC01CD
:10E4D000ED91FC910284F385E02D1995829761F00E
:10E4E000CFEFDFEFCE01DF91CF911F910F91FF9022
:10E4F000EF90DF90CF900895F6018085807F846053
:10E50000808786E090E00E940EAE8C01009741F378
:10E51000ECE7F6E0DC01ED93FC9380E4DF011D9273
:10E520008A95E9F780E490E0F8019383828315826D
:10E530001482D701ED91FC910284F385E02DC7018F
:10E540001995EC010196C9F0C232D10509F44DC00C
:10E55000C032D1050CF449C0B8018C2FCC35D1059F
:10E5600049F5D701ED91FC910284F385E02DC701B7
:10E570001995EC018F3F980721F4C8010E94AAAEBB
:10E58000B1CF8236910541F15CF48F32910509F1EA
:10E590008C359105D9F0829761F6B80182E20AC004
:10E5A0008E369105E1F04CF4B8018CE0C636D10509
:10E5B00009F0BFCF0E942F67BCCF8237910591F041
:10E5C000B80189E0C437D105A9F3B3CFB8018CE510
:10E5D000F1CFB8018FE2EECFB80188E0EBCFB80100
:10E5E0008AE0E8CFB8018DE0E5CFF801848195811C
:10E5F000009749F00190F081E02DE80FF91F319765
:10E600008081882321F0B80180E00E942F67D80123
:10E6100014968D919C910E940EAEEC01009739F0FA
:10E620006CE776E00E94DABEC8010E94AAAEF6014D
:10E63000D287C187D0E0C0E055CF8DE090E00E9446
:10E640000EAE009729F02DE0FC0111922A95E9F712
:10E6500008950F931F93CF93DF930097E1F0EC01A0
:10E660000C851D850115110579F0D8018D919C91BE
:10E67000009739F0DC01ED91FC910488F589E02DDB
:10E680001995C8010E94AAAECE01DF91CF911F91CA
:10E690000F910C94F9B1DF91CF911F910F910895D3
:10E6A000AF92BF92CF92DF92EF92FF920F931F93A0
:10E6B000CF93DF9300D01F92CDB7DEB76115710500
:10E6C000B1F06B01182FDB011C96AD90BC90F501E9
:10E6D000E080F180D701ED91FC910688F789E02D6B
:10E6E000C7011995811106C0C6010E9429738FEFD9
:10E6F0009FEF13C0F5019281911124C0D701ED91D4
:10E70000FC910190F081E02D612FC7011995F7016F
:10E710008789811111C090E080E00F900F900F90D9
:10E720000F90DF91CF911F910F91FF90EF90DF90AD
:10E73000CF90BF90AF900895612F8FEA98E00E942C
:10E740008F6EE9CF812F8F7D81548A31B8F280EDB1
:10E75000810F8A3098F283ED810F823078F21F3575
:10E7600069F21E3759F21132B1F086EC810F823016
:10E7700090F08AED810F873070F01D3361F0812FAA
:10E780008F7E8F3241F08DED810F823020F01B356E
:10E7900011F01D3511F491FFB1CF19821A821B823D
:10E7A0001C82812F012E000C990B9F931F938BE0ED
:10E7B00095E09F938F938E010F5F1F4F1F930F93D1
:10E7C0000E9456BF6E01F4E0CF0ED11C0F900F9047
:10E7D0000F900F900F900F90D8016D918D01D70180
:10E7E000ED91FC910190F081E02DC7011995F701A1
:10E7F0008789882339F0F801319760818FEA98E0A2
:10E800000E948F6E0C151D0539F785CF2C9A08953F
:10E810002C9808951F93CF93DF93182F60E270E038
:10E820000E94031BC82F61E270E0812F0E94031B2E
:10E830009C2FDF91CF911F9108958EBD00000DB4E4
:10E8400007FEFDCF8EB50895CF92DF92EF92FF9233
:10E850000F931F93CF93DF93EC017A018B016C012F
:10E86000C40ED51ECC15DD05A9F00E9408748FE0FA
:10E870000E941D748D2F0E941D748C2F0E941D7488
:10E88000219680E00E941D74F80181938F010E94FF
:10E890000674E8CFC701DF91CF911F910F91FF90D0
:10E8A000EF90DF90CF900895CF92DF92EF92FF929A
:10E8B0000F931F93CF93DF93EC017A018B016C01CF
:10E8C000C40ED51ECC15DD05A1F00E94087480EFA2
:10E8D0000E941D748D2F0E941D748C2F0E941D7428
:10E8E0002196F80181918F010E941D740E94067487
:10E8F000E9CFC701DF91CF911F910F91FF90EF906A
:10E90000DF90CF9008951F93CF93DF93D82F192FC7
:10E91000C62F0E94087480EF0E941D74812F0E94F0
:10E920001D748D2F0E941D748C2F0E941D740E94D7
:10E93000067481E0DF91CF911F910895EF92FF92CD
:10E940000F931F93CF93C82F7B0180E590E00E9427
:10E95000B38768E270E08C2F0E94031B082F69E2E6
:10E9600070E08C2F0E94031B282F302FB90121E06B
:10E9700030E0A7018C2F0E9422880E947B1B81E03F
:10E9800090E0CF911F910F91FF90EF900895CF935A
:10E99000DF931F92CDB7DEB7FC01218D328D8FEF53
:10E9A0009FEF232B41F0BE016F5F7F4F808D0E9450
:10E9B0009E74898190E00F90DF91CF910895FF922E
:10E9C0000F931F93CF93DF93F82E80E590E00E9482
:10E9D000B38710E000E08F2D0E946969EC01892B5C
:10E9E00021F08F2D0E9469698C01C017D10799F71A
:10E9F0000E947B1BCE01DF91CF911F910F91FF9061
:10EA00000895AF92BF92CF92DF92EF92FF921F9341
:10EA1000CF93DF93182F6B017A0180E590E00E947D
:10EA2000B387B12CA12C812F0E946969EC01892B3D
:10EA300021F0812F0E9469695C01CA15DB0599F7F5
:10EA40002097F9F463E070E0812F0E94031B84316A
:10EA500059F0882349F0C1E0D0E08C3111F4D0E0C6
:10EA6000C0E0D195C195D1090E947B1BCE01DF91F9
:10EA7000CF911F91FF90EF90DF90CF90BF90AF901C
:10EA80000895EC16FD060CF4E7011C161D0664F74C
:10EA900068E270E0812F0E94031BE82E69E270E0BB
:10EAA000812F0E94031B282F3E2D79019E01A60174
:10EAB000B701812F0E942288EC0EFD1E4F2D68E2C7
:10EAC00070E0812F0E94F91A4E2D69E270E0812FCB
:10EAD0000E94F91A60E470E0812F0E94B687C4CFCB
:10EAE000CF93DF93FC01218D328D2115310529F45F
:10EAF0008FEF9FEFDF91CF910895EC01808D42174A
:10EB0000530708F0A9010E9401751816190684F729
:10EB1000298D3A8D281B390B3A8F298FEBCF0F9314
:10EB20001F93CF93DF931F92CDB7DEB7FC01218DEA
:10EB3000328D232B41F48FEF9FEF0F90DF91CF9118
:10EB40001F910F9108958C0141E050E0BE016F5F6D
:10EB50007F4FFC01808D0E940175181619065CF725
:10EB6000F801818D928D0197928F818F898190E03C
:10EB7000E4CF0F931F93CF93DF9300D000D01F9269
:10EB80001F92CDB7DEB78C01D80159968D919C911B
:10EB90005A97892B41F0ED91FC910284F385E02D89
:10EBA000C8011995F1CFF801808D0E94DF74181605
:10EBB0001906B4F548E050E0BE016F5F7F4FD80101
:10EBC00058968C910E94017518161906F4F4D80114
:10EBD000509684E0FE01319601900D928A95E1F7FE
:10EBE0008D8190E0982F88272E81820F911DF8014A
:10EBF000958B848B8F81282F30E0322F22278885B8
:10EC0000820F932F911D928F818F28960FB6F894C3
:10EC1000DEBF0FBECDBFDF91CF911F910F91089541
:10EC200090E080E0F2CF4F925F926F927F928F924E
:10EC30009F92AF92BF92CF92DF92EF92FF920F938B
:10EC40001F93CF93DF93CDB7DEB763970FB6F894DA
:10EC5000DEBF0FBECDBF7C016B013A01FB0120E09E
:10EC600090E080E06AE03191332309F461C040ED27
:10EC7000430F4A3008F04DC0689FA001699F500DB6
:10EC80001124CA01C097830F911D37FD9A958F3FBC
:10EC9000910549F340F3F701428153816481758105
:10ECA0008091030890910408A0910508B09106088E
:10ECB000481759076A077B0709F42EC28701085FC6
:10ECC0001F4F0E94438D6F7077277C5FC8010E94A1
:10ECD0008513813009F025C28AE793E09A838983FE
:10ECE000F70182819381A481B5818B839C83AD835D
:10ECF000BE8345E350E0BE016F5F7F4FC8010E94B5
:10ED0000B469892BA9F5D12CC12CC8010E947013BC
:10ED100017C03E3209F0BFCF233009F4BCCFD30176
:10ED2000A20FB11D12968C932F5F90E080E09BCFD5
:10ED3000233009F0B0CFF3018583CC24C394D12CC8
:10ED4000C60163960FB6F894DEBF0FBECDBFDF914C
:10ED5000CF911F910F91FF90EF90DF90CF90BF90D8
:10ED6000AF909F908F907F906F905F904F9008959D
:10ED70000E94438DF701778366837627672776277E
:10ED80007A83698342E050E0BE016F5F7F4FC80124
:10ED90000E94EA6981E090E09E878D8742E050E022
:10EDA000BE01635F7F4FC8010E94EA6980E091E085
:10EDB0009E878D8742E050E0BE01635F7F4FC801B0
:10EDC0000E94EA691E861D8642E050E0BE01635F34
:10EDD0007F4FC8010E94EA6942E050E0BE01635FD4
:10EDE0007F4FC8010E94EA6942E050E0BE01635FC4
:10EDF0007F4FC8010E94EA695601F601808188238D
:10EE000001F16501F60181912F01882311F08E3205
:10EE1000B1F446018A189B081814190474F48F86FB
:10EE200041E050E0BE01615F7F4FC8010E94EA6986
:10EE3000A401B501C8010E94EA695201DECF620156
:10EE4000E1CF1F8641E050E0BE01615F7F4FC80106
:10EE50000E94EA69C12CDD24D394DE86CD8642E08F
:10EE600050E0BE01635F7F4FC8010E94EA69DE8601
:10EE7000CD8642E050E0BE01635F7F4FC8010E9433
:10EE8000EA69C8010E947C69892B09F43CCFF3E050
:10EE9000AF2EB12C230122E0420E511CEEC0F7012F
:10EEA0004281538164817581808D918DA28DB38D56
:10EEB000481759076A077B0709F024C1848D958D8F
:10EEC000C59709F01FC181A192A15DEFC52EDD2478
:10EED000DA940C970CF4C5C04CE050E0BE016F5FB3
:10EEE0007F4FC8010E9470758B819C81982789276C
:10EEF00098279A8B898B29813A81322723273227B9
:10EF0000F701468157814217530709F000C197FF67
:10EF1000FEC08F7092703BEFC32EDD24DA94892BF4
:10EF200009F09FC06F8078847624672476242AEFC6
:10EF3000C22EDD24DA946114710409F492C0D12C3C
:10EF4000C12C8D819E81982789279827C816D906BC
:10EF500040F541E050E0BE01635F7F4FC8010E9471
:10EF600070758D85882351F08D859FEF980F9D8753
:10EF7000882321F0C8010E948F75F6CF8D858111FD
:10EF8000E8CFC8010E948F75C8010E948F75C80123
:10EF90000E948F75C8010E948F75FFEFCF1ADF0A9C
:10EFA000D0CF912C812C41E050E0BE016D5E7F4FAF
:10EFB000C8010E9470758B89982F907C61F488231A
:10EFC00089F08B899FEF980F9B8B882341F0C801B4
:10EFD0000E948F75F6CFC8010E948F751B8A8B899E
:10EFE0008111E1CF42E050E0BE01615F7F4FC80177
:10EFF0000E94707542E050E0BE01635F7F4FC80120
:10F000000E947075C8010E948F75C8010E948F759B
:10F01000C8010E948F75C8010E948F7542E050E0C0
:10F02000BE016F5E7F4FC8010E9470758F85988901
:10F030008115914009F040C0CD84DE84DC24CD24CC
:10F04000DC2481E0C816D104B9F589899A89811533
:10F05000944009F04EC044E050E0B201C8010E9463
:10F0600070750E940F5481E0A81AB10809F44DCEC2
:10F07000FFEFCF16DF0609F048CE0E94438D3B011B
:10F080004C01C8010E94B975181619060CF407CF77
:10F090000E94438D6619770988099909613A7F4072
:10F0A0008105910558F50E940F5461E070E080E001
:10F0B00090E00E94FE8AE5CFD12CC12C89899A89E3
:10F0C000982789279827C816D90638F4C8010E94BE
:10F0D0008F75FFEFCF1ADF0AF1CF2FEF821A920A56
:10F0E0006814790409F05FCF96EFC92EDD24DA9415
:10F0F000B8CFE7EFCE2EDD24DA94B3CFCC24CA9478
:10F10000DC2CAFCF6EEFC62EDD24DA94AACF4CEF05
:10F11000C42EDD24DA94A5CF8EEFC82EDD24DA9438
:10F120000FCED12CC12C0CCE2F923F924F925F92DA
:10F130006F927F928F929F92AF92BF92DF92EF92E7
:10F14000FF920F931F93CF93DF93CDB7DEB7E49772
:10F150000FB6F894DEBF0FBECDBF7C014A015B0144
:10F1600019010E94438D2B013C0187010D5B1F4F4C
:10F17000C8010E94B975181619069CF00E94438DAB
:10F18000641975098609970986169706A806B906AF
:10F1900008F488C162E370E080E090E00E94FE8A9B
:10F1A000E7CF42E250E0BE016F5F7F4FC8010E948F
:10F1B000707589818230D1F0D12C8D2DE4960FB6F7
:10F1C000F894DEBF0FBECDBFDF91CF911F910F919D
:10F1D000FF90EF90DF90BF90AF909F908F907F90C7
:10F1E0006F905F904F903F902F900895F801848921
:10F1F00095898334910501F76D817E818F81988592
:10F200000E9478BA2B013C01F10140825182628256
:10F21000738246E050E0B701685F7F4FCE014D96A4
:10F220000E9480BE892B41F6F70180819181A281E5
:10F23000B381481659066A067B0608F4BDCF84815F
:10F240009581A681B78184159505A605B70508F4B3
:10F25000B3CF89899A89AB89BC8986879787A08B28
:10F26000B18B8EECA82EB12CC8010E948F75F1E0F5
:10F27000AF1AB108C9F7D12CC70182969AA789A7FE
:10F28000F701B696FCA7EBA708969EA78DA73C971B
:10F290004F01899698AB8FA73897FAABE9AB170166
:10F2A000F6E12F0E311CC5979CAB8BABF801818D1D
:10F2B000928D181619060CF080CFC8010E948F7528
:10F2C0008333910509F4D4C0A4F58130910509F484
:10F2D00074C074F4892B51F3C8010E948F75B82E45
:10F2E000BA94FFEFBF1611F3C8010E948F75F8CFD3
:10F2F0008330910509F46CC0069771F7C8010E942C
:10F300008F75A82E44E050E06BA97CA9C8010E942B
:10F310007075712C612CEA2DE450FF0B5F016A14AB
:10F320007B0424F6C8010E948F75FFEF6F1A7F0AD5
:10F33000F6CF8A33910509F46FC074F585339105D2
:10F34000A1F1C69749F6C8010E948F75B82EF70142
:10F35000828D811109C0838D811106C0848D811138
:10F3600003C0858D8823A1F0EFA5F8A940805180C6
:10F3700062807380B401CE0183960E94B86F8DA124
:10F380009EA1AFA1B8A584159505A605B705D9F529
:10F3900044E050E0B40118C08B33910509F452C029
:10F3A0008F3F910509F482CF97CFC8010E948F75D6
:10F3B000C8010E948F75D82E79CFC8010E948F7521
:10F3C00044E050E069A97AA9C8010E9470756ECF27
:10F3D000C8010E948F75A82E44E050E0B101C80119
:10F3E0000E947075712C612C8A2D8450990B5C01E0
:10F3F0006A147B040CF05ACFC8010E948F759FEFEE
:10F40000691A790AF5CFBA94FFEFBF1609F44ECF07
:10F41000C8010E948F75F7CFC8010E948F7544E024
:10F4200050E06BA57CA5C8010E947075F70166A12C
:10F4300077A180A591A50E9478BA66A377A380A73B
:10F4400091A734CFC8010E948F7544E050E06DA5AC
:10F450007EA5C8010E947075F70162A573A584A5F9
:10F4600095A50E9478BA62A773A784A795A71ECF17
:10F47000C8010E948F7544E050E069A57AA5C801D3
:10F480000E947075F70162A173A184A195A10E94E9
:10F4900078BA62A373A384A395A366A777A780AB6A
:10F4A00091AB04CFDD24DA9488CE2F923F924F9215
:10F4B0005F926F927F928F929F92AF92BF92CF9204
:10F4C000DF92EF92FF920F931F93CF93DF9300D0C1
:10F4D00000D0CDB7DEB78C010E947FAF2FEC37E0B4
:10F4E00040E050E00E9407BADC01CB010196A11D6B
:10F4F000B11DF80184839583A683B78380839183AC
:10F50000A283B3835801F3E4AF0EB11CC5010E947E
:10F51000701364E470E0C5010E948513882309F428
:10F5200045C10E94438D2B013C01480182E4880EB5
:10F53000911C48EEC42E43E0D42EE12CF12C52E075
:10F54000252E1E821D82D4018C918330B1F1811150
:10F5500066C0F80184819581A681B7810196A11DBD
:10F56000B11D84839583A683B7830E94438D64195C
:10F57000750986099709A70196010E94E5B9A901B5
:10F5800061E0C8010E94226A81E0D4018C938D81E0
:10F590009E810197C1F20E94438D64197509860905
:10F5A0009709D801D6962D913D914D915C91D997AF
:10F5B000261737074807590720F6C5010E94701320
:10F5C000F80184819581A681B7810196A11DB11DA5
:10F5D00084839583A683B7830E94438DF801FE96AA
:10F5E00060837183828393838D819E8126960FB67B
:10F5F000F894DEBF0FBECDBFDF91CF911F910F9169
:10F60000FF90EF90DF90CF90BF90AF909F908F9042
:10F610007F906F905F904F903F902F90089584302F
:10F62000F1F4F80184819581A681B7810196A11D2D
:10F63000B11D84839583A683B7830E94438D64198B
:10F64000750986099709A70196010E94E5B9A901E4
:10F6500063E0C8010E94226AD4012C9298CF8130C5
:10F6600051F5F80142AD53AD64AD75AD9E012F5F0C
:10F670003F4FC8010E949478382EF2E08F1390C05B
:10F6800089819A81AB81BC81F80184839583A683AB
:10F69000B7830E94438D6419750986099709A701EC
:10F6A00096010E94E5B9A90163E0C8010E94226A9F
:10F6B000D4013C926CCF823009F069CFF80142ADA1
:10F6C00053AD64AD75AD9E012F5F3F4FC8010E94E1
:10F6D0009478382EF5E08F135DC0E3E0D401EC930D
:10F6E000F80182A193A1A4A1B5A1892B8A2B8B2B10
:10F6F00041F484E893E0A0E0B0E082A393A3A4A344
:10F70000B5A3F80186A197A1A0A5B1A5892B8A2B45
:10F710008B2B61F482A193A1A4A1B5A1B695A79565
:10F720009795879586A397A3A0A7B1A7F80182A56F
:10F7300093A5A4A5B5A5892B8A2B8B2BA9F482A10F
:10F7400093A1A4A1B5A1AC01BD0123E07695679575
:10F75000579547952A95D1F7841B950BA60BB70BA8
:10F7600082A793A7A4A7B5A7F80186A197A1A0A5F2
:10F77000B1A586A797A7A0ABB1AB82A593A5A4A579
:10F78000B5A582AB93ABA4ABB5AB81E090E09E8313
:10F790008D83FDCE96E0891303C0D4011C92F7CE71
:10F7A000BFEF3B12F4CEF4011082F1CE1E821D8217
:10F7B0001BCFCF93C82F80E590E00E94B38760E114
:10F7C00070E08C2F0E94B6874FEF62E070E08C2FC4
:10F7D0000E94F91ACF910C947B1BFF920F931F93F9
:10F7E000CF93DF93C82FD62F8A01F22E0E94D97BA8
:10F7F00080E590E00E94B3874D2F4F2970E060E0D4
:10F800008C2F0E94F91A01151105D1F0412F64E0E7
:10F8100070E08C2F0E94F91A402F65E070E08C2F69
:10F820000E94F91A61E070E08C2F0E94B6870E9456
:10F830007B1B81E0DF91CF911F910F91FF90089585
:10F8400000917A0610917B060F5F1F4F10937B0685
:10F8500000937A06DBCFBF92CF92DF92EF92FF92B6
:10F860000F931F93CF93DF9300D000D0CDB7DEB7B7
:10F87000FC01208D243009F05DC06A017B018C0100
:10F88000B12C63E070E08B2D0E94031B81114AC0F4
:10F89000F801B08EF801808D843009F44BC096E0F9
:10F8A000EAE7F2E0DE01119601900D929A95E1F7F8
:10F8B000F70193819F779C8394819D8395819E839B
:10F8C000B7016E5F7F4F0E94321BB601F801808D39
:10F8D0000E94211BF801808D90E0982F882746E038
:10F8E00050E0BE016F5F7F4F8A5F9B4F0E94547450
:10F8F000F801128E118E20E8A60162E0808D0E9430
:10F90000ED7B81E026960FB6F894DEBF0FBECDBF2B
:10F91000DF91CF911F910F91FF90EF90DF90CF90EB
:10F92000BF900895883109F4B3CFB394F4E0BF12C7
:10F93000A8CFB0CF80E0E6CFCF93C82F80E590E08E
:10F940000E94B38763E070E08C2F0E94031BC82FD6
:10F950000E947B1B8C2FCF9108958F709927823046
:10F96000910518F0029761F00895809155089091E3
:10F970005608DC01ED91FC910680F781E02D199489
:10F980008091570890915808DC01ED91FC91008C12
:10F99000F18DE02D19958091570890915808DC0160
:10F9A000ED91FC910488F589E02DE9CF8F929F922B
:10F9B000AF92BF92CF92DF92EF92FF92CF93DF93FD
:10F9C000EC014A015B01C12CD12C7601CE010E94D1
:10F9D000431B882399F0C814D904EA04FB0474F487
:10F9E000CE010E94F313892B89F38FEFC81AD80A2E
:10F9F000E80AF80ACE010E94D913E8CFDF91CF912F
:10FA0000FF90EF90DF90CF90BF90AF909F908F903E
:10FA100008952F923F924F925F926F927F928F92B2
:10FA20009F92AF92BF92CF92DF92EF92FF920F938D
:10FA30001F93CF93DF9300D000D01F921F92CDB7BA
:10FA4000DEB78C016B010E944072019619F48FEFB2
:10FA50009FEF1DC0D801ED91FC910284F385E02D4C
:10FA6000C80119957C018F3F980789F3D801ED9162
:10FA7000FC910684F785E02D682FC8011995B2E244
:10FA8000EB16F104E9F4B601C8010E945D722896F4
:10FA90000FB6F894DEBF0FBECDBFDF91CF911F919F
:10FAA0000F91FF90EF90DF90CF90BF90AF909F901D
:10FAB0008F907F906F905F904F903F902F90089520
:10FAC000EDE2EE16F10429F0C701C0970A9708F09D
:10FAD00043C1D801ED91FC910284F385E02DC8016A
:10FAE00019957C018F3F980709F4B1CF8D9799F54F
:10FAF000D801ED91FC910284F385E02DC8011995A0
:10FB00007C01019609F4A3CFEFEFFFEFF887EF83B5
:10FB1000C701C097812C912C54010A9708F5AAE0DF
:10FB2000B0E0A50194010E9426BA30E3E31AF1087F
:10FB30004701FF0CAA08BB08860E971EA81EB91E17
:10FB4000D801ED91FC910284F385E02DC80119954F
:10FB50007C01C097E2CF21E030E038872F83D8CFF7
:10FB6000BEE2EB16F10401F1C7018F7D85349105EA
:10FB7000D9F0AF81B885A50194010E9431BAF60190
:10FB800061877287838794878085807F8260808782
:10FB9000D801ED91FC910684F785E02D6E2DC8010A
:10FBA000199590E080E073CFC501B4010E94A2B81E
:10FBB0002B013C01312C212CFEE2EF16F10499F5CA
:10FBC000D801ED91FC910284F385E02DC8011995CF
:10FBD0007C01312C212C20E030E040E251E4C301D3
:10FBE000B2010E9401B94B015C01B7016053710978
:10FBF000072E000C880B990B0E94A2B8A501940156
:10FC00000E948FBA2B013C01B1E02B1A3108D801B8
:10FC1000ED91FC910284F385E02DC80119957C01DA
:10FC2000C0970A97C0F2C7018F7D8534910509F00E
:10FC300040C0D801ED91FC910284F385E02DC8010C
:10FC400019957C01D801ED91FC918B32910519F544
:10FC50000284F385E02DC80119957C01E1E0EE8373
:10FC6000B12CA12C8AE0982ED801ED91FC91C7010E
:10FC7000C0978A30910508F59A9C90019B9C300DA5
:10FC800011245C01A20EB31E0284F385E02DC8018D
:10FC900019957C01E9CF8D9749F40284F385E02D15
:10FCA000C80119957C013FEF3E83DACF81E08E8356
:10FCB000D7CFB1E0BE83B12CA12CEF81F885BF0175
:10FCC000FF0F880B990B0E94A2B8A30192010E941A
:10FCD00001B92B013C01B501BB0C880B990B0E94AB
:10FCE000A2B84B015C01FE816F2FFF0F770B880BD1
:10FCF000990B0E94A2B89B01AC01C501B4010E94FE
:10FD000001B94B015C01B101330C880B990B0E94C6
:10FD1000A2B89B01AC01C501B4010E948FBA9B013E
:10FD2000AC0160E070E080E291E40E94A8BB9B011E
:10FD3000AC01C301B2010E9401B9D60119966D93BD
:10FD40007D938D939C931C9718968C911897807F28
:10FD5000836018968C931CCFBBE5EB16F10409F079
:10FD600062C0D801ED91FC910284F385E02DC801B9
:10FD700019958B35910509F06ACEF6018085807F53
:10FD800085608087C8010E944072D801ED91FC9186
:10FD90000284F385E02DC80119958D35910509F48C
:10FDA00000CFD801ED91FC910684F785E02D682FF6
:10FDB000C8011995BB24BA940E941D737C01009759
:10FDC00009F445CEBB2031F1F60197838683C80143
:10FDD0000E944072B701C8010E94097D892B09F079
:10FDE00036CEC8010E944072D801ED91FC91028488
:10FDF000F385E02DC8011995B12C47018C3291058E
:10FE0000D9F221E030E08D35910509F08DC030E068
:10FE100020E08AC0D40113969C938E931297FC0124
:10FE200095828482D4CFBBE7EB16F10409F08AC037
:10FE3000D801ED91FC910284F385E02DC80119955C
:10FE40008B37910509F003CEF6018085807F8660AF
:10FE50008087C8010E944072D801ED91FC91028414
:10FE6000F385E02DC80119958D37910509F499CED8
:10FE7000D801ED91FC910684F785E02D682FC8012B
:10FE8000199599249A940E941D737C01009709F496
:10FE9000DECD992009F44DC0F60197838683C80111
:10FEA0000E944072B701C8010E945D72019609F478
:10FEB000CECDC8010E944072D70119968D919C91B8
:10FEC0001A9711969C938E931A961C921E921997CC
:10FED000D801ED91FC910284F385E02DC8011995BC
:10FEE000CA9709F0B4CDC8010E944072B701C80199
:10FEF0000E94097D019609F4AACDC8010E944072B2
:10FF0000D801ED91FC910284F385E02DC80119958B
:10FF1000912C57018C32910509F4B5CF21E030E0E6
:10FF20008D37910509F473CF88279927821B930B8E
:10FF3000AECDD50113969C938E931297FC01B5829A
:10FF4000A482ADCFBEE6EB16F10421F519821A8228
:10FF50001B821C82D801ED91FC910484F585E02D73
:10FF600044E050E0BE016F5F7F4FC80119950497D0
:10FF700009F06DCD44E050E06BEF74E0CE010196E6
:10FF80000E94F1BE009709F062CDF6012085207F26
:10FF900020877DCDF6E6EF16F10441F59E012F5F37
:10FFA0003F4F790185E0D9011D928A95E9F7D80183
:10FFB000ED91FC910484F585E02D45E050E0B90118
:10FFC000C8011995059709F042CD45E050E065E07C
:10FFD00075E0C7010E94F1BE009709F038CDF60127
:10FFE0002085207F21602087118651CDF4E7EF1610
:10FFF000F10409F02CCD19821A821B821C82D801CF
:020000021000EC
:10000000ED91FC910484F585E02D44E050E0BE01C3
:100010006F5F7F4FC8011995049709F018CD44E030
:1000200050E060E075E0CE0101960E94F1BE0097BD
:1000300009F00DCDF6012085207F2160208721E089
:10004000218725CDEF92FF920F931F93CF93DF93DC
:100050007C018B01D0E0C0E0C7010E94DA6D97FD02
:1000600007C0F80181938F012196C430D105A1F713
:10007000CE01DF91CF911F910F91FF90EF900895E6
:100080000F931F93CF93DF93CDB7DEB762970FB671
:10009000F894DEBF0FBECDBF8C01CB01F8011182F9
:1000A0001082138212821582148240E1BE016F5FBA
:1000B0007F4F0E94B7B1BE016F5F7F4FC8010E94A2
:1000C0005A6D62960FB6F894DEBF0FBECDBFDF91BA
:1000D000CF911F910F910895CF93DF93A09178084E
:1000E000B0917908109709F444C052961C921E9260
:1000F000519754961C921E92539784E890E01D9657
:100100009C938E931C971E961C921E9780E090E302
:1001100050969C938E931F97ED91FC9111970088B8
:10012000F189E02D70E060E0CD011995C3E9D2E0DE
:100130008091780890917908DC01ED91FC91B2E012
:10014000C739DB07C1F00284F385E02D19952991A9
:10015000022E000C330B8217930751F3809178081D
:1001600090917908DC01ED91FC910488F589E02DEE
:10017000199580E005C00488F589E02D199581E086
:10018000DF91CF910895AF92BF92CF92DF92EF921D
:10019000FF920F931F93CF93DF935C017B018B0141
:1001A000040F151FEB016E01CE18DF08C017D10731
:1001B00041F0C5010E94DA6D1816190614F48993EE
:1001C000F2CFC601DF91CF911F910F91FF90EF9079
:1001D000DF90CF90BF90AF900895CF93DF932091A1
:1001E000780830917908232B11F480E056C0EC0197
:1001F0000E946C808823C9F3FE0101900020E9F77A
:100200003197EC1BFD0B709780F7A0917808B091A7
:10021000790852961C921E92519754961C921E92E7
:10022000539784E890E01D969C938E931C971E969E
:100230001C921E9780E090E350969C938E931F979C
:10024000ED91FC9111970088F189E02D60E470E058
:10025000CD011995BE0180917808909179080E948E
:100260001C6F8091780890917908DC01ED91FC91E8
:100270000190F081E02D60E01995EC018091780803
:1002800090917908DC01ED91FC910488F589E02DCD
:10029000199581E0CD2B09F4A8CFDF91CF91089576
:1002A000CF93DF932091780830917908232B11F4B4
:1002B00080E056C0EC010E946C808823C9F3FE01E7
:1002C00001900020E9F73197EC1BFD0B709780F748
:1002D000A0917808B091790852961C921E9251977D
:1002E00054961C921E92539784E890E01D969C931E
:1002F0008E931C971E961C921E9780E090E350965A
:100300009C938E931F97ED91FC9111970088F18932
:10031000E02D60E570E0CD011995BE01809178086F
:10032000909179080E941C6F8091780890917908CB
:10033000DC01ED91FC910190F081E02D60E01995D8
:10034000EC018091780890917908DC01ED91FC91A5
:100350000488F589E02D199581E0CD2B09F4A8CF0B
:10036000DF91CF9108950F931F93CF93DF9300D028
:100370001F92CDB7DEB7FC0182819381A481B58144
:1003800089839A83AB83BC838091780890917908A4
:10039000892B11F480E049C00E946C808823D1F33E
:1003A000A0917808B091790852961C921E925197AC
:1003B00054961C921E92539784E890E01D969C934D
:1003C0008E931C971E961C921E9780E090E3509689
:1003D0009C938E931F97ED91FC9111970088F18962
:1003E000E02D60E170E0CD01199580917808909141
:1003F0007908DC01ED91FC910280F381E02D44E06D
:1004000050E0BE016F5F7F4F19958C018091780895
:1004100090917908DC01ED91FC910488F589E02D3B
:10042000199581E0012B09F4B5CF0F900F900F9033
:100430000F90DF91CF911F910F9108950F931F930C
:10044000CF93DF9300D01F92CDB7DEB7FC0182813E
:100450009381A481B58189839A83AB83BC83809186
:10046000780890917908892B11F480E049C00E94A6
:100470006C808823D1F3A0917808B09179085296C6
:100480001C921E92519754961C921E92539784E888
:1004900090E01D969C938E931C971E961C921E971F
:1004A00080E090E350969C938E931F97ED91FC9182
:1004B00011970088F189E02D6CE170E0CD0119956C
:1004C0008091780890917908DC01ED91FC9102808F
:1004D000F381E02D44E050E0BE016F5F7F4F19953E
:1004E0008C018091780890917908DC01ED91FC9164
:1004F0000488F589E02D199581E0012B09F4B5CF29
:100500000F900F900F900F90DF91CF911F910F914F
:1005100008950F931F93CF93DF9300D01F92CDB711
:10052000DEB7FC0182819381A481B58189839A839E
:10053000AB83BC838091780890917908892B11F462
:1005400080E049C00E946C808823D1F3A091780894
:10055000B091790852961C921E92519754961C9213
:100560001E92539784E890E01D969C938E931C975F
:100570001E961C921E9780E090E350969C938E935B
:100580001F97ED91FC9111970088F189E02D64E1AE
:1005900070E0CD0119958091780890917908DC017F
:1005A000ED91FC910280F381E02D44E050E0BE012A
:1005B0006F5F7F4F19958C01809178089091790831
:1005C000DC01ED91FC910488F589E02D199581E01D
:1005D000012B09F4B5CF0F900F900F900F90DF9182
:1005E000CF911F910F9108950F931F93CF93DF9396
:1005F00000D01F92CDB7DEB7FC0182819381A48128
:10060000B58189839A83AB83BC838091780890916C
:100610007908892B11F480E049C00E946C808823FE
:10062000D1F3A0917808B091790852961C921E924D
:10063000519754961C921E92539784E890E01D9611
:100640009C938E931C971E961C921E9780E090E3BD
:1006500050969C938E931F97ED91FC911197008873
:10066000F189E02D68E170E0CD011995809178085D
:1006700090917908DC01ED91FC910280F381E02DED
:1006800044E050E0BE016F5F7F4F19958C0180916F
:10069000780890917908DC01ED91FC910488F58946
:1006A000E02D199581E0012B09F4B5CF0F900F9043
:1006B0000F900F90DF91CF911F910F910895CF93DD
:1006C000DF9300D01F92CDB7DEB719821A821B824A
:1006D0001C8287E789838091780890917908892B1B
:1006E000E9F10E946C808823C9F1A0917808B0914B
:1006F000790852961C921E92519754961C921E9203
:10070000539784E890E01D969C938E931C971E96B9
:100710001C921E9780E090E350969C938E931F97B7
:10072000ED91FC9111970088F189E02D6CE070E06B
:10073000CD011995BE016F5F7F4F80917808909130
:1007400079080E9422808091780890917908DC01D4
:10075000ED91FC910488F589E02D199569817A81E4
:100760008B819C810F900F900F900F90DF91CF9114
:1007700008950F931F93CF93DF9300D01F92CDB7AF
:10078000DEB769837A838B839C838091780890910C
:100790007908892B11F480E049C00E946C8088237D
:1007A000D1F3A0917808B091790852961C921E92CC
:1007B000519754961C921E92539784E890E01D9690
:1007C0009C938E931C971E961C921E9780E090E33C
:1007D00050969C938E931F97ED91FC9111970088F2
:1007E000F189E02D6CE070E0CD01199580917808D9
:1007F00090917908DC01ED91FC910280F381E02D6C
:1008000044E050E0BE016F5F7F4F19958C018091ED
:10081000780890917908DC01ED91FC910488F589C4
:10082000E02D199581E0012B09F4B5CF0F900F90C1
:100830000F900F90DF91CF911F910F910895CF935B
:10084000C82F0E945F83677FC0FF6860CF910C94C0
:10085000B983CF93C82F0E945F83C770687F6C2BCA
:10086000CF910C94B983CF93C82F0E945F83C77038
:10087000C295C07F6F786C2BCF910C94B9830F9386
:100880001F93CF93DF938B01FC01C681D781209703
:1008900059F0B801888199810E94A8BE892B21F066
:1008A0000A80DB81C02DF3CFCE01DF91CF911F9164
:1008B0000F91089561157105C1F0DC011696ED9157
:1008C000FC911797309731F417967C936E93169797
:1008D0000895FC01828193810097D9F77383628325
:1008E000DB011596FC93EE93149708952AE00C947F
:1008F0003F6E462F50E070E060E02AE00C943F6EBF
:10090000AB01770F660B770B2AE030E00C94966E04
:10091000FC0186819781009739F0662329F06150A8
:10092000FC0182819381F7CF0895CF93DF93EC018F
:10093000FA013296E60FF71FDC019D012C1B3D0BDF
:10094000CF01861B970B4D91442311F04193F5CFB6
:10095000AC01421B530B640F751FFB0132973083B0
:1009600061507109FB012083DF91CF91089580913F
:100970001F0890912008009711F480E02FC0DC013F
:10098000ED91FC910688F789E02D19952091420898
:100990003091430881111FC0232B79F78DEF9FEF12
:1009A000909343088093420880911F0890912008FB
:1009B000DC01ED91FC910680F781E02D1995809185
:1009C0001F0890912008DC01ED91FC910488F589C5
:1009D000E02D1995D2CF81E0232B79F60895DC0123
:1009E0001696ED91FC9180E0309729F08F5F0280A0
:1009F000F381E02DF9CF0895CF93DF93FC01C281FD
:100A0000D3812097C1F088858F70823029F4898541
:100A10009A85DF91CF910895853069F4CE010E94C7
:100A2000EF84882341F060E0CE010E948884FC01BD
:100A300081859285EECF90E080E0EBCFDF92EF9260
:100A4000FF920F931F93CF93DF93EC017B0140E064
:100A500052E00E94852FD82E811171C066E97CE199
:100A60008CE499E00E94826FD70119968D919C9138
:100A7000009709F441C0DC01ED91FC91028CF38DEB
:100A8000E02D19958C0180E00231110520F4F80168
:100A9000EF57FD4F8081982F9295907F89818F70BD
:100AA000892B89836BE87CE18CE499E00E94826F5A
:100AB000B8018CE499E00E94808463E87CE18CE4D6
:100AC00099E00E94826F698162956F708CE499E071
:100AD0000E9479848CE499E00E948B6E89818295D2
:100AE0008F70843068F4823098F58130B9F11C82BF
:100AF0001D821E821F8215C0F701008510E0C3CF42
:100B0000883039F0893099F780E090E0A6E9B2E4C6
:100B100004C080E090E0A0EAB1E48C839D83AE83C2
:100B2000BF8340E052E0B701CE010E941D2FCE01ED
:100B30000E944E2A60E07AE0C7010E9495308D2D18
:100B4000DF91CF911F910F91FF90EF90DF9008956B
:100B500084E68E838F818E7F8F831D828FEF8C83BF
:100B6000E0CFCF92DF92EF92FF92DC011196EC91F1
:100B70001197E295EF70EC3098F4F0E08827EC5391
:100B8000FA478F4F0C9470BA2786EA85EA85D0859C
:100B9000D085D0850D86EE85D085D085D785D78543
:100BA0008FEF9FEFFF90EF90DF90CF900895149616
:100BB0008D919D910D90BC91A02DB7FD48C08F3FA8
:100BC0009105A105B10571F36CF38FEF90E0A0E002
:100BD000B0E0E8CF14968C9190E0E4CF1496CD90DD
:100BE000DD90ED90FC90179720E030E0A901C7015F
:100BF000B6010E949BB887FD2AC020E030E04FE795
:100C000053E4C701B6010E94A3BB18161CF1C7012B
:100C1000B6010E946DBBCB01C5CF14966D917D913D
:100C20008D919C911797673F2FEF7207820792076C
:100C300074F061152AE07207810591055CF42AE0E1
:100C400030E040E050E00E9407BAC901ABCF90E02D
:100C500080E0A8CF8FEF90E0A5CFCF92DF92EF9208
:100C6000FF920F931F93CF93DF9300D000D0CDB7A7
:100C7000DEB78C016C0188E0C80ED11C30E1E32E98
:100C8000F12CF80181918F0190E024E095958795F2
:100C90002A95E1F7092E000CAA0BBB0B89839A83D6
:100CA000AB83BC83FE82ED82BE016F5F7F4F8BE919
:100CB00098E00E94F458F801319780818F7090E09D
:100CC000B0E0A0E089839A83AB83BC83FE82ED828F
:100CD000BE016F5F7F4F8BE998E00E94F4580C15BE
:100CE0001D0579F626960FB6F894DEBF0FBECDBF70
:100CF000DF91CF911F910F91FF90EF90DF90CF90F8
:100D000008954F925F926F927F928F929F92AF92CF
:100D1000BF92CF92DF92EF92FF920F931F93CF93E8
:100D20006B017C01742EAC019B010E9403BC68E640
:100D300075E0811126C046015701E894B7F82FEFFE
:100D40003FEF4FE75FE7C501B4010E9403BC81118B
:100D50000CC02FEF3FEF4FE75FE7C501B4010E94E2
:100D60009BB86CE675E0181664F02FEF3FEF4FE785
:100D70005FE4C701B6010E94A3BB1816ACF460E79C
:100D800075E08CE499E0CF911F910F91FF90EF9067
:100D9000DF90CF90BF90AF909F908F907F906F909B
:100DA0005F904F900C94306E2FEF3FEF4FE75FEC6A
:100DB000C701B6010E949BB887FDE1CF20E030E07B
:100DC000A901C701B6010E949BB810E000E087FFAF
:100DD0000AC06DE28CE499E00E948F6E8C01F7FAF4
:100DE000F094F7F8F094C0E060E070E080E09FE3FA
:100DF0007C1641F020E030E040E251E40E94FBBA72
:100E0000CF5FF6CFA70196010E948FBA2B013C015C
:100E10000E9474BB4B015C012AE0BC01A4018CE47C
:100E200099E00E943F6E7C01E00EF11ECC23D1F1CF
:100E3000C501B4010E94A0B89B01AC01C301B2017D
:100E40000E948EBA4B015C016EE28CE499E00E9434
:100E50008F6EE80EF91EC15028F120E030E040E22C
:100E600051E4C501B4010E9401B92B013C010E946B
:100E700074BB4B01B12CA12C2AE0B501A4018CE478
:100E800099E00E943F6EE80EF91EC501B4010E9470
:100E9000A0B89B01AC01C301B2010E948EBA4B0104
:100EA0005C01D9CFC701CF911F910F91FF90EF90B7
:100EB000DF90CF90BF90AF909F908F907F906F907A
:100EC0005F904F9008950F931F93CF93DF93EC01A2
:100ED000209731F10A811B8188858295807F8595D5
:100EE00085958595859583FD06C08E819F810097A8
:100EF00011F00E94638788858F70843031F4898572
:100F00009A85009711F00E94AAAE88819981009776
:100F100011F00E94AAAECE010E94AAAEE801D8CF7D
:100F2000DF91CF911F910F9108950F931F93CF934E
:100F3000DF938C010E941D73EC01892B71F0C801B5
:100F40000E944072BE01C8010E94097D019629F4E9
:100F5000CE010E946387D0E0C0E0CE01DF91CF9147
:100F60001F910F9108958CBD9DBD0895CF93C82FFB
:100F7000462F61E070E00E94F91A61E070E08C2F6A
:100F80000E94031B8111F9CFCF910895CF93DF9376
:100F9000EC018AE793E0998388831A821B821C8282
:100FA0001D8280E590E00E94B387BE016E5F7F4F97
:100FB00044E050E08FE090E00E9424740E947B1B8C
:100FC000CE01DF91CF910895EF92FF920F931F937F
:100FD000CF93DF9300D01F92CDB7DEB71092690791
:100FE00002967C0110E000E0F70181917F014AE068
:100FF000BE016F5F7F4F90E00E94B7B140E150E0CB
:10100000BE016F5F7F4F89E697E00E94E1BE03302B
:10101000110531F060EB74E089E697E00E94BBBEF9
:101020000F5F1F4F04301105F9F689E697E00F9026
:101030000F900F900F90DF91CF911F910F91FF9024
:10104000EF900895AF92BF92CF92DF92EF92FF920E
:101050000F931F93CF93DF931F921F92CDB7DEB7ED
:101060007A836983BA01A901E981FA81F770082FAF
:1010700010E0000F111F0F57184FD8018D919C9150
:101080008E0F9F1F9F01240F351F21303840A0F085
:101090005A016B0160E078E07B01EE1AFF0AA701BC
:1010A000B6010E942474A5014E195F09B6016E0DA8
:1010B0007F1DF801808191810F900F90DF91CF917A
:1010C0001F910F91FF90EF90DF90CF90BF90AF9066
:1010D0000C9424748F929F92AF92BF92CF92DF9222
:1010E000EF92FF921F93CF93DF93182F7B014A015A
:1010F000590164E270E00E94031BC82E65E270E0B3
:10110000812F0E94031B9C2DE80EF91E970137705A
:10111000C12ED12CCC0CDD1CC6018758984F6C0118
:10112000FC0180819181820F931FA9014A0D5B1DF3
:101130004130584060F1C0E0D8E0C21BD30BAE0193
:10114000B4010E945474A5014C1B5D0BB4016C0FDB
:101150007D1FF601808191810E945474EA0CFB1C72
:101160004F2D64E270E0812F0E94F91A4E2D65E246
:1011700070E0812FDF91CF911F91FF90EF90DF9072
:10118000CF90BF90AF909F908F900C94F91AA501CB
:10119000B401E2CFFF920F931F93CF93DF93F82E0A
:1011A00010E000E08F2D0E940A74EC01892B21F0E1
:1011B0008F2D0E940A748C01C017D10799F7CE01B8
:1011C000DF91CF911F910F91FF90089520E3FC01D3
:1011D00020833296862F82958F706F706A3030F43C
:1011E000605D6293682F8111F5CF0895695CF9CF36
:1011F0008150823108F05AC0E82FF0E08827EC5F78
:10120000F6478F4F0C9470BA2489288916891C8957
:10121000208956892B89318935893B893F894389C2
:1012200049894D895689518957895B898091800008
:101230008F77809380000895809180008F7DF9CF13
:1012400080918000877FF5CF84B58F7784BD089526
:1012500084B58F7DFBCF8091B0008F778093B000F5
:1012600008958091B0008F7DF9CF809190008F77A5
:10127000809390000895809190008F7DF9CF8091A8
:101280009000877FF5CF8091A0008F778093A0009A
:1012900008958091A0008F7DF9CF8091A000877F75
:1012A000F5CF809120018F77809320010895809160
:1012B00020018F7DF9CF80912001877FF5CF1F938B
:1012C000CF93DF93282F30E0F901E75BF64E84914E
:1012D000F901E755F64ED491F901E151F64EC4916A
:1012E000CC23A9F0162F81110E94F888EC2FF0E092
:1012F000EE0FFF1FE15DF64EA591B4918FB7F89404
:10130000EC91111108C0D095DE23DC938FBFDF91E3
:10131000CF911F910895DE2BF8CFCF93DF9390E00C
:10132000FC01E755F64E24918151964EFC018491C3
:101330008823C9F090E0880F991FFC01E157F64E11
:10134000A591B491FC01E15DF64EC591D491611176
:101350000DC09FB7F8948C91209582238C9388813F
:10136000282328839FBFDF91CF910895623051F4E5
:101370009FB7F8943C91822F809583238C93E881CA
:101380002E2BEFCF8FB7F894EC912E2B2C938FBF91
:10139000EACF863308F0865320917B00982F98700F
:1013A000277F922B90937B008770806480937C00D2
:1013B00080917A00806480937A0080917A0086FD23
:1013C000FCCF809178009091790008953FB7F89410
:1013D0008091940990919509A0919609B0919709EF
:1013E00026B5A89B05C02F3F19F00196A11DB11D80
:1013F0003FBFBA2FA92F982F8827BC01CD01620FBC
:10140000711D811D911D42E0660F771F881F991F76
:101410004A95D1F708958F929F92AF92BF92CF9243
:10142000DF92EF92FF920F931F93CF93DF93D091B0
:10143000D907D13208F0D7C0182FC091D8070E9421
:10144000E6896B017C018091B00781116BC082E05D
:101450008093B0071093AF078FEF8093AE07109281
:10146000AD07D093AC07A8EBB7E0ECE8F7E080E07D
:10147000D81391C010928B0780918B07CC0FC82B8B
:10148000C0938B0780918A07813009F088C0109241
:101490008A070E94E6896B017C0180918B0780930B
:1014A000BB008091B2079091B307A091B407B091AF
:1014B000B507892B8A2B8B2BA1F00E94E68900911E
:1014C000B2071091B3072091B4073091B5076C199A
:1014D0007D098E099F09061717072807390708F4A1
:1014E00042C08091BC0083FDD8CF85EC8093BC00C6
:1014F0000E94E6896B017C018091B007823009F47B
:1015000050C08091AE078F3F09F46FC08091AE0745
:10151000803209F46CC08091AE07803309F469C051
:1015200084E026C08091B2079091B307A091B407E0
:10153000B091B507892B8A2B8B2B09F484CF0E949D
:10154000E6898090B2079090B307A090B407B0905E
:10155000B5076C197D098E099F0986169706A8069E
:10156000B90608F070CF8091B1070E94841D85E014
:101570001092B7071092D9071092B607DF91CF915A
:101580001F910F91FF90EF90DF90CF90BF90AF90A1
:101590009F908F9008959D9191938F5F69CF85EE75
:1015A000A5CF8091B2079091B307A091B407B091F5
:1015B000B507892B8A2B8B2B09F49ECF0E94E689D5
:1015C0000091B2071091B3072091B4073091B5078D
:1015D0006C197D098E099F09061717072807390717
:1015E00008F08ACFC0CF81E0C3CF80E0C1CF82E0D6
:1015F000BFCF83E0BDCF81E00C940B8A8F929F9286
:10160000AF92BF92CF92DF92EF92FF926B017C017B
:101610000E94E6894B015C01C114D104E104F1048C
:10162000B9F00E94E689681979098A099B09683E20
:1016300073408105910580F321E0C21AD108E108C9
:10164000F10888EE880E83E0981EA11CB11CE4CF3F
:10165000FF90EF90DF90CF90BF90AF909F908F90D2
:101660000895DF92EF92FF920F931F93CF93DF9332
:1016700000D000D000D0CDB7DEB78C017B01AE0129
:101680004F5F5F4F0E946E20D82E882309F459C007
:10169000F7018081803109F454C08FE78D83F80110
:1016A000858196810E94EA1EB701F80185819681A5
:1016B0000E94FA1F40E06EE4F801858196810E9445
:1016C000371F40E06B81F801858196810E94371FAA
:1016D00040E06C81F801858196810E94371FF701F7
:1016E0008081803139F040E06D81F80185819681FB
:1016F0000E94371FF801858196810E94EA1EB7017A
:10170000F801858196810E94FA1FF801408168E402
:10171000858196810E94371F64E170E080E090E04F
:101720000E94FE8AF8018081882331F06AE070E02F
:1017300080E090E00E94FE8AF801858196810E94F7
:10174000EA1E8D2D29960FB6F894DEBF0FBECDBFD1
:10175000DF91CF911F910F91FF90EF90DF9008954F
:10176000CF936CE271E080E090E00E94FE8ACFB7F8
:10177000F89480919809811127C0E4E2FAE18491FC
:10178000EEEDF9E19491E82FF0E0EE0FFF1FE15745
:10179000F64EA591B491EC91E92321F461E085E343
:1017A0000E945F8961E085E30E948D898CB580612C
:1017B0008CBD8CB580648CBD61E084E30E948D8912
:1017C00061E083E30E948D89809198098F5F809307
:1017D0009809CFBF249A80E590E00E94B38767E024
:1017E00090E080E00E94837465E58BE190E00E94C8
:1017F000837465E58AE190E00E9483740E947B1BFC
:1018000080E090E490937A078093790780E090E6F7
:10181000909382078093810780E098E490937C07FF
:1018200080937B0780E098E69093840780938307FA
:1018300080E090E590937E0780937D0780E090E7BD
:10184000909386078093850780E098E590938007C2
:1018500080937F0780E098E79093880780938707BD
:10186000CF910895CF92DF92EF92FF920F931F9343
:10187000CF93DF936C01EB017A0189010E94B08B59
:1018800080E590E00E94B38746E050E060E878E0B1
:1018900089E090E00E945474C60102960E94661B83
:1018A000C70102960E94741BC80102960E946D1B1C
:1018B0000E947B1B8A819B81AC81BD81809309083A
:1018C00090930A08A0930B08B0930C08DF91CF9176
:1018D0001F910F91FF90EF90DF90CF900895CF92DE
:1018E000DF92EF92FF92CF93DF93CDB7DEB7689789
:1018F0000FB6F894DEBF0FBECDBFFA012AE733E082
:101900003A8329835FEF5B835C835D831E82388724
:101910002F83C280D380E480F580C986DA86EB8687
:10192000FC863E872D87FB0142815381648175814E
:101930004F87588B698B7A8B3C8B2B8BFC01828178
:101940009381A481B5818D8B9E8BAF8BB88F9E01C7
:101950002F5F3F4FAE01495F5F4FBE01635F7F4F17
:10196000CE0143960E94328C68960FB6F894DEBF83
:101970000FBECDBFDF91CF91FF90EF90DF90CF9062
:1019800008950F931F93CF93DF93CDB7DEB768977A
:101990000FB6F894DEBF0FBECDBFFB01DC0112967F
:1019A0004D915D916D917C9115974D8B5E8B6F8BF9
:1019B000788F8AE793E09A83898321E0288F0D89C5
:1019C0001E892F89388D0B831C832D833E83988736
:1019D0008F83028113812481358109871A872B87A0
:1019E0003C879E878D874F87588B698B7A8BAE019A
:1019F0004F5F5F4FBE01695F7F4FCE010D960E9422
:101A00006F8C68960FB6F894DEBF0FBECDBFDF9126
:101A1000CF911F910F910895CF93DF93CDB7DEB78C
:101A200062970FB6F894DEBF0FBECDBFFC01828176
:101A30009381A481B5818F87988BA98BBA8B2AE774
:101A400033E03A83298341E04A8B4F85588969897D
:101A50007A894B835C836D837E8338872F83898764
:101A60009A87AB87BC87BE016F5F7F4FCE01079619
:101A70000E94C18C62960FB6F894DEBF0FBECDBF38
:101A8000DF91CF9108952FB7F894609190097091EC
:101A9000910980919209909193092FBF0895EF9237
:101AA000FF920F931F93CF93DF9300D01F92CDB778
:101AB000DEB7FA0120E08E010F5F1F4F9E2F9F7748
:101AC000EE0FEF2FEE1FFF0BF195309709F09068A6
:101AD000D801A20FB11D9C932F5F309779F730E0AA
:101AE000FB01E21BF30B8483FB01E21BF30B359636
:101AF000D801CD01801B910B821793071CF48D91A7
:101B00008193F7CF2F5F3F4F80911F08909120085E
:101B10008901040F151F621B730B6B5F7F4FDC0184
:101B2000ED91FC910280F381E02DA80119957C01D3
:101B30000E94438D60932B0870932C0880932D088E
:101B400090932E0881E00E151F0509F080E00F909C
:101B50000F900F900F90DF91CF911F910F91FF90F9
:101B6000EF900895AF92BF92CF92DF92FF920F93C2
:101B70001F93CF93DF936C01EB018A01F22E0E9439
:101B8000B784882309F442C0A0902308B0902408A9
:101B9000B501C6010E9485B19801295F3F4F820FB0
:101BA000931FA816B90690F1609121087091220840
:101BB00045E050E0C6010E949584AC019E01200FD3
:101BC000311FFE01EC01CE1BDF0BDE01AE0FBF1F8C
:101BD0006091210870912208E217F30729F08191A2
:101BE000A60FB71F8C93F1CF0550110980E3F110B8
:101BF00081E3400F511FDF91CF911F910F91FF9013
:101C0000DF90CF90BF90AF900C944F8D80E0DF912C
